:109B7500414952434F544543004256332E35302018
:109B8500504F52004241542000532F4E2146414927
:109B95004C555245005245454E54455221532F4E82
:109BA50000434F4E5441435420414952434F54457D
:109BB5004300475053004032444000403344400086
:109BC5004F464621564F4F404D454E55000A16000B
:109BD5000180000300007E0000FE00001E0000362C
:109BE5000003E60001C4000000000FFFE050524FE3
:109BF50043555240534154530043414C4940414C15
:109C0500542020230053454C4543414F20005445E3
:109C15004C4153202020004D415041202020200060
:109C250043454E54524F202000564152494F202063
:109C350020004241524F4752414600524F54415332
:109C45002020200050524F58494D20200050494CAB
:109C5500614F202020004D4152434F532020004F9B
:109C6500524947494E414C00202020214D45442171
:109C7500202020204449530020545241434B214C7D
:109C85004947200020545241434B2144455320006D
:109C95004D41524B00545241434B2D4143494D20B8
:109CA500004E4F5254482D4143494D200021534108
:109CB50049522020200153454C4540524F54410103
:109CC500414A55535420414C545501564F4F53204A
:109CD500202020686901564F4F5320544F4468692E
:109CE5000150494C614F202020686901524F544171
:109CF500532020206869014149525350414345682A
:109D05006901434F4E4649475552686900414A55D6
:109D1500535420414C5455004241524F4740414C09
:109D250054550047505320414C5455524100514E13
:109D35004820202020402148504100464C004C4FEF
:109D450047564F4F2056415A494F20003E21534117
:109D5500495220202000534149522020014D4F53A4
:109D6500545241015452414E5346014150414741DD
:109D75005200215341495220202001434F4D3A20A2
:109D8500202020202001544E432031232035374BFD
:109D950001544E4320312320392E360101505743BB
:109DA500403130234035374B015057434031302344
:109DB5004031394B01014D58504031302340353742
:109DC5004B014D58502034232035374B014D585009
:109DD5002031232035374B014D5850403130234039
:109DE50031394B014D58502031232031394B002159
:109DF50053414952202020014E4F564F2050494C87
:109E0500614F014D4F44492050494C614F0141502C
:109E150041472050494C614F0101434F4D3A015292
:109E25004543452050494C614F01454E5649205008
:109E3500494C614F01454E564940544F444F5301DB
:109E4500014449532050492D504920014150414773
:109E550040544F444F532000444952202144495314
:109E650054004752415620004C4F43414C4041431A
:109E75005455414C00475241564152202020200064
:109E85002053544F52452157505420002046554CDD
:109E95004C2000214041504147415220005345523A
:109EA500200049522020005553422000555342209E
:109EB500004C49535400454E564900204552524FD7
:109EC500205452414E534D495420200021534149BD
:109ED500522020200153454C4540524F54410149E1
:0D9EE5004E532050494C614F20014D4F4419
:109EF200494620524F544101494E56455220524F35
:109F0200544101415041472050494C614F01415059
:109F120041472020524F54410143594C2052414461
:109F220049555301434F4D3A015245434542205250
:109F32004F544101454E56494120524F544101432D
:109F42004845434B20524F0053454C4521524F54F4
:109F520041004E4F564F0020414C54404F52444016
:109F6200210021494E5645525445524000494E5611
:109F72004552540021404150414740505453002122
:109F82004150414720524F54004D454D20434845D2
:109F9200494120002140454E5640524F5441002035
:109FA20020524144495553002153414952014341F2
:109FB200524043545221504320015645524043548B
:109FC20052202020014150414740544F444F5320DA
:109FD2000101434F4D3A0152454345424520435406
:109FE2005201454E56494152204354520056455261
:109FF2002043545220004D4F5645522020004D4FD1
:10A00200564552205041524100455343414C412054
:10A0120020582F5920534149520041504147204472
:10A022004953004155544F204C4947004445534C35
:10A032004947414E444F002020205A4F4F4D004483
:10A04200495354204B4D0044495354204E4D002156
:10A052005341495220202001564152494F2020208D
:10A0620068690158432D434F4E464968690152546D
:10A07200412D434F4E46686901474552414C2020CD
:10A082002068690154454C41202020206869010163
:10A09200014D4F442E464143494C01434F4E462009
:10A0A200464142524901544553544520564F4F01AF
:10A0B20041504721544F4421564F4F0021534149AB
:10A0C2005220202001534F4D4445534301444553F0
:10A0D20043212D014D4F44404445534301494E56BF
:10A0E20040444553430153454E564152402020407F
:10A0F2002301564F4C554D450143414C4920564191
:10A1020052494F01544F4E45200146524551554543
:10A112004E43015641522041564020304023014EC9
:10A122004554544F2D0154455354415220534F4DE1
:10A132000053444553434C49470053444553434419
:10A142004553004E414F204455414C0043414C4938
:10A1520020564152494F00455350455241522031F9
:10A1620030204D494E202000414E5445532043415A
:10A172004C49425241522000215341495220202051
:10A182000143414D494E484F20014155544F4345EB
:10A192004E5401014D45442F444953200146494E36
:10A1A2004553534520014C2F44010156454E54213D
:10A1B200542D55500143454E5421542D55500157AD
:10A1C20041595054214252470021534149522020C3
:10A1D2002001484F5240494E4943494F015052498C
:10A1E2004D45014652455155203A015154444520AE
:10A1F200202020202001554C54494D0143594C53F5
:10A20200494740202040230153454C40524F54417E
:10A21200200101010143594C520143594C20542D54
:10A2220055500021534149522020200101554E49E9
:10A232005401434C49434B40302C40202301434FAF
:10A242004E5452415354014E4D4541213138330150
:10A25200494D50454C4C455201494D502D43414CBE
:0DA2620001432D564152494F015445432000
:10A26F00202040303040250141004E4F20414750C3
:10A27F00532F464C00414C54492D4750532020003A
:10A28F00464C47542D4C4556454C004147505320A2
:10A29F003C3E20464C0040574159504F494E5420A8
:10A2AF004558495354204000574159504F494E5437
:10A2BF00002053414952202020210052454345425E
:10A2CF004552004C49565240003C2D204C495354A6
:10A2DF00202D3E2020455849540053454C004E45F3
:10A2EF005854005450542050524F5800545054203A
:10A2FF00414E54450041504720404C454700415086
:10A30F00472040534F4D004445532020202020200C
:10A31F00202000204445530046414C4841475053AC
:10A32F0020200020475241564152202000524F54C6
:10A33F004120004D4150524F58004C495354410059
:10A34F0045544500414C54403000524F5441205623
:10A35F00415A49410020544F4F404D55434820002A
:10A36F00214053454C404C495354002053454C40D9
:10A37F0057505440210021405245434542455240D9
:10A38F00002020404F204B40202021004F4B0056F3
:10A39F004152004649580047415445215800504FFB
:10A3AF004E544F504152544900535443594C20007E
:10A3BF00404445530054502000406A40494E20000D
:10A3CF004067404F5554002046414C4841202021C2
:10A3DF00002053414952004D4F44490059404540D8
:10A3EF0053004D4F444920204E4F5620475241565F
:10A3FF0041520050524F5820202053454C2020539B
:10A40F00414952005843542D464C49474854200067
:10A41F005553454400454E54455220004D4D2E4D49
:10A42F004D4D20004D4D2753532E53005747532169
:10A43F003834002040554054404D40200055405482
:10A44F00404D002055544320004C4F43414C005386
:10A45F0057495353474400414C54005355494058B2
:10A46F000041564740203040230035303000313610
:10A47F00343000205D203130404B632F70005D2061
:10A48F0020203140632F2300205D202035404B5486
:10A49F0053005D203230304046504D004063402025
:10A4AF004B63004654204B6300406340204E4D00E9
:10A4BF004654204E4D004D2F53003230305E003544
:10A4CF0030305E003122003222003322003522006C
:10A4DF00382200464C3700464C313600464C333359
:10A4EF0000464C36350046313030004631363000AC
:10A4FF0046323630005E252640534F47005E2526F4
:10A50F004054415300414C540056415200225E2F9B
:10A51F0024004B545300532F4E002224004B540061
:10A52F00225E004E4D00302C3500312C3000322C85
:10A53F003000302C3600312C3200322C3500332CC9
:10A54F003800372C3500403135004033300040366D
:10A55F0030005441534B00464C2D44415445005458
:10A56F005000544F46005354410046494E004C4151
:10A57F004E00534554204F464653455400495341CE
:10A58F0020484549474854004155544F2D474F20C7
:10A59F000053544152540020434845434B40414CD3
:10A5AF004C005241442044495354004053454C40C1
:10A5BF004845494748543A00475053404241524F4B
:10A5CF0040414C4C0053494E4B40312D3221632FAB
:02A5DF00230057
:1063FC00304D2475A7049005C2E0F51CE0F51DE0B6
:10640C00F51EE0F51FE0F56DE0F56EE0F56FE0F5DB
:10641C0054126FBE1269FC2275C70375C6E475B9B8
:10642C0001E5BCB48143126FBE1255E48E628F63DA
:10643C007568F97569001264D2203C2D203B2B1233
:10644C0066071265DB856D1C856E1D856F1E855478
:10645C001F12653E203C12203243201D231266077A
:10646C001269FCE532242850DC2212653E203CF9EE
:10647C00203DF6203205201DBD80EF301DB880EA8E
:10648C001266071269FC856D1C856E1D856F1E8555
:10649C00541F1265F11269FC203DCE809912682AB6
:1064AC00201D0D755310740012678D203DBB808626
:1064BC00E553540FC553C4540F2035051266A28002
:1064CC000312678D808BC23CD23B12658EFD126528
:1064DC008EFC12658EC39573F565EC9574F564EDC1
:1064EC009575600504600A800EE56424E050118007
:1064FC0006E5642420400912658E12658E02658EB5
:10650C0012658EFD12658EFC12658EC39576F5674D
:10651C00EC9577F566ED9578600904600122E566E7
:10652C00F48002E5668562F0A474E025F04002C2B6
:0D653C003B22C23C12658EA2E7923DA2E612
:10654900921DA2E592324026A2E492E592E692E7F4
:10655900FC12658E2565F565EC3564F56412658E6A
:10656900FC12658E2567F567EC3566F56622A2E4AF
:106579009235540F79C6F712658E09F7301D051249
:10658900658EF55322E5697023E56860302404407F
:106599002CE56875F004A485F0C7F5C675B901E561
:1065A900BCB4811985BD68756902801E54037010D9
:1065B90005C675B901E5BC056953690F22D23C22AC
:1065C900147004E5BD80F0147004E5BE80E9E5BFF0
:1065D90080E575A7009006F6E56DF0A3E56EF0A3DA
:1065E900E56FF0A3E554F02275A7009006F6E0F5F3
:1065F9006DA3E0F56EA3E0F56FA3E0F55422E56421
:10660900B2E7F56D85656EAB67E566FC30E707C3F4
:10661900E49BFBE49CFCAA62A9631252E4E56630A0
:10662900E707C3E49DFDE49EFEEEB2E7F56F8D54E6
:106639002275380C1268931268DED5530122753819
:106649000C1268641268D4D5530122753800126897
:0E6659007C1268A3D5530122753800126864C4
:106667001268A3D553012275380312689312690F74
:10667700D5530122753803126864126905D5530191
:106687002275380F12687C126934D5530122753888
:106697000F126864126934D55326229066A72373B4
:1066A7008091807780688059804A803B802C801D4C
:1066B700800E80DA80CB80BC80AD809E808F80800A
:1066C700753815126893126956D553012275381516
:1066D70012686412694BD553012275380912687C18
:1066E70012691CD553012275380912686412691C96
:1066F700D55301227538061268931268C6D553011F
:10670700227538061268641268BBD55301227538A2
:106717001212687C1268ECD5530122753812126880
:10672700641268ECD553012202663A75381512686F
:1067370093126956D553012275380F12686412698E
:1067470034D553012275380F12687C126934D5533A
:106757000122753803126864126905D55301227541
:10676700380312689312690FD55301227538001246
:1067770068641268A3D553012275380012687C1229
:1067870068A3D55326229067922373809E80A980A1
:10679700B480BF80CA80D580E08010801B802680AF
:1067A70031803C80478052805D806875380C126864
:1067B700641268D4D553012275380C126893126895
:0E67C700DED55301227538121268641268EC98
:1067D500D553012275381212687C1268ECD5530125
:1067E500227538061268641268BBD55301227538C4
:1067F500061268931268C6D55301227538091268C6
:106805006412691CD553012275380912687C126916
:106815001CD553012275381512686412694BD5537E
:10682500012202673278C686040886037AED125281
:10683500A278CAA60408A60378C686040886037A41
:10684500621252A278CCA60408A60378C68604086C
:1068550086037AB51252A278C8A60408A603227543
:106865001A6A751B0A78CA8618088619126AA778E3
:10687500CC86060886072278C88618088619E4F5A6
:106885001AF51B126AA778C886060886072278C6F5
:106895008618088619751A00751B01026AA7E51D79
:1068A5002519F51DE51C3518F51CC3E51F9FF51FBA
:1068B500E51E9EF51E22C3E51F9FF51FE51E9EF5ED
:1068C5001EC3E51D9519F51DE51C9518F51C22E55A
:1068D5001D2FF51DE51C3EF51CC3E51F9519F51F7C
:1068E500E51E9518F51E22C3E51D9FF51DE51C9EA9
:0968F500F51CC3E51F9519F51F00
:1068FE00E51E9518F51E22E51F2FF51FE51E3EF528
:10690E001EE51D2519F51DE51C3518F51C22C3E5E0
:10691E001D9519F51DE51C9518F51CE51F2FF51F86
:10692E00E51E3EF51E22E51D2FF51DE51C3EF51C50
:10693E00E51F2519F51FE51E3518F51E22C3E51DA9
:10694E009FF51DE51C9EF51CE51F2519F51FE51E7F
:10695E003518F51E22E51A7009E51B70058C068D9B
:10696E000722ED851BF0A4A2F792D5ED851AF0A4AF
:10697E00AEF0FFEC851BF0A4A2D53FEE35F0FF92F2
:10698E00D5EC851AF0A42FFFE435F030D50104FEC6
:10699E0022E4F51AF51BEF4E7003051B22EF651965
:1069AE007006EE65187001227808C3EF33FFEE33E0
:1069BE00FEEF9519F5F0EE95184003FEAFF0E51ACF
:1069CE0033F51AD8E5F4F51A751BFF7805C3EF33C6
:1069DE00FFEE33FEEF9519F5F0EE95184003FEAF7E
:0369EE00F0E51BB6
:1069F10033F51BD8E5F4C403F51B22E51D9511E51C
:106A01001C9510500BE56E9511E56D951050012206
:106A1100E51F9511E51E9510500BE5549511E56F95
:106A21009510500122E51D9513E51C9512400BE5CB
:106A31006E9513E56D9512400122E51F9513E51E34
:106A41009512400BE5549513E56F951240012253C1
:106A51002CF8C3E51F9554FFE51E956FFE9260501B
:106A610007C3E49FFFE49EFEC3E56E951DF519E59E
:106A71006D951CF5189261500BC3E49519F519E455
:106A81009518F518C3E5199FE5189E9262500AE51D
:106A910018CEF518E519CFF51912699FE52C5407A1
:106AA10075F003A4F538E538906AAD73026AC50242
:106AB1006AD9026AE7026AFF026B12026B25026B56
:106AC10033026B4B851C16851D17C3E4951FF51505
:106AD100E4951EF514026B5E851C16851D17851E37
:106AE10014851F158077C3E4951DF517E4951CF5F2
:106AF10016C3E4951FF515E4951EF514805FC3E4F4
:056B0100951DF517E4ED
:106B0600951CF516851E14851F15804CC3E4951F2C
:106B1600F517E4951EF516851C14851D1580398517
:106B26001E16851F17851C14851D15802BC3E4951D
:106B36001FF517E4951EF516C3E4951DF515E495A6
:106B46001CF5148013851E16851F17C3E4951DF5C5
:106B560015E4951CF5148000C3E5179513E5169505
:106B66001210D70122E5159513E514951210D701D9
:106B760022E519F92517FFE518F83516FED3EF9526
:106B860011EE9510500122E5119517FDE5109516A9
:106B9600FC402A4D6027126963E5152FF515E514AB
:106BA6003EF514E5159513E514951210D70122E567
:106BB600199DF9E5189CF8851016851117E5172912
:106BC600FFE51638FEE5139FE5129E500BC3E5134D
:106BD6009517F9E5129516F8E51A700AE51B700681
:106BE600AA00AB018013E9851AF0A4E5F0FBE8855D
:106BF6001AF0A42BFBE435F0FAE5152BFBE5143A65
:066C0600FAE5119BE51008
:106C0C009A10D70122EB9515FDEA9514FCC3E515F6
:106C1C009511E514951010D717E5139BE5129A50B2
:106C2C0036E5139515FFE5129514FE126EDB8027E1
:106C3C00EB9511FFEA9510FEAA00C001126EDBD095
:106C4C0003E5172BFBE5163AFAEB99F517EA98F5DD
:106C5C0016851115851014C2D5E5466002D2D5AA49
:106C6C0056E98AF0A4ABF0E88AF0A42B30D5047571
:106C7C00F00384F8700122E5172513FDE516351293
:106C8C00FCED8AF0A4ABF0EC8AF0A42B30D50475A3
:106C9C00F00384FEE5152513FDE5143512FCED8A91
:106CAC00F0A4ABF0EC8AF0A42B30D50475F003847F
:106CBC00F9E538906CC373026CDB026CE7026CF084
:106CCC00026CF9026CFF026D0B026D12026D17C3A0
:106CDC00743E9EFFC3743E99FE8032C3743E9EFF89
:106CEC00AE018029AF06C3743E99FE8020AF06AE7C
:0D6CFC0001801AC3743E9EFEC3743E99FFD2
:106D0900800EC3743E99FF8007C3743E9EFEAF0197
:106D190008EF2437FFE51B7007E51A700CE8800EB1
:106D2900A2E7E51A50030460F488F0A4E5F06001D5
:106D390004F923FA98FBC3E998C333F9906D4BE53D
:106D49003873026D63026D90026DC5026DF2026EB9
:106D59001F026E4C026E79026EA605A7800BEB30FE
:106D6900E7032A8002291E1FFBEEC45403F583EEB4
:106D79005408C42FF582EE5407243883F5F0E04512
:106D8900F0F0D8DA05A72205A7800BEB30E7032A34
:106D99008002290E1FFBEEC45403F583EE5408C488
:106DA9002FF582EE5407240B83F5F0E045F0F0D877
:106DB900DA05A722804020100804020105A7800BEC
:106DC900EB30E7032A8002291E0FFBEEC45403F5BA
:106DD90083EE5408C42FF582EE540724EC83F5F0B2
:106DE900E045F0F0D8DA05A72205A7800BEB30E7DC
:056DF900032A800229BD
:106DFE000E0FFBEEC45403F583EE5408C42FF58238
:106E0E00EE540724BF83F5F0E045F0F0D8DA05A77D
:106E1E002205A7800BEB30E7032A8002291F1EFBF9
:106E2E00EEC45403F583EE5408C42FF582EE5407D6
:106E3E00249283F5F0E045F0F0D8DA05A72205A7F5
:106E4E00800BEB30E7032A8002291F0EFBEEC454A1
:106E5E0003F583EE5408C42FF582EE5407246583A0
:106E6E00F5F0E045F0F0D8DA05A72205A7800BEB88
:106E7E0030E7032A8002290F1EFBEEC45403F5836C
:106E8E00EE5408C42FF582EE5407243883F5F0E053
:106E9E0045F0F0D8DA05A72205A7800BEB30E70303
:106EAE002A8002290F0EFBEEC45403F583EE54081C
:106EBE00C42FF582EE5407240B83F5F0E045F0F075
:106ECE00D8DA05A7228040201008040201EC701FBA
:086EDE00ED20E740D2E023CFD4
:106EE60023CF30E7F980357B08801A7B1080167B2C
:106EF6002080127B40800E20E4ED20E3EE20E2EFBE
:106F060020E1F07B80EE8BF0A4CF8BF0A4E5F02F90
:106F1600FFEC8BF0A4CD8BF0A4E5F02D2499838FA4
:106F2600F0A433E5F033FBE98BF0A4E5F0C88BF071
:106F3600A428F9E435F0F822FFFEFCFAF8F6F4F29C
:106F4600F0EFEDEBEAE8E6E5E3E1E0DEDDDBDAD9FA
:106F5600D7D6D4D3D2D0CFCECCCBCAC9C7C6C5C458
:106F6600C3C1C0BFBEBDBCBBBAB9B8B7B6B5B4B372
:106F7600B2B1B0AFAEADACABAAA9A8A8A7A6A5A45E
:106F8600A3A3A2A1A09F9F9E9D9C9C9B9A99999822
:106F96009797969594949392929190908F8F8E8DC9
:106FA6008D8C8C8B8A8A8989888787868685858455
:106FB600848383828281818075A700906FE4E54691
:106FC600FA24FA50027A05EA2323F978107F04930B
:106FD600F60809E9DFF9906FFCEA93F556227FC2BD
:106FE600803E7F4680BA7E8C81747D1882E87A3036
:106FF60085D074608BA08080402010081270080233
:10700600725ED215D274D273C219C23A1255E48E88
:1070160047757D0075460575520212905112022180
:10702600E53524EB500E1290517F1990A01C127575
:10703600F812DD0DE55275F016A4F570127214758E
:107046007E151270DF7F237E09909FF812760A1252
:10705600DD0D10000810010D10021280E21271877A
:1070660075330180DA1271CC75330180D2757E00DA
:107076001270DF7E0090A00B12763D7F237E059076
:10708600A00012760A12713012DD0DE55210000FC3
:1070960010010510028780D5045403F55280CE12E4
:1070A60070DF7F237E0B90A03B12760AE5466007D1
:1070B6001460041412405D12DD0DE5461000081040
:1070C600010B10021180D860D6154680D2B4050295
:1070D60080CD054680C902702375320012DEE37F3B
:1070E600017E11909FEF12763D7E0012D5A4E57EBB
:1070F600D26612D5FB75170812DA2E12409C7571EE
:1071060000C20612D74B741BFFF5177E0F90A041E5
:10711600305D0390A04912763D129094125C1512D0
:107126004602C206126424021D46E552601414602B
:107136001E1460297F647E2D791C12717A1E1FD958
:10714600F9227F6A7E1F792812717A1FD9FA227F67
:10715600487E2D791C12717A0F1ED9F9227F567E30
:107166003379281F12DE280F0F12DE281F12DE28A1
:107176001ED9F0221E12DE280E0E12DE281E02DE98
:1071860028E552605514606814606D800075709E25
:107196001272018003757000E5732540F573E435BE
:1071A60074F574E43575F5752275701612719E8046
:1071B6000375702DE5762542F576E5773541F57749
:1071C600E43578F57822E55260CB1460DC1460E192
:1071D60080007570441271BA800375705AE5739514
:0971E60040F573E5749400F574A2
:1071EF00E5759400F575227570711271E380037562
:1071FF007088E5769542F576E5779541F577E578F0
:10720F009400F57822E54690722A93F540FEAD473B
:10721F00E4FFFC1253778E418F4222020C1830602C
:10722F00C07F40120D8B121D5C12DD0D1274D9EB55
:10723F007005909D4A800B1272E790A390500390B7
:10724F00A3D67F3F7E0412760A12DD0D12DDEE12F9
:10725F00DE1E753709909FAA121C4290726E730240
:10726F00029302742E02700202750A02725E02729B
:10727F008602729F0272307F2E1215C980D17F361F
:10728F007E0490A36412760A12DD0D12DDEE80BF2C
:10729F007F37120D8B121D5C12DD0D1274BD12475C
:1072AF0092D2AC1000A9306DFA127397203BCF40E9
:1072BF00ED7568F97516001273E440FB1275807F47
:1072CF00367E29E51612D38412DD0D05161276B01F
:1072DF0078C6B6F7E20274B77C0512479212DC2724
:1072EF00744112DC38745312DBF5EB12DC16127694
:1072FF00C25003DCE5227515F975160010000EE576
:10730F0015602512733940051273605002D3227F26
:10731F003F7E29E51612D38412DD0D7F1412DE0590
:10732F000516E51664F870D4C322127C7875B9017E
:10733F00E5BCB4811AE5BDF51570037516F778C66F
:0B734F00A616127DC1127DB9127DB997
:10735A00C3027DB9D3227F0575F019D5E0FDD5F0BA
:10736A00FA12479212DC27744112DC38744212DB9B
:10737A00F57E0F78C6E60812DBF5DEF912DC191283
:10738A0076C2400122DF012275F00080CEC23B1294
:10739A004792D2AC12DB80204C3CB440F712DB851A
:1073AA00B4400312DB85B4412DF53812DB85B453A2
:1073BA002512DB85FA12DB85E538701A12DB85B4F3
:1073CA000D1412DB85B40A0EC3E5169A4003027641
:1073DA00A7C2ACD23B22C2ACD32212770612479282
:1073EA00D2AC1000F112DB80204CEBB440F412DB7B
:1073FA0085B4400312DB85B441DCF53812DB85B471
:10740A0042D47E1078C612DB85F608DEF9E53870BC
:10741A00C512DB85B40DBF12DB85B40AB9C2ACC391
:10742A002202725E7F0A120D8B121D5C12DD0D1292
:10743A0074BD1247ABD2AC1000E712DB85B440F53D
:10744A00F53812DB85B46EED12DB85E538600A1279
:10745A0047AB744F12DC0180DC1247AB744012DC7C
:10746A0038E51612DC0112DC0B7568F97516001284
:10747A0047ABD2AC10003912DB85B440F7F53812AD
:10748A00DB85B44EC07E1078C612DB85F608DEF9BD
:10749A001247ABE5386007744F12DC0180D11275D0
:1074AA00800516745112DC0178C6B6F7C212751D32
:0C74BA0002725E751500751603127C6FDF
:1074C60075B901E5BC30E70205160515E51524205A
:1074D60050EB227B007515F9127C7875B901E5BC75
:1074E600B481010B0515E515240450EC7515011240
:1074F6007C6F75B901E5BCB481010B0515E5152452
:107506002050EC227F1C120D8B121D9F4006751514
:10751600F912751D02725EE51560372404401A24BF
:107526001E5019E515240740028027127C78127533
:10753600590515E515240450F2751501127C6F7571
:10754600B901E5BC30E7031275590515E515242088
:1075560050EA2212756E124E2C05C6124E2C05C626
:10756600124E2C05C6024E2C74FF80057404800151
:10757600E4F5BCF5BDF5BEF5BF22E568606AF51514
:107586000515E5152404501D751501127C6F75B996
:1075960001E5BC30E70280190515E515242050EBFE
:1075A600751500800C241C60F750E0E51524065084
:1075B60037E56875F004A485F0C7F5C675BC81E5A6
:1075C60015F5BDF56878C6B6F70375BD00081275E2
:1075D600E31275DD1275DD86BC0886BD0886BE0819
:0975E60086BF08124E2C05C622D6
:10C0010012ADFC12C10012818912C08512819112F8
:10C01100C09202AE0012ADFC12C1001281897F5A9A
:10C02100C23C12806B128267783F79437F607EEA5F
:10C0310012C0F41281917F6512806B128267783D84
:10C0410079417F207E4E12C0F4303C2012C2B612DC
:10C05100C111783F794312C070783D794112C070A7
:10C0610012C2B678D7E65480F6753700029266C3DD
:10C07100E796FF1819E796FE0809C3E69FF7181916
:10C08100E69EF7227F5B7E0690A46A12763D1F80B2
:10C091000A7F667E14745912D49D1F127EF47E3974
:10C0A100E402D4BC7866E620E73418C3E69472084B
:10C0B100E694045029C318E6941F08E69404401E30
:10C0C1007869E620E71818C3E6940E08E694015053
:10C0D1000DC318E6947508E694004002D322C322EA
:10C0E100E67D0030E7011D08E62BFB18E63CFCE489
:0EC0F1003DFD22C3EB9FF6F71819EC9EF6F703
:10C0FF002212C0A5400CE47842F608F67840F60804
:10C10F00F6227864C3E6946AF55708E6944CF55620
:10C11F000808C3E69458F55B08E694AEF55A7539EE
:10C12F0000AC56AD57EC12B1A9784C12B237AC5ADD
:10C13F00AD5BEC12B1A9785012B2377F2B7E867DA2
:10C14F00777C1812B16E785012B22B12B07A12B1EE
:10C15F006E785012B22B12B07A12B16E785012B2B2
:10C16F002B12B07A12B16E7F367E847D257C6412DD
:10C17F00B16E785012B22B12B07A12B16E784C1297
:10C18F00B22B12B07A12B16E7F3F7EA27D607C8B94
:10C19F0012B16E785012B22B12B07A12AE6812AE84
:10C1AF006812B2437F3F7E807D057CE6053912B071
:10C1BF007A784812B2377F2C7E937D477C7F12B1FD
:10C1CF006E785012B22B12B07A12B16E785012B242
:10C1DF002B12B07A12B16E784C12B22B12B07A12B7
:10C1EF00B16E7F357EB47DF87CDF12B16E78501260
:10C1FF00B22B12B07A12B16E785012B22B12B07AF3
:10C20F0012B16E7F3F7EED7D227CCD12B16E784CE8
:10C21F0012B22B12B07A12AE6C12AE68784412B210
:10C22F00377F317E397D9D7CE712B16E784C12B22B
:10C23F002B12B07A12B16E784C12B22B12B07A1256
:04C24F00B16E784410
:10C2530012B22B12AE6C12B16E7F2C7E377D0C7C2A
:10C26300A312B16E784C12B22B12B07A12B16E785F
:10C273004C12B22B12B07A12B16E784C12B22B124E
:10C28300B07A12AE6C12B2437F3F7E807D027C9FF8
:10C29300053912B07A784412B237784812B22B12A9
:10C2A300B1E08E428F43784412B22B12B1E08E403C
:10C2B3008F4122753900AC42AD43EC12B1A97848E5
:10C2C30012B237AC40AD41EC12B1A9784412B23787
:10C2D3007F2B7E537D507C0912B16E784812B22BAE
:10C2E30012B07A12B16E784812B22B12B07A12B130
:10C2F3006E784412B22B12B07A12B16E7F347EF292
:10C303007DCD7CA312B16E784812B22B12B07A1293
:10C31300B16E784812B22B12B07A12B16E7F3F7EA3
:10C323000A7D2E7CAE12B16E784412B22B12B07A13
:10C3330012AE6812AE68784C12B2377F2B7E4F7DF7
:10C34300AF7CB212B16E784812B22B12B07A12B12E
:10C353006E784812B22B12B07A12B16E784812B2CC
:10C363002B12B07A12B16E7F357EB17D4B7C951264
:10C37300B16E784812B22B12B07A12B16E784412B1
:10C38300B22B12B07A12B16E7F3F7E497DCD7C45D0
:10C3930012B16E784812B22B12B07A12AE6C12AE92
:10C3A30068785012B237784C12B22B12B1E08D5527
:10C3B3008E568F57785012B22B12B1E08D598E5A88
:04C3C3008F5B7864B0
:10C3C700E557246AF608E556344CF608E555340473
:10C3D700F608E55B2458F608E55A34AEF608E43566
:03C3E70059F622E2
:1090B40012ADFC12974512AE007F6690A44C127656
:1090C4003B1291227F5A78C41290FE12910678C600
:1090D4001290FE1290E97F6578C81290FE129106F4
:1090E40078CA1290FE7E2DE51B12D4BC7E33E51A9D
:1090F40012D4BC7E39E51902D4BC86040886030266
:1091040052417E15E51C12D4BC7E1BE51B12D4BC57
:109114007E21E51A12D4BC7E27E51902D4BC7F5AFD
:109124007E01E53A12D3D27E0B909B39E53B930244
:10913400D4CFE6FF08E6FE08E6FD339217E45001BB
:10914400F4FC12B25475130A75390112B45278D76B
:10915400E6C2E775F00A84F9303D02A9F012B25470
:109164008913053912B42B30170A053912B43E0598
:109174003912B43EA80302B23712ADFC129745C2AD
:109184003C7F5A7E0312841812912212DD0D1000C6
:109194000810011510022080EFE53A146004153A16
:1091A4008003753A3CD23C80DFE53AB43C05753A1D
:1091B4000180F2053A80EE7E031284137E0B128442
:1091C4001812912212DD0D10000810011510022052
:1091D40080EFE53BB40205753B158002153BD23C9C
:1091E40080DFE53BB41505753B0280F2053B80EE5C
:1091F4007E0B1284137F5A78C41290FE12910612C9
:07920400926F12827778C41B
:10920B001292C778C61290FE1290E91292A1751CA9
:10921B000012827778C61292C77F6578C81290FECB
:10922B0012910612926F12827778C81292C778CA7F
:10923B001290FE1290E91292A1751C00128277789F
:10924B00CA1292C7303C14E53B24F4500B78C9E6A4
:10925B002410F618E63427F61292CD12AE00127DCA
:10926B00F902DD0DC2247E15E51C128368F51CD2B4
:10927B00247E1BE51B128368F51B1023E77E21E57B
:10928B001A128368F51A1023E67E27E519128368F4
:10929B00F5191023E822C2247E2DE51B128368F5F5
:1092AB001BD2247E33E51A128368F51A1023E77E4E
:1092BB0039E519128368F5191023E622ECF608EB51
:1092CB00F622129B5178C8E6FE0886073395E0FD1F
:1092DB00FC12B16E7FE87E037D007C0012B452124B
:1092EB00B16E78CAE6FE0886073395E0FDFC12B432
:1092FB002B12B16E7F807E697D677CFF12B42BECE5
:10930B0012B1A512B16E7F3F7E807D0D7C1D12B018
:10931B007A12B16E7F3D7E407D007C0012B16E787B
:10932B00BC12B22B12B07A12B16E7F3E7E807D00E2
:10933B007C0012AE6C12B16E78BC12B22B12B07AEA
:09934B0012B16E7F3F7E807D00AF
:109354007C0012AE6812B16E78B412B22B12B07ADD
:1093640012B0F2783C12B2377F407E807D007C00E0
:1093740012B16E783C12B22B12B07A12B2D112B181
:109384006E7F3F7EA87D007C0012B16E78B812B269
:109394002B12B07A12B07A12B16E7F407E007D003B
:1093A4007C0012B16E783C12B22B12B07A12B2D198
:1093B40012B16E7F3F7EC07D007C0012B07A12AE87
:1093C4006C12B16E78B812B22B12B07A12B16E78F8
:1093D4003C12B22B12AE6C785412B23712B2BB7874
:1093E4005812B23712B16E12B07A12B16E78C0123E
:1093F400B22B12B07A784412B237785412B22B12CC
:10940400B2D1783C12B23712B16E12B07A12B16E88
:1094140078BC12B22B12B07A783C12B2377F3E7EFF
:10942400C07D007C0012B16E783C12B22B12B07A6F
:1094340012B16E7F3F7E007D007C0012AE6C12B1D3
:109444006E783C12B22B12B07A12B16E7F3F7E80DE
:109454007D007C0012AE6C12B16E78B412B22B1285
:10946400B07A787012B23778C4E6FE08860733956E
:10947400E0FDFC12B16E7FE87E037D007C0012B437
:109484005212B16E78C6E6FE0886073395E0FDFCFD
:1094940012B42B12B16E7FE07E5E7DF87CFF12B4B5
:1094A4002BEC12B1A512B16E7F3F7E7F7DE57CC9A6
:0594B40012B16E78709A
:1094B90012B22B12B07A12B0F2785012B2377F3F43
:1094C9007EF07D007C0012B16E783C12B22B12B096
:1094D9007A12B16E7F3F7EC07D007C0012AE6C12A5
:1094E900B16E783C12B22B12B07A12B16E7F3F7E08
:1094F900807D007C0012AE6C783C12B23778BC12C9
:10950900B22B12B16E7F3F7E807D007C0012AE6867
:1095190012B16E783C12B22B12B16E78B412B22B22
:1095290012B07A12B07A784012B237785412B22B4C
:1095390012B309783C12B23712B16E12B07A78744C
:1095490012B2377F417E107D007C0012B16E78C067
:1095590012B22B12B07A12B16E7F407E807D007CF0
:109569000012B16E784412B22B12B07A12B16E7F2A
:10957900417E207D007C0012AE6812B16E784412E3
:10958900B22B12B07A12B16E7F407E407D007C0012
:1095990012B16E787412B22B12B07A12B16E7F408A
:1095A9007EA07D007C0012AE6C12AE6C12AE681209
:1095B900B16E785012B22B12B07A12B16E78501285
:1095C900B22B12B07A12B16E7F3D7E2A7DAA7CAB96
:1095D90012B07A12B16E7F3F7E007D007C0012AE20
:1095E9006812B16E783C12B22B12B16E787012B259
:1095F9002B12B07A12B16E784012B22B12B0F2125D
:10960900B16E785012B22B12B07A12B16E78501234
:10961900B22B12B07A12B07A12B16E785412B22B00
:0C96290012AE6812B16E7F4A7E517DD2F5
:109635007CCB12B07A12B1E078AC12B2377F407EA3
:10964500007D007C0012B16E787412B22B12B07AD4
:1096550012B16E7F3F7E807D007C0012AE6C12B130
:109665006E784412B22B12AE6C12B16E785012B2F3
:109675002B12B07A12B16E785012B22B12B07A1248
:10968500B16E785012B22B12B07A12B16E7F3E7E57
:109695002A7DAA7CAB12B07A12B16E785012B22B29
:1096A50012AE6812B16E785812B22B12B0F212B126
:1096B5006E7F4A7E517DD27CCB12B07A12B1E01218
:1096C500B16EAF3AEF3395E0FEFDFC12B16E7F400F
:1096D5007E7E7D057C0012B45212B16E7F607E7570
:1096E5007D587CFF12B42B12B42B78B012B23778A8
:1096F500AC751B6412971C8F1C78B0751B6712978D
:109705001CE51C75F00AA42FFF249C50027F0078ED
:10971500D7E654802FF62275390012B22B12B16E9E
:109725007F0A7E007D007C0012B4FEA81BE513F6BF
:1097350008E512F608E511F6335004EFF404FF22AC
:10974500C23D78647BAC129136D23D78677BB0120E
:109755009136129B517F007EE47D577C0012B16EDD
:1097650078AC12B22B12B42B12B16E7F007E537DF2
:0E977500077C0012B4FE12B18D85133B7F807D
:109783007ECB7DA47C0012B16E78B012B22B12B4E2
:109793002B12B16E7F407E7E7D057C0012B4FE12DB
:1097A300B18DE513F56F04F53A85126E85116D855C
:1097B300106C7F407E7E7D057C0012B16E786C124A
:1097C300B22B12B45212B16E7F607E0C7DA27C006C
:1097D30012B16E78B012B22B12B42B12B43E786C65
:1097E30012B23778AC12B22BEC12B1A512B16E7F64
:1097F300347E9C7D2B7C5F12B07A785412B2371280
:10980300B2BB785012B237786C12B22BEC12B1A5FE
:1098130012B16E7F347E9C7D2B7C5F12B07A12B1C5
:109823006E785012B22B12B07A784012B2377F4062
:109833007E007D007C0012B16E785412B22B12B000
:109843007A12B2D112B16E7F3D7EC07D007C0012D0
:10985300B16E78BC12B22B12B07A12B16E7F3E7E1B
:10986300C07D007C0012AE6C12B16E78BC12B22BBC
:1098730012B07A12B07A12B16E7F3D7E407D007CC9
:109883000012B16E78BC12B22B12B07A12B16E7F95
:109893003E7E807D007C0012AE6C12B16E78BC12ED
:1098A300B22B12B07A12B16E7F3F7E807D007C00B6
:1098B30012AE6812B16E785412B22B12B07A12AE95
:1098C3006812B16E7F407E807D007C0012B16E789D
:1098D3005412B22B12B07A12B2D112B16E7F3D7E06
:1098E300707D007C0012B16E78BC12B22B12B07A7C
:1098F30012B16E78BC12B22B12B07A12B07A12AED9
:109903006C12B16E78B412B22B12B07A785812B2CC
:1099130037785412B22B12B2D1783C12B237785442
:1099230012B22B12B309785412B237783C12B22B0D
:1099330012B16E12B07A12B16E78BC12B22B12B0A1
:109943007A783C12B2377F3E7EC07D007C0012B134
:109953006E783C12B22B12B07A12B16E7F3F7E004A
:109963007D007C0012AE6C12B16E783C12B22B12E9
:10997300B07A12B16E7F3F7E807D007C0012AE6CA8
:1099830012B16E78B412B22B12B07A787012B23769
:10999300785012B22B12B16E12B07A12B16E78C037
:1099A30012B22B12B07A784412B237785412B22B17
:1099B30012B16E12B07A787412B237784012B22BA9
:1099C30012B16E12B07A783C12B2377F407E807D3E
:1099D300007C0012B16E784412B22B12B07A12B12D
:1099E3006E7F417E107D007C0012AE6C12B16E78EA
:1099F3004412B22B12B07A12B16E787412B22B12D7
:109A0300B16E7F407EA07D007C0012AE6812AE6C0A
:109A130012B16E783C12B22B12B07A12B16E7F3D46
:109A23007E2A7DAA7CAB12B07A12B16E7F3F7E0094
:109A33007D007C0012AE6C12B16E785412B22B1200
:109A4300B16E787012B22B12B07A12B16E783C12EA
:109A5300B22B12B07A12B07A12B16E785812B22BBE
:109A630012AE6C12B16E7F3F7E7F7DE57CC912B072
:019A73007A78
:109A740012B16E7F4B7E187D967C8012AE6C12B153
:109A8400E012B16E7FE87E037D007C0012B4FE120A
:109A9400B18D78C8A61208A61308A60608A60778EA
:109AA4007412B22B12B16E7F3F7E807D007C001257
:109AB400AE6812B16E784412B22B12AE6C12B16E53
:109AC4007F3E7E2A7DAA7CAB12B07A12B16E7840BA
:109AD40012B22B12B07A12B16E783C12B22B12B0C1
:109AE4007A12B16E784012B22B12AE6C12B16E7F44
:109AF4003F7E7F7DE57CC912B16E787012B22B1265
:109B0400B07A12B07A12B16E7F487EF47D247C0064
:109B140012AE6C12B1E012B16E7FE87E037D007C60
:109B24000012B4FE12B18D78C4A61208A61308A6BA
:109B34000608A607223F3F4344454647484A4B4C44
:109B44004D4E5051525354555657583F3FE4F539F2
:109B5400F5A7909B65791078B4E493F6A308D9F936
:109B64002232A5C24A4A19DC3A885CDB3BFFD6DCC8
:019B74003BB5
:10ADFC00D2D58002C2D575A70490040078107F0BC1
:10AE0C0012AE2878267F0512AE28783C7F2212AE2F
:10AE1C0028786A7F0F12AE2875A7002230D506E677
:10AE2C00F008DFFB22E0F608DFFB22D2D58002C25D
:10AE3C00D575A7049006FA78737F0612AE2875A70D
:10AE4C000022DA0CD902800BD906303701B3500539
:10AE5C0002AFDB923702AFC7D9F680F9D236800247
:10AE6C00C23612B00C303606C86002B237C8923601
:10AE7C00DAD0D9E4B8000A12B053A236923702AF36
:10AE8C00B060FBB51300400F12B053A23692F7A27C
:10AE9C00379236A2F79237C398F40424E740DF24A4
:10AEAC0019AD29AC28AB277A00C394084008CDCC47
:10AEBC00CBCAE4CD80F424086010F9C3ED13FDEC8B
:10AECC0013FCEB13FBEA13FAD9F1A236303701B3BA
:10AEDC0040308A17E5102BF518E5113CF519E512F1
:10AEEC003DF51A501A13F51AE51913F519E518134F
:10AEFC00F518E51713F5170513E513700205140281
:03AF0C00AF66E449
:10AF0F00C39AF517E5109BF518E5119CF519E51295
:10AF1F009DF51A500DB237C378177F04E496F608E3
:10AF2F00DFFA7A047019E513C39408F5135002156C
:10AF3F0014E4C517C518C519F51ADAE802B00720C9
:10AF4F00E7BAE5137002151415137817C37F04E6DB
:10AF5F0033F608DFFA80E8E51A20E7137817C37F86
:10AF6F0004E633F608DFFAE513700215141513E53E
:10AF7F00173378187F03E63400F6500E08DFF775A5
:10AF8F001A800513E51370020514E51420E75470B9
:10AF9F0027E513604E046020851A12851911851854
:10AFAF00105326F0AC10AD11A237E51313FFE512C5
:10AFBF0092E7FEA81302B18DE4F512F511F510F525
:10AFCF00147513FF5326F043260580D8E5FFF512BD
:10AFDF00F511F510751400F513D2375326F04326EB
:10AFEF000980C15326F0432603E4F512F511F5103D
:10AFFF00F514F513C23780AC5326F080EC79017A43
:10B00F00018512F0E513A2F7339237751400F5138B
:10B01F006002D2F785F012A813B8FF0809E512C233
:01B02F00E739
:10B030006001098C278D288EF0A2F7EF3304700A87
:10B040000AC2F705F00AD5F0011A146002D2F7859A
:10B05000F02922C88813C512C529C512C511C528F3
:10B06000C511C510C527C51022DA03B8000302AF09
:10B07000DBD9028002D9F702AFC712B00C3037011A
:10B08000B392377004D9E78005DADEB8000302B066
:10B0900007D9E2C3947E500215142513F51350020C
:10B0A00005147815760008B81BFA78277915E60894
:10B0B000FAE8FC78108AF0E608A427F709E5F037EB
:10B0C000F7500989F00907E760FBA9F0B813E61902
:10B0D00019ECF8B82AD802AF6602AFF2B8FFFA024C
:10B0E000AFDBD9FB02AFC7DAF6B800F002B0071247
:10B0F000B24312B00C303701B392377007D9E3B8BE
:10B1000000E280DBDAE1B8000280E1D9D5C8C3985B
:10B1100050021514247F50020514F513781A760096
:10B120007A1A7B80C3E5109527E5119528E51295DD
:10B13000294016C3E5109527F510E5119528F5115E
:09B14000E5129529F512E64BF623
:10B14900DA0302AF66EB03FB30E703187600C3E5C9
:10B159001033F510E51133F511E51233F51240CA34
:10B1690030E7DD80B6E53905396010D0F0D0E0C0B0
:10B1790010C011C012C013C0E0C0F08F138E128D21
:10B18900118C1022E539146010D0F0D0E0D013D022
:10B1990012D011D010C0E0C0F01539227920800CEE
:10B1A9007910800479087D007E007F003392D550A4
:10B1B9000312B21DEC33400FEF33FFEE33FEED33D4
:10B1C900FDEC33FCD9EE22EECCF5F0747E29A2D544
:10B1D90013FF92F7AEF022EF8EF0A2F7D2F7339277
:10B1E900D5C3947F5006E4FFFEFDFC229420400461
:10B1F90074FF80F304CCFEE4FFFAE5F0CC6012C3DF
:10B20900CC13CCCD13CDCE13CECF13CF0450EEDA61
:10B21900EC30D5D7C3E49FFFE49EFEE49DFDE49C9A
:03B22900FC22E61E
:10B22C00FC08E6FD08E6FE08E6FF22ECF608EDF663
:10B23C0008EEF608EFF622CFC513CFCEC512CECD51
:10B24C00C511CDCCC510CC22E4F513F512F511F5D2
:10B25C001022E493FCA3E493FDA3E493FEA3E493F4
:10B26C00FFA322C0E012B16E12B07A12B2A212B2D7
:10B27C005ED0E0C0E012B16E12B29912B07A12B187
:10B28C006E12B25E12AE6CD0E0D5E0E722AC48ADE7
:10B29C0049AE4AAF4B228C488D498E4A8F4B227453
:10B2AC00FF7809FFFEFDFCE52654F048F526221236
:10B2BC00B36204A2E1927F1420E01590B3E374040E
:10B2CC0012B26F802912B36230E102B27F20E0EB40
:10B2DC008C4C8D4D8E4E8F4F90B3F7740412B26F11
:10B2EC0012B16EAC4CAD4DAE4EAF4F12B07A307F4A
:10B2FC0004EF6480FFEE33EF337001FF2212B36270
:10B30C00C0E08C4C8D4D8E4E8F4F90B41B7403123D
:10B31C00B26F12B16EAC4CAD4DAE4EAF4F12B07AA7
:01B32C00EC34
:10B32D00C54CFCEDC54DFDEEC54EFEEFC54FFF9076
:10B33D00B40B740312B26FD08212B16EAC4CAD4D22
:10B34D00AE4EAF4FE58230E00712B0F2B27F809D76
:10B35D0012B0EF8098EE33EF3324605007D0E0D079
:10B36D00E002B2ABEFA2E7547F927FFF12B16E7C89
:10B37D00837DF97E227F3E12B07AEE33EF33248146
:10B38D00501012B16E12B1E012B1A5EFB2E7FF127B
:10B39D00AE6CEE33EF33602A2403F8C313FFEE9245
:10B3AD00E7FEE82481E4501A12B16E12B1E0EF0409
:10B3BD00C2E0FCF58212B1ADEFB2E7FF12AE6CE563
:10B3CD008203FAEE33EF33600B148FF0A2F713FF05
:10B3DD00EE92E7FEEA2283FA703AE4E9AABCF8E0BD
:10B3ED00813EE6E99DBF0000803F1A3C2839666921
:10B3FD0099BBE335A33DE75D25BFDB0FC93FCCDB33
:10B40D008D41EE3649C43F91C9453DF8B0C50000A8
:10B41D00803F34F517C373FA2F45DDFD0AC6EF25BE
:10B42D0013FFEE3512FEED3511FDEC3510FC02B1BA
:10B43D008DC3EF9513FFEE9512FEED9511FDEC9575
:10B44D0010FC02B18DEFF88513F0A4FFE513C5F0E4
:0AB45D00CEF9A42EFEE435F0CDFA7E
:10B4670088F0E512A42EFEED35F0FDE433CC85130C
:10B47700F0A42CFCE5128AF0A42CFCE51189F0A4B9
:10B487002CFCE51088F0A42CFC89F0E512A42DFD16
:10B49700EC35F0FCE51188F0A42DFDEC35F0FC8AC5
:10B4A700F0E513A42DFDEC35F0FC02B18DE4CCF8EA
:10B4B700E4CDF9E4CEFAE4CFFB75F020C3E513330E
:10B4C700F513E51233F512E51133F511E51033F5F0
:10B4D70010EF33FFEE33FEED33FDEC33FCEF9BEE65
:10B4E7009AED99EC98400CFCEF9BFFEE9AFEED99D4
:10B4F700FD0513D5F0C622C2D5EC30E705B2D5124B
:10B50700B21DE51030E70DB2D512B52112B4B41251
:10B51700B21D800312B4B430D515C3E49513F513E7
:10B52700E49512F512E49511F511E49510F5102242
:10A5E100E57124885002D2191255E48E4712D1E246
:10A5F1001290941259A0305E0F12593E12878312A5
:10A60100586F12BF9312419712387D12473E103690
:10A6110029201F1C301219E412A76712A77C12A867
:10A621007C12A89E30510302A92812ABF9205109CE
:10A63100C251E4F552F545F5442275A7007583072B
:10A64100E559C454F0F582E0F538A3E0F518A3A369
:10A65100A3E0F51E74FF12A7671255E48E1C8F1B31
:10A661007510DF751100E51164B4700612A732751B
:10A67100111012A6FF4028AE1CAF1B12566C2032DF
:10A681001EAC03AB027A0C125279ED701275A70061
:10A69100758304851182ECF00583E510F00511D571
:10A6A10010C412A73275C70375C6E075A7049005DB
:10A6B100007F0412A6EDDFFB75A700122AC612590E
:10A6C1003EE4F5A7F8F559758307E8C4F582E0651E
:10A6D100387011A3E06518700BA3A3A3E0651E7089
:10A6E1000388592208C3E5589850DC22E0F5BCE004
:10A6F100F5BDE0F5BEE0F5BF124E2C05C622E51012
:10A7010075F004A4F5C685F0C775B901E5BC334001
:0BA711001F05C605C675B90185BE64B2
:10A71C0085BF6505C675B90185BC6685BD6785BEF7
:10A72C006885BF69C322E51124FE502E75A7007FF2
:10A73C0010AE111E7583048E82E0FD1582E0CDB53E
:10A74C0005005012F00582CDF00583E0FD1582E086
:10A75C00CDF00582CDF0DEDCDFD72275A754900456
:10A76C000005A79005007FB4F0F0DFFC75A7002270
:10A77C0012BDF0C2517B077AFFE4FFF5A7900400ED
:10A78C0012A862ED244C4035EC603075A7008D8228
:10A79C0005A712A8287583058D82E02410401CF0B3
:10A7AC0005A7E02CF0500505A7E004F0BA000CBB9F
:10A7BC000009D251EF24DC50027F23DFC3EA60058D
:10A7CC0012A7DB8006EB600312A81375A7002230DA
:10A7DC00E0047553082230E1047553182230E2046A
:10A7EC007553282230E3047553382230E404755332
:10A7FC00482230E5047553582230E604755368221C
:10A80C0030E7037553782230E0047553882230E129
:10A81C00047553982230E2037553AA22ED54F0C408
:10A82C00232390A832735302FE225302FD225302BB
:06A83C00FB225302F7228B
:10A842005302EF225302DF225302BF2253027F221E
:10A852005303FE225303FD225303FB225303FB2225
:10A8620012BD2812BBB6E4F5F7C2B2C2B2ADF7F51B
:10A87200F7C2B2C2B2ACF7D2B22290050078B4E00D
:10A882006015FD54F0C4CD7C00540FFE1583E0FF2B
:10A89200125377EFF005830582D8E422758304789A
:10A8A200FF088882E060FAF5D38812E512244C5042
:10A8B200012285D3D288D4881279FF0512E512606D
:10A8C200F00908E875F0B484A8F08882E060ECF53D
:10A8D200D3B9000280D5B9230050D0C395D292D10A
:10A8E2005002F40409FEE4FFFCAD0112538474012A
:10A8F200FA25D475F0B484A8F0AC06AB0712526BFB
:10A90200EB30E7010CE5D22C30D1029C9C8882F01E
:10A912000AEAB501DCE512244C50012285D3D28526
:10A9220012D4A812809390040012A9E78C068B051A
:10A9320012A9E7E4FFF512F5118C148B13C3ED9BFA
:0EA94200F9EE9CFA4012E51199E5129A500ABE
:10A950008C148B138A1289118F528F82E0F9C3ED08
:10A9600099FDEE9400FEE582245A5002244C75F0C5
:10A97000B48485F082E0FA2DFDEE3400FEEB9AFB04
:10A98000EC9400FCE92BFBEC3400FC0FBFB4B0E509
:10A990005224D3400224B4F552C3E51333FBE5142B
:10A9A00033FCE511FE2BFBE512FF3CFC1253D9E909
:10A9B000F890A9F993F511FDEBF513FFECF514FEF2
:10A9C0007C001253778F44E890AAF993FAAB13AC4A
:10A9D000141252A2AF03AE04AD117C00125377EFF4
:10A9E0007002F552F545227C007B007F5AE02BFB7C
:10A9F000EC3400FC0582DFF522B4B4B4B4B4B4B4D2
:10AA0000B4B4B4B4B4B4B4B4B4B4B4B3B3B3B3B30B
:10AA1000B3B3B3B3B3B3B3B3B2B2B2B2B2B2B2B20E
:10AA2000B2B1B1B1B1B1B1B1B0B0B0B0B0B0B0AF1E
:10AA3000AFAFAFAFAEAEAEAEAEAEADADADADADAC39
:10AA4000ACACACACABABABABAAAAAAAAA9A9A9A95E
:10AA5000A9A8A8A8A8A7A7A7A7A6A6A6A5A5A5A58B
:10AA6000A4A4A4A4A3A3A3A2A2A2A2A1A1A1A0A0C2
:10AA7000A0A09F9F9F9E9E9E9D9D9D9D9C9C9C9BFC
:10AA80009B9B9A9A9A99999999989898979797963B
:10AA9000969695959594949493939392929291917E
:10AAA00091919090908F8F8F8E8E8E8D8D8D8C8CBE
:10AAB0008C8B8B8B8A8A8A89898988888887878703
:10AAC0008686868585858484848383838282828149
:10AAD00081818080807F7F7F7E7E7E7E7D7D7D7C8C
:10AAE0007C7C7B7B7B7A7A7A7979797878787777CE
:10AAF0007776767675757574740002030506080915
:10AB00000B0C0E101113141617191A1C1D1F2122DD
:10AB1000242527282A2B2D2E303133343637393A45
:10AB20003C3D3F404243454648494B4C4E4F5052B6
:10AB300053555658595A5C5D5F6061636466676837
:10AB40006A6B6C6E6F707273747677787A7B7C7ECA
:10AB50007F80818384858688898A8B8D8E8F909172
:10AB6000929495969798999B9C9D9E9FA0A1A2A434
:10AB7000A5A6A7A8A9AAABACADAEAFB0B1B2B3B40D
:10AB8000B5B6B7B8B9BABBBCBDBEBFC0C0C1C2C301
:10AB9000C4C5C6C7C7C8C9CACBCCCCCDCECFD0D010
:10ABA000D1D2D3D4D4D5D6D7D7D8D9DADADBDCDC36
:10ABB000DDDEDEDFE0E0E1E2E2E3E4E4E5E5E6E776
:10ABC000E7E8E8E9EAEAEBEBECECEDEEEEEFEFF0CC
:10ABD000F0F1F1F2F2F3F3F4F4F4F5F5F6F6F7F739
:10ABE000F8F8F8F9F9FAFAFAFBFBFBFCFCFDFDFDBD
:10ABF000FEFEFEFEFFFFFFFFFFC251E4F544F81426
:10AC0000FB900400A9007C0FC2D112AD14E824050A
:10AC1000F8B8B4F08B13E5122403FA244C5001FA6F
:10AC2000BBFF012275112C8A1912AD4B8F16203DE6
:10AC300012AA1975112312AD4B8F15751600303DF0
:10AC4000E2801175112312ACF3751500303D05E853
:01AC50002FD4
:10AC510013F51575111212ACF3751400303D05E8AA
:10AC61002F13F514EA2404F552244C5002F552E452
:10AC7100F51AF51BF51CE516600AFB7A00AF137E89
:10AC8100FF12ACB9E515600AFB7A4FAF137EFF12D4
:10AC9100ACB9E516600DFB7A00E5146006FF7ECFC6
:10ACA10012ACB9AE1CAF1B7C00AD1A1253778F45A5
:10ACB100EF2513F544D25122EFF5F0A4FCADF0EBF2
:10ACC100F5F0A49CFCE5F09DFDEB8AF0A4FAABF055
:10ACD100EF8EF0A49AF8E5F09BF9E833F8E933F93F
:10ACE1007B0012541D051AE51B2BF51BE4351CF5E1
:10ACF1001C22EA2511F9244C5001F9C2D112AD12DE
:10AD0100303D428F00C3EA9511F9500324B4F9D2C2
:10AD1100D17C09E4FDFEFF8982E060062FFFE43E5D
:10AD2100FE0D09B9B4027900DCEDED20D118F51E54
:10AD310024FE923D500F125384EFB5030050068557
:10AD41001E1FFB881222F51D80E612ACF3203D4345
:10AD5100740212ADEA12ACF3203D38740412ADF264
:10AD610012ACF3203D2D740612ADEA12ACF3203D76
:10AD710022740812ADF212ACF3203D17740A12AD21
:10AD8100EA12ACF3203D0C740C12ADF212ACF320BC
:10AD91003D0122C3E89F605088148F158A16400830
:10ADA1001ABAFF0A7AB380060ABAB4027A0012AC60
:10ADB100F3303D34C3E89FF9602EC3E5149515FBCC
:10ADC1006930E7D4E930E703F404F9EB30E702F442
:10ADD10004C3995002AA16E5142515C82F28FFE4CB
:10ADE100FC33FE7D04125377222AFA244C5001FAD7
:0BADF10022C3CA9AFA500324B4FA22CD
:10BB7D00758000C2B212DE03D2B275F83022758024
:10BB8D0000C2B2F5F7C2B2C2B2D2B222758000C203
:10BB9D00B2F5F7C2B2C2B2856CF7C2B2C2B2856B52
:10BBAD00F7C2B2C2B2856AF722758000C2B275F7CC
:10BBBD0003C2B2C2B2856FF7C2B2C2B2856EF7C20E
:10BBCD00B2C2B2856DF72212BC0D740612BB8B7416
:10BBDD000212BB998FF7C2B2C2B2D2B222909E7A34
:10BBED007F631275F812DD0DD214120D8112757668
:10BBFD00124E2C12BC0D740612BB8B74C712BB8B6C
:10BC0D0012BC1340FB22758000C2B275F705C2B29B
:10BC1D00C2B2C2B2C2B275F705C2B2C2B2C2B2C22C
:10BC2D00B2E5F7D2B2A2E022120D8185BF6C85BEBE
:10BC3D006B756A00E56B7015E56A701112BC0D74B9
:10BC4D000612BB8B74D812BB99D2B2D21F22E54B10
:10BC5D000475F03C8485F04B12BF18852E72E55F9C
:10BC6D00030354C0F8E55E543F28F57C305501229E
:10BC7D0012BCB212BC1340F7E54C60F312BC0D12AE
:10BC8D00BCC912BC9780F112BC0DC21F740612BB49
:10BC9D008B740212BB99787086F708B880FAD2B20D
:10BCAD0012BCE6808F787075A704758304E54CC4CB
:0CBCBD00F5827F10E6F0DFFC054C8019DA
:10BCC900787075A704758304154CE54C30E701E4D9
:10BCD900C4F5827F10E0F6DFFC75A70022741025F9
:10BCE9006A54F0F56AE4356BF56BE4356C540FF57D
:10BCF9006C22E54B75F010A4256A54F0F56AE5F05D
:10BD090080E4E56A24F054F0F56AE56B34FFF56BDD
:10BD1900E56C34FF80D7E56A24FF80ECC380EBE54E
:10BD29006D24F054F0F56DE56E34FFF56EE56F3472
:10BD3900FF540FF56F2212BD9712BDBFC22DC25419
:10BD4900C255E57F7002D255147002D254E54A30CB
:10BD5900E00122B4061C20540D12BD0B12BE67125D
:10BD6900BEF712BF2F221284377E0412DDFB754AFB
:10BD7900012220550D12BCE612BED612BF1812BE02
:10BD890040221284377E0412DDFB754A05227403B2
:10BD990012BB997870E4F5F7C2B2C2B2A6F708B837
:10BDA90080F3D2B222740312BB99E4F5F7C2B2C28E
:10BDB900B2E5F7D2B222E575F8541F30E40244E047
:10BDC900F57585722EA2779226E57C543F30E502FF
:10BDD90044C0F55EE57C54C02323F55FE57FC2E7E7
:10BDE90079BCF709A77E22856C6F856B6E856A6DB4
:01BDF9002227
:10BDFA00856F6C856E6B856D6A22E4FEFF7407752C
:10BE0A00A704F5838E8274FFF0DFFD75A700227404
:10BE1A00067E007FB012BE09E4F55AF55B2275A7CB
:10BE2A0004758306E55A600A75F00A84E5F0700223
:10BE3A00740AC4F58222307720E55A2402400205AA
:10BE4A005A12BE28E55AF0E573F0E574F0E575F08C
:10BE5A00E576F0E577F0E578F075A700223077F916
:10BE6A0012BE287F1074FFF0DFFDE55A24F5500357
:10BE7A0012BE92155AE55AB4FF02055AC3E55A95FD
:10BE8A005B50D6755B0080D112BDF07F0A056D0547
:10BE9A006D12BBB6E4F5F7C2B2C2B2E5F7D2B23060
:10BEAA00E704DF02800512BD2880E2056D12BBB6E9
:10BEBA0012BE28E55A24F6F07F06E4F5F7C2B2C2AC
:10BECA00B2E5F7F0DFF4D2B275A70022053FE53FED
:10BEDA00B43C17753F00053EE53EB43C0D753E0087
:10BEEA00053DE53DB41803753D000249FE153FE5E1
:10BEFA003FB4FF17753F3B153EE53EB4FF0D753E57
:10BF0A003B153DE53DB4FF03753D170249FE054269
:10BF1A00E542B43C0F7542000541E541B43C057564
:0CBF2A0041000540221542E542B4FF0F23
:10BF360075423B1541E541B4FF0575413B1540226D
:10BF4600AC40AB41A842EC75F03CA42BFBE435F0C9
:10BF5600FC7A3C12526BEB28FBE43CFC22E53FC327
:10BF660013F8AB3E79AEE7800E120D4AE5BE75F0CA
:10BF760005A4FB7800E5BF75F03CA42BFBE435F087
:10BF8600FC7A1E12526BEB28FBE43CFC2212BF6FBC
:10BF9600AE04AD0312BF638C148B13120D54E5BFB0
:10BFA600FF24F650027F01E5BE75F096A4AAF0F9CB
:10BFB600C3ED9513FBEE9514FC924E4B70112011B8
:10BFC6000E30480B75364B3003037536FFD22E30D4
:10BFD6004E02DF1F7A0212526B75A7009004EEEC38
:10BFE600F0A3EBF0C3E5BF9F04BF0102D2E79005C3
:0BBFF600CBF022ED29FDEE3AFE80B5F5
:10DDE80012DDF112DDF112DDF17E0480067E028083
:10DDF800027E017F0080087F6480027F017E00EF41
:10DE08004E6012E4FD0D1D0DEDC394AD40F7EF1FFC
:10DE180070ED1E80EA22753500C200C201C20222DE
:10DECF00F5D8D2DCE5F520E7FBE5DA540FFEAFD944
:04DEDF0075D80022D0
:10DAD6007F767E06909B8912760A740412DECF7CCE
:10DAE600007D52125377EFF875F00A84C0F07F7606
:10DAF6007E2312D4BC7E29742E12D4CF7E2ED0E083
:10DB060012D4BC7E35745612D4CF7F6B7E1190DB57
:10DB16003F12D4FBE824E04001220423F824E75016
:10DB260002781812DB2FD8FB227F6CE82411FE79CD
:10DB36000512DE280E0FD9F922071DFFFFFFE08030
:10DB4600000020C0000038E0000008F0000038F8AF
:07DB5600000020FFFFFFE0CB
:10DB5D0012DB8530E6022409540F75F00AA4F51581
:10DB6D0012DB8530E6022409540F25152212DB85C0
:10DB7D00540F2275F000800875F044800375F0078E
:10DB8D00E4206D09D5E0FAD5F0F7D24C229247C2C8
:10DB9D00ACE54F623885504FA26E926D859950C29B
:10DBAD006FD2ACC24CA2472212DBBFC4FA12DBBF4C
:10DBBD002A2212DB8520E603540F22540724092262
:10DBCD00E612DBD418E608FAC412DBDAEA540F4485
:10DBDD0030F924C6E950112407800D75F00A84C070
:10DBED00F012DBF3D0E0443030530975F00085E0DE
:10DBFD00E0D5F0FA3099FDC299F599623822E538F1
:10DC0D0080F2E53812DBD4800812DBF5E53812DB43
:10DC1D00F5740D12DBF5740A80CE744012DBF574C9
:10DC2D004080C5742C80C1742E80BD75380080B8BD
:10DEF50085A0835383FE438380858384F0758400E6
:01DF050022F9
:10D9840074A212DEF574A112DEF574A612DEF5742B
:10D99400A412DEF574C012DEF5742512DEF512DA77
:10D9A4001475C70375C6FC75B90112B5377408122E
:10D9B400DECFEE75F020A4FEEF54F80303032E240B
:10D9C40092C313FE24EA50027E16EE90D9FD9325ED
:10D9D400BCFE24E6501F24E8401B748112DEF5EEE1
:10D9E40012DEF512DA21744012DEF5742F12DEF520
:10D9F40074AF02DEF57E2680E1F7F7F8F8F9FAFB5A
:10DA0400FCFDFEFF0000000001010202020303030B
:10DA1400A8BCA9BDAABEABBFACC7ADC62288BC8991
:0ADA2400BD8ABE8BBF8CC78DC622E1
:10DD0D00C006C007C5F075A7019000007EB7E58C71
:10DD1D00240340FA12DD2F1EBEAFF3C5F0D007D09D
:10DD2D00062275A700EE12DEF5741012DEF57404EE
:10DD3D0012DEF585A08343838185838475A7517F8A
:10DD4D0020E0F0E0F0E0F0E0F0DFF6E4F5A7F58498
:01DD5D0022A3
:10DEE30075A711900000E4C583F0C58330E2F8F50F
:02DEF300A72264
:10DE2800EF20E723EE20E71F20E61C05A7C45403D4
:10DE3800F583EE5408C42FF582EE5407240983F5C0
:10DE4800F0E045F0F005A722804020100804020108
:10DE5800EF20E723EE20E71F20E61C05A7C45403A4
:10DE6800F583EE5408C42FF582EE5407240983F590
:10DE7800F0E055F0F005A7227FBFDFEFF7FBFDFECE
:10D47C00FDA42582F582E5F03583F583ED22905FDE
:10D48C00B47A0475F00512D47C7D05805E7A058033
:10D49C00027A04547FC0E0C083C082C39420500140
:10D4AC00E4905F6412D48F802E9060C27A05800560
:10D4BC0090617F7A0675F00712D47C7D07802C7AF8
:10D4CC000580027A06C0E0C083C082C3942050015C
:10D4DC00E490610F12D4C1D082D083D0E022905E50
:10D4EC00D875F00A12D47C7D0A7A07C2D18002D298
:10D4FC00D1C0A7C082C083C007C006C0E030D1092C
:10D50C0075A704E493FDE493FAEEFB75A704EBFE18
:10D51C00EAFC7901D9067908E493F5D4E5D423F52E
:10D52C00D420E01612DE580EDCEA0FDDE1D0E0D09C
:10D53C0006D007D083D082D0A72212DE2880E890B4
:10D54C005E1875F00E12D47C7D0E7A0812D4F7900A
:10D55C005EC075F00212D47CE493FDE4A393FACE82
:10D56C002408CE7C0812D5787C06AD02ED23FD2074
:0ED57C00E00712DE580FDCF42212DE2880F7E2
:10D36700F5D2C2D58036F5D2D2D58030F5D224F6A3
:10D3770050090E0E24A650030E0E0EE5D2F5D275F7
:10D38700F0648485F0D3C2D57009D2D5742012D445
:10D39700CF800312D4BCCE2406CEE5D375F00A8421
:10D3A70085F0D3700A30D507742012D4CF800312CA
:10D3B700D4BCCE2406CEE5D312D4BCE5D222F5D216
:10D3C70075F0648485F0D3C2D58022F5D2C2D580AA
:10D3D70025F5D2D2D5801FF5D275F0648485F0D3B8
:10D3E700C2D57009D2D5742012D4CF800312D4B518
:10D3F700CE2405CEE5D375F00A8485F0D3700A30C4
:10D40700D507742012D4CF800312D4B5CE2405CE0D
:10D41700E5D312D4B5E5D222F5D2C2D58035F5D2FF
:10D42700D2D5802F30E70DF404C0E0742D12D49DBF
:10D437000E0ED0E0F5D275F0648485F0D3C2D570B6
:10D4470009D2D5742012D49D800312D48ACE240425
:10D45700CEE5D375F00A8485F0D3700A30D507740A
:10D467002012D49D800312D48ACE2404CEE5D31291
:05D47700D48AE5D22279
:1075EF00909E7A1275F802DD0D7E00800E7405FEF6
:1075FF00F51EE4FFF51DF51F203C3375A700E4933E
:10760F00700122A3B40204051D8003B4010A051FF3
:10761F00EF2409FFAE1E80E612D4CF7D06B44002E0
:10762F007D03B421027D02EE2DFE80D27E0075A770
:10763F0000E493700122A3B40204051D8003B4017A
:10764F000F051FEF2407FFAE1E80E612D4998008A6
:10765F00B45B0050F612D49D0EB4210280D30EB449
:10766F00400280CDB42C0280C80E0EB45F0280C1E0
:10767F00B45B0040BC0E0E80B8E60812D4CFEE24E7
:10768F0006FED513F422909BB7307409909BBB3044
:10769F007303909BC002760A75F019D5E0FDD5F003
:1076AF00FA12479212DC27744F12DC38744B12DC3B
:1076BF0016C322C250127706124792D2AC12DB8049
:1076CF00304C1212DB80304C0C12DB80304C06D267
:1076DF0050C2ACD322B440E512DB85B4400312DBB9
:1076EF0085B44FED12DB85B44BE712DB8512DB85DA
:1076FF0012DB85C2ACC32230530975F008D5E0FD0B
:10770F00D5F0FA227F0575F019D5E0FDD5F0FA1204
:10771F00479212DC27745712DC38745012DBF57461
:09772F008112DBF5E56312DBF5C4
:10773800E56212DBF578D0E612DBF508B8D7F8E693
:10774800F8795F30E702792FE912DBF512DBF512E1
:10775800DBF512DBF5745812DBF5744312DBF5E444
:1077680012DBF5E8C2E775F00A84C425F012DBF5F0
:107778007864E612DBF508B869F8E612DC161276CA
:10778800C2400122DF02800A20508B75F000808001
:10779800D250C2ACD322127706C250124792D2AC52
:1077A8002002EF12DB80204CE7B440F412DB85B4F2
:1077B800400312DB85B457DAF53812DB85B450D2B2
:1077C80012DB8512DB85F56312DB85F56278D01252
:1077D800DB85F924A0500353015FE924E0400279D6
:1077E8005FA60108B8D8E8780612DB85D8FB12DB5B
:1077F80085FC53040FC4540F75F00AA42CFC249C78
:1078080050027C0078D78601E4B92F02D2E72CF623
:10781800786412DB85F608B86AF812DB85E538600B
:107828000302779A12DB8512DB85C2ACC32290A2D1
:10783800A58003909EC07F2012763B12DD0D02DDED
:10784800F9753400C26B12790512DDF9127CB5E5C1
:10785800166003127861020259127F17121D8912ED
:10786800DD0D10002010010280F8127D2050131247
:107878001D9412783610000D10010280F8121D3682
:0578880080D7127AA573
:10788D0022C26BD22775480A122ABA753400127DAE
:10789D00EDC26A123312106A0512024A80ED12020D
:1078AD004A127C47127D9F127DF978D0E6642660DE
:1078BD0044127F17121D8912DD0D100038100102C0
:1078CD0080F8127D20501BE965156018121D941269
:1078DD00783612DDF110001D10010280F8121D36F0
:1078ED0080BCD26B127DCB751607855917122B33C1
:1078FD007535008096020259127CB5127927127DDA
:10790D00F97F1912794190A2D27E1212763D7E2313
:10791D00E51602D43B90A41F80EF7862E41279380B
:10792D0078D0745F12793818E4F6227F08F608DFF4
:10793D00FC227F7B7E007810742012D49DCE24040F
:10794D00FED8F5227F197E0812763D7E28909EA2E4
:10795D00305303909EA702763DC26B1279271279A0
:10796D0071020259C251127DF990A2CA12795112B7
:10797D001D5C127CB57F2012791012DD0DE516709D
:10798D000512DDEE803675A6FF3051031276B0126A
:10799D004792D2AC200025306DFA1277A1400C121F
:1079AD007D204011127AA5D25180BB105003127860
:1079BD003BC25180D1D25112783680CAC2AC22D28C
:1079CD002775480A122ABA753400C26B127DEDC2B2
:1079DD006A123312106A0512024A80EB12024A1221
:0D79ED007C47127D9F127DF91279FD50DA62
:1079FA00020259909EBB127951121D6E12DD0DC3FF
:107A0A0010001310010510020E80F41277134001C2
:107A1A002212783B80DDD3C2AC22D227C26B7548D2
:107A2A000A122ABA753400127DEDC26A1233121094
:107A3A006A0512024A80EDD26B127C47127D9F12B0
:107A4A007C6F75B901E5BCB2E7F5BC124E2C751610
:107A5A0007855917122B3380CB127CB5E516601FA8
:107A6A0078D0E53D127A96E53E127A96E53F127A8B
:107A7A0096765A08765F12C7A4127DCB027C867F5F
:107A8A003E7E11909E9112760A02DD0D75F00A84EF
:107A9A004430F608E5F04430F60822D26B127DCB6A
:107AAA00127C86E51775F01084240AF54824E850FC
:107ABA000375480A122AC68558592275320012BE21
:107ACA000475A704900700751500127C6F75B9013B
:107ADA00E5BC20E705E515F0801004600D648260BE
:107AEA000975BCFF75B90575B9020515E515242098
:107AFA0050D8E58224FE4003027B9EA882187F00AC
:107B0A0075A7007583078882E0FE75F004A4127CCD
:107B1A001AA9BCAABDABBEACBF1582E0FD75F004C4
:107B2A00A4127C1AC3E995BC404C7052EA95BD4038
:0D7B3A0045704BEB95BE403E7044EC95BF8E
:107B47004037703DEE75F004A404127C1AA9BCAA54
:107B5700BDABBEACBFED75F004A404127C1AC3E93B
:107B670095BC4015701BEA95BD400E7014EB95BE91
:107B77004007700DEC95BF5008EEF00582EDF0154B
:107B870082E5826009C3EF95825003027B120FC31F
:107B9700E89F4003027B0A75A70490070075C70397
:107BA70075C6A8E0F5BCE0F5BDE0F5BEE0F5BF752C
:107BB700B90575B90205C6E58224204006E5C62445
:107BC7002050E00875C70375C68075B901E5BC127A
:107BD7007C04F5BCE5BD127C04F5BDE5BE127C0452
:107BE700F5BEE5BF127C04F5BF75B90205C6E5C64B
:107BF700245850D6E5320470FB75A70022B4FF0164
:107C070022F975A704900700E582686005E06970AE
:107C1700F7E922F5C685F0C775B901E5BC645F7061
:107C27000375BC27E5BD645F700375BD27E5BE64BA
:107C37005F700375BE27E5BF645F700375BF2722BA
:107C470075C703E54875F004A42480F5C6E55975A2
:107C5700F00484A8F00825C6F5C675B901A9BCAA21
:077C6700BDABBEACBF8615EA
:107C6E0022E515242050037515DFE51575F004A4E3
:107C7E0054FCF5C685F0C722E51724204028E517E9
:107C8E0075F00484A8F00824A8F5C675C70375B965
:107C9E0001A9BCAABDABBEACBFA61589BC8ABD8B63
:107CAE00BE8CBF124E2C22E4F516F51579FF127C10
:107CBE006F75B901E5BCB4FF040516A9150515E5E8
:107CCE0015242050E9891579FF75C70375C6A87567
:107CDE00B90109E5BC04601B09E5BD04601509E5A1
:107CEE00BE04600F09E5BF04600905C6E5C6242081
:107CFE0050DD09891722751600751501127C6F75F6
:107D0E00B901E5BC20E70205160515E5152420503E
:107D1E00EB227900E975F004A454FCF5C685F0C792
:107D2E0075B901E5BC20E73078D066702B08E5BD4B
:107D3E0066702508E5BE66701F08E5BF66701905FA
:107D4E00C675B90108E5BC66700E08E5BD6670081B
:107D5E0008E5BE667002D32209E9242050B6C3227C
:107D6E00127D8E127D76A8017F08E0F608DFFB22D9
:0B7D7E00127D8E127D86A8017F08E6B2
:107D8900F008DFFB2278D0796275A704758307EBC9
:107D9900C454F0F58222127C6F78D0127DB9E5BC0B
:107DA900F9C23C20E702D23C127DB97862127DB952
:107DB90075B901A6BC08A6BD08A6BE08A6BF0805D8
:107DC900C622127C6F78D0127DDB127DDB786212BD
:107DD9007DDB86BC0886BD0886BE0886BF08124EB4
:107DE9002C05C62212593E12DEE312857902DD0DF9
:107DF90012DEE37F007E0990A2B712760A7F0A7E1F
:107E090012E5150412D3737F1412C98E121D367F21
:107E1900277E0875130778D0127688E6793E30E711
:107E290002792F7E34E912D4CF7F3D7E0190A43BA5
:107E390012763D20311B3030031290B4C23B1280C0
:107E4900A9127E5FD23B1280A9127E711280F08046
:107E59007C12C00180E6C23B7F4474532017027430
:107E69004E7E0012D4CF8017D23B7F4F7457201714
:107E79000274457E0012D4CF7E06E51E12D4BC7E64
:107E89000CE51D12D4BC7E12E51C12D4BC7E1774FD
:107E99008112D4CF7E1CE51B12D4BC7E22E51A12B6
:107EA900D4BC7E28742E302602742712D4CF7E2D9E
:107EB900E51912D4BC7E33E51812D4BC7E393026BC
:0F7EC90007742C12D4CB7E3BE53702D4BC742D4A
:107ED800201702742B7F707E1512D4CF127EF47E89
:107EE8003A12D31C7E0190A46602760A7E1BE51C1A
:107EF80012D4BC7E21E51B12D4BC7E27E51A12D40D
:107F0800BC7E2DE51912D4BC7E33E51802D4BC1210
:107F18007F95127FC0128297127DF91282EF201787
:107F28001E10021B12483312C7A4127F7D121D4176
:107F38007F347E2F127695127E3212DD0D80E2128A
:107F48001D36203026203128C23B1280A9127FD549
:107F580078661281A9D23B1280A9127FEA78691249
:107F680081A91280F012806402824C12917D80F205
:107F780012C01680EDE57D75F01084AAF075F00A40
:107F8800A42A547FFA78D7E654802AF6227F277EDF
:107F98000879D08700C001D224B9D002C224128344
:107FA80076D001A70010230909EE2406FEB9D7E30D
:107FB8002219EE24FAFE80DB7E3479D7E7A2E79215
:107FC8001712832379D7E7A21792E7F722C224C2B0
:107FD8003B751E007F447E00128333801E1023ED04
:107FE800802AD23BC2247F4F7E0012833BD2247E5C
:107FF80006E51E128368F51E1023E7D2247E0CE5E1
:108008001D128368F51D303BD41023E1D2247E1263
:10801800E51C128368F51C1023E17E1CE51B128306
:0380280068F51BDD
:10802B001023E67E22E51A128368F51A1023E87EE8
:10803B002DE519128368F5191023E87E33E5181224
:10804B008368F5181023E87E393026027E3BE5372E
:10805B00128368F5371023E3227F707E1512832B72
:10806B00C2247E1BE51C128368F51CD2247E21E5FD
:10807B001B128368F51B1023E77E27E51A12836812
:10808B00F51A1023E67E2DE519128368F5191023D6
:10809B00E87E33E518128368F5181023E82278D7A9
:1080AB00E6C2E775F00A847866F537303B057869E8
:1080BB0085F03712811930262BE53775F003A404B0
:1080CB000475F00584FBE51975F00AA4251875F005
:1080DB0006A42BFBE435F0FC12548DF53712548DAE
:1080EB00F5188B1922E563FC339217AB6250031220
:1080FB0054FE305C0A7AD2125279784012541BAE7D
:10810B0004AF037C277D101253848F1C8037E6FD50
:10811B0033921718860418860350031255067A09F2
:10812B00792778C01254188B1EADD3ACD2AB06791D
:10813B00EA78601254168B1DAF06AED27C177D7099
:10814B001253848F1CAF05AE047C037DE81253845D
:0F815B008F1BAF05AE047C007D641253848F1A16
:10816A00ED75F00A84F51985F01822EC3392175050
:10817A00031254FE751D30301786751D2D808178C7
:10818A00427B607CEA800678407B207C4E12C0E10C
:10819A00792778101254168B1CAF06AED280AB30FA
:1081AA00262AE51975F00AA4251875F00AA42537B8
:1081BA00FBE435F0FC7A0512526B8C068B077C00C7
:1081CA007D031253778E048F031280E3E51E75F048
:1081DA000AA4251D75F00AA4251C75F006A4251B02
:1081EA00FBE435F0FC7A0A12526BEB251AFBE43CED
:1081FA00FC7A0A125279EB2519FBE43CFCE43DFDBA
:10820A007A0A12528BEB2518FBE43CFCE43DFD3064
:10821A001703125506A60518A60418A60378D7E66A
:10822A00A2E7923DC2E775F00A84FCABF0303B0E40
:10823A00AB37EC75F00AA42BA23D92E7F622AC37D5
:10824A0080F0128267305C0A7A4012527978D21230
:10825A00541B3017031254FE8C638B6222128277EE
:10826A007A0A12526BEB2518FBE43CFC22E51C75DA
:08827A00F00AA4251B75F00AAF
:10828200A4251AFBE435F0FC7A0A12526BEB25198D
:10829200FBE43CFC221282C912DDF5C202C22312A7
:1082A20082C910000810010510021B80F51031ED83
:1082B20010300D102604D22680E3D230C23180DD88
:1082C200D231C23080D7227F3590A42412763B90DF
:1082D200A44220300F90A45E20310990A4332026BE
:1082E2000390A42B1F7E1712760A02DD0D7F357EC6
:1082F20001909E6D12763D7F347E3A128418744E40
:1083020012D4CF12DD0D12DDF5C2027F347E3AD2D5
:108312001775115975124E802675112E7512278008
:108322001E75113E75122F801675112B75122D8038
:108332000E75114E7512538006751145751257123E
:108342008418E511301702E51212D4CF12DD0D1098
:10835200000810010510020B80F5D23C1017E3D281
:108362001780DF0284134430F8128372E8540F221C
:10837200C2218002D221A22492229223128418E8DE
:1083820030E709D23C7430302102745FF812D4CF46
:1083920012DD0D10003410010510025D80F5D23C93
:1083A200102266102367B43909745F2021DF74300C
:1083B20080DBB45F04742D80D4B42D04744180CD6D
:1083C200B45A04743080C60480C3D23C30240610F0
:0F83D2002237102338B44104742D80B1B42D0428
:1083E100745F80AAB45F04743980A3B43009745AED
:1083F10020219B74398097148094B48908D223E892
:1084010012D4CF800DF8C223800874898001E8025C
:10841100838F90842D8003908429C007EF2408FF67
:1084210012D4FBD00702DD0D0205F8F802050000A9
:10DCAD0075A70090DCDF75F02D84C2D5C2D1601749
:10DCBD00D2D1146007D2D514600DC2D1E5F093FC1A
:10DCCD00742D95F093FB22E5F093FB742D95F09355
:10DCDD00FC220009121B242C353E474F58606870FA
:10DCED007880888F969DA4ABB2B8BEC4CACFD4D964
:10DCFD00DEE2E6EAEDF0F3F6F8FAFCFDFEFFFFFFDB
:10DDA700D23D8002C23DED8BF0A430E70205F0C3FF
:10DDB700E895F020D50425F025F0FEED8CF0A43091
:10DDC700E70205F0C3E995F030D10425F025F0FF0F
:10DDD700203D0B2487500122EF24CC40012202DE94
:01DDE7002813
:10D74B00203A7A7E1C7F5312DE287F5912DE281E68
:10D75B007F5712DE287F5512DE287E2312DE287FAC
:10D76B005712DE281E7F5912DE287F5312DE281F28
:10D77B007E2012DE287F5A12DE287E1E12DE287FC4
:10D78B005212DE28120D54E5BD20E0143006117F35
:10D79B00357E1C90D807E571700390D81102D4FB2D
:10D7AB00E5716018E57012DCAD781F79567D0912B2
:10D7BB00DDAB303A0312D7DA0DBD16F3227E1C7F98
:10D7CB005390D7F012D4FB200CD612C9EA80C0C0FC
:10D7DB00060E30D5021E1E12DE28D0061F30D102D7
:10D7EB000F0F02DE28070700386C446C3800050564
:10D7FB002070D8702005057088A88870080710382D
:10D80B007CFE383838000807102844C62828380012
:10C7C90090A4707F717E2312763D120D54E5BC7ED4
:10C7D9003112D48A30121AC23C120D54E5BCFB75D1
:10C7E900F00AA4F904FAC23D12BDF012CA67303D3D
:10C7F9000122DAF712C96E7C00EBF4042E4019AD60
:10C8090003125377EFA2D1203C077E237F6502D024
:10C81900E9AE16AF1702C90FAD01125377EF12D166
:10C82900D7203C077E237F6502D10DAE16AF1702D4
:10C83900C9337F567E0512C99A7F3D12C9AD7F6FF4
:10C8490012C9AD12C9EA7E0A7F4112CA1D7E227F32
:10C859005912CA1D2012012212BDF0857A1D855E6A
:10C869001C857B1B855F1A7AC0C23D12CA63203DB5
:10C879005212C96E7C007D1412537774562F20D141
:10C88900029F9FFF24CB40028037EF24885002800B
:10C8990030EA1475F00384FE12DE28C3E51B957B8C
:10C8A900FEE51A955F92D55004EEF404FEEEC3132B
:10C8B900FE24E0400C741F2E30D5029E9EFE12DE2F
:10C8C90028DAA8227F5212C8DF7F5A12C8DF7517EB
:10C8D90053751600802B7E0012DE580EBE12F92207
:10C8E9007F157E28742012D4CF7F1C7E2812DE5833
:04C8F9000EBE40F936
:10C8FD00223012E712C8E975171575162DD23C02B4
:10C90D00C7E2C23D6002D23D92D175F080305C0429
:10C91D00F5F08001A4A2E792D5E5F075F03284F828
:10C92D00E5F075F00584C0E0E5F0A2D533C0E0E890
:10C93D00601E12D4BCEE2406FED0E0F8D0E012D476
:10C94D00BCEE2406FE742C12D4CF0E0EE802D4BC1D
:10C95D007420303D07742B20D102742D12D4CF805A
:10C96D00D4C3ED957AFFEC955EFE92D1500312542F
:10C97D00EE227F1512C9867F327E3E12DE28DEFB47
:10C98D00227E0912DE280EBE36F9227E0112DE2825
:10C99D000E0EBE3FF8227E3312DE280EBE40F92267
:10C9AD007E047D1112DE280E0E0EDDF81F1F7E3562
:10C9BD0090A479305C057E3190A47D02763D74059E
:10C9CD00305C097E32740112D48A74067E3612D41C
:10C9DD008A7E3A740012D48A7E3D02D48A7F417ECB
:10C9ED001F7D0F12DE280F0F0FDDF8227F687D03EC
:10C9FD0080047F677D0512DE280FDDFA227F667DBC
:10CA0D000780F37E1F7F5012DE281F1FBF3EF822C6
:07CA1D007D0A12DE280E0E57
:10CA24000F0FDDF722203D07123BB97003D23D22E0
:10CA3400056D12BBB6E4F5F7C2B2C2B2ABF7F5F7B7
:10CA4400C2B2C2B2E5F7FA30E411EB251DF51DE4DC
:10CA5400351CF51C0519EA30E3010ED2B2801578B5
:10CA64000380027801203D07123BB97003D23D22B6
:10CA7400D8F3056DE56D2409F56D12BBB6E4F5F741
:10CA8400C2B2C2B2ADF7F5F7C2B2C2B285F71BF5B6
:10CA9400F7C2B2C2B2E5F7FCD2B2543F30E5024469
:0FCAA400C0CC54C02323F51AE56D24F6F56D229E
:10D672007E017F0990D6F012D4FB2051097E037FF0
:10D6820000743F02D4CFE4FEFFC3E54512CD39FD5D
:10D69200940AED403D9464ED4002746312D36D7EB2
:10D6A200017F09E552240575F02D84AAF075F00575
:10D6B200A4CA75F00B842A90D6DB9312DCADBCB8F9
:10D6C200027BB87D04EE2DF8EF2DF90D12DDA7DDFA
:10D6D200FB227E0312D4BC80C6000C1622222D39F6
:10D6E200444F4F5A66707C7C87939EA9A900090912
:10D6F2000800410000000000888000000000410096
:10D702000800120D68E5BCB4F8339004C3E0602C45
:10D71200FA24F340277F137E0012DE280F0F12DE59
:10D72200280E12DE581F1F12DE580EDAEC7F147E0E
:10D732000012DE280E12DE580EBE12F5229005CC23
:09D74200E0C3941240F60480C714
:10CD3900305D0A75F08AA42480E5F034002220745D
:10CD4900157F017E1190CDC112D4FB7F0A7E0AE5C1
:10CD59002E540702D3847F087E1190CDD112D4FBC3
:10CD690020730C7F0A7E1712DE580E0E12DE587FD2
:10CD7900007E0BE57112CD3912D3737F0C7E11E55C
:10CD890071602F0EE57064B4602864B475F0328464
:10CD9900C0F012D4B5CE2405CED0E075F00584C01C
:10CDA900F012D4B5CE2405CED0E023302D010402F3
:10CDB900D4B590877502760A070FFFFFC473BDAF1C
:10CDC900A463B5FBCDE7FFFF030F0100FFFE03805E
:10CDD900306701227F3F7E00748812D4CFE551600D
:10CDE900F2120D6D85BCF01207E012CD3975F064B1
:10CDF90084F87E06E5F012D3D2E860D77E0002D42B
:10CE0900BC120D6DE5BE70012214600814603BE58B
:10CE19003F1340367F367E00747712D4CF207301DA
:10CE29002279BC87040987031252137E05781DE60F
:10CE390060097E0012D4B5EE2405FE18E6600712DB
:10CE4900D4B5EE2405FE18E68019909D407F377E03
:10CE59000012763DAB60AC611252161F7E09781D37
:10CE6900E6600712D4B5EE2405FE18E612D4B5EE35
:03CE79002405FE8F
:10CE7C0018E602D4B5202C012290CE8B02D4FB05EF
:10CE8C000EFFF0E01CF004F81CFFF0301201227FC2
:10CE9C00637E00909BD212D4FB7F1512C9867F1F34
:10CEAC0012C9867F2912C9867F177E06E53F30E0BE
:10CEBC000B90A48D305C0390A4A180132074077E8A
:10CECC0001909BF2800990A482305D0390A497128C
:10CEDC00760A307306E54E6002154E205718E54E63
:10CEEC00B40113120D77C3E55C9560F5BCE55D9557
:10CEFC0061F5BD124E2C7F217E01E53F30E02130E3
:10CF0C005705909D1D8016E54E7005909D28800D4F
:10CF1C00909BFE12760A7E30E54E02D3D812760A2A
:01CF2C0022E2
:10D23F001252137F207E05751900781DC2D5E63076
:10D24F00D51712D4B5EE2405FE18B818F17E1F7449
:10D25F0063305C02748202D4CF7005B8191880E273
:10D26F00D2D5CE24FACE7484301702742D12D4CFB7
:10D27F00EE2406FE80C8742012D4CB80C8781C80A0
:10D28F000D7F007E23AC5EAB7A125213781DC2D590
:10D29F00E630D50C12D4BCEE2406FE18B818F122D5
:10D2AF007005B8191680EDD2D53017E4CE24FACE1A
:10D2BF00742D12D4CFEE2406FE80D5742012D4CF55
:10D2CF0080D5125213781DC2D5E630D51612D48AE6
:10D2DF00EE2404FE18B818F10E745E305C02742749
:10D2EF0002D4997005B8191680E3D2D53017DACE6B
:10D2FF0024FCCE742D12D49DEE2404FE80CB74201A
:10D30F0012D49D80CBC23D12D3270F0F0E0E746324
:10D31F00305C02748202D4CF125213781DC2D5E64C
:10D32F0030D50C12D4EAEE2408FE18B818F122708A
:10D33F0005B8191680EDD2D5301716740BCE24F818
:10D34F00CE12D4EAEE2408FE80D5740C12D4EA80F3
:08D35F00D5303DCB740A80E5D6
:10D81B007F797E24E55F30E70122AC5F1CAB7B1286
:10D82B005241E51B700E742012D4CFEE2405FE126C
:10D83B00D869800C12D869E51B12D4B5EE2405FE0D
:10D84B00E51A12D4B5EE2405FE742C12D4CF0E0EAD
:10D85B00E51912D4B5EE2405FE745E02D4CF742DF7
:10D86B00201702742B12D4CFEE2406FE22E55F3074
:10D87B00E70122AC5F1CAB7B125241E51B700E74AF
:10D88B002012D49DEE2404FE12D8C2800C12D8C2F2
:10D89B00E51B12D48AEE2404FEE51A12D48AEE2478
:10D8AB0004FE742C12D49D0E0EE51912D48AEE24AC
:10D8BB0004FE742A02D49D742D201702742B12D4EB
:06D8CB009DEE2404FE2284
:10D0D9007F097E2530040512D1D38028A275E57910
:10D0E900C23D6002D23D92D175F080305C04F5F00A
:10D0F9008001A4A2E792D5E5F075F03284F8E5F055
:10D1090075F00584C0E0E5F0A2D533C0E0E8602AF7
:10D1190012D4EAEE2408FED0E0F8D0E012D4EAEE08
:10D129002408FE0F0FE52B5403701F746012D4CF2F
:10D139001F1FEE2404FEE802D4EA740C303D067485
:10D149000A20D1010412D4EA80C9205904742E801E
:10D15900DC205804747F80D5748080D13004051296
:10D16900D1D38028A275E579C23D6002D23D92D122
:10D1790075F080305C04F5F08001A4A2E792D5E552
:10D18900F075F03284F8E5F075F00584C0E0E5F05B
:10D19900A2D533C0E07F3E7E1CE8602012D54BD07B
:10D1A900E0F8D0E07F3E7E2812D54B7F447E327472
:10D1B9002E12D4CF7F3E7E37E802D54B303DE07446
:10D1C9000A20D1010412D54B80D59005CAE075F02B
:10D1D9000A84F8E4C5F0C2D522301105E54AB40243
:10D1E90050C39006E9E0957AFB9006E8E0955EFC6D
:06D1F90050031254FEEC8D
:10D1FF00C31360047B63800FEB13FB249C40F52467
:10D20F004F4004C20480079005CAEBF0D204900689
:10D21F00E6E09006E8F09006E7E09006E9F0E55EBC
:10D22F009006E6F0E57A9006E7F02212D21D80DE36
:10CAB300E54424F64001227800E552206607C39539
:10CAC30070500224B40475F00384F9E928FE24C4E9
:10CAD3005001FE12CAF512CB011E12DE28C3E998DB
:10CAE300FE5003243CFE12CAF51E12DE2808B81FAE
:10CAF300DA22EE2420FE24C250032402FE22E8247C
:10CB0300F1E8C2D55006D2D5E8F4241F23FF90CB19
:10CB13008393CF0493FAE545F5F0A4ACF0FB1252EE
:10CB2300A2E544F5F0A49BFBE5F09CFCEB2420FB81
:10CB3300EC3400FC12CB64FAE5458FF0A430E70235
:10CB430005F0E5F020D502F4042A75F00520190359
:10CB530075F00384FF24DF50027F20C374329FFFEC
:10CB630022EC24F0500BEB2460EC340090CBD393F5
:10CB730022EB33FBEC33FCEB33EC3390CBA393226C
:10CB8300FF00FF03FA0BF318EA2ADE40CF58BE7307
:10CB9300AB8D96A880C068D64FE835F51BFD00FF26
:10CBA30000080B0E101214151718191B1C1D1E1F3D
:10CBB30020212223242526262728292A2A2B2C2D07
:10CBC3002D2E2F2F3031313233333434353636373F
:10CBD300373839393A3A3B3B3C3C3D3D3E3E3F3F9B
:10CBE3004042444648494B4D4E505253555658596E
:10CBF3005B5C5D5F60616364656668696A6B6D6EEB
:10CC03006F7071727374767778797A7B7C7D7E7FAF
:10CC1300808182838485868788898A8B8B8C8D8E9D
:10CC23008F9091929394949596979899999A9B9CA7
:10CC33009D9E9E9FA0A1A2A2A3A4A5A6A6A7A8A9C4
:10CC4300A9AAABACACADAEAFAFB0B1B1B2B3B4B4F3
:10CC5300B5B6B6B7B8B9B9BABBBBBCBDBDBEBFBF2D
:10CC6300C0C1C1C2C3C3C4C5C5C6C7C7C8C8C9CA72
:10CC7300CACBCCCCCDCECECFCFD0D1D1D2D2D3D4C0
:10CC8300D4D5D5D6D7D7D8D8D9DADADBDBDCDDDD16
:10CC9300DEDEDFDFE0E1E1E2E2E3E3E4E5E5E6E671
:10CCA300E7E7E8E8E9EAEAEBEBECECEDEDEEEEEFD3
:10CCB300EFF0F1F1F2F2F3F3F4F4F5F5F6F6F7F73A
:10CCC300F8F8F9F9FAFAFBFBFCFCFDFDFEFEFFFFA9
:10CCD300E54524FD400122E552206607C3957050C7
:10CCE3000224B40475F00384241FFE24C2500324D9
:01CCF300023E
:10CCF400FE12CD2EEEFD241EFE24C250032402FE9D
:10CD040012CD2EE544240275F00520190375F003B5
:10CD140084F4042432FF24EE500F12CD23AE051EFA
:10CD24001E7C0512DE280EDCFA227F1512DE280F87
:05CD34000FBF2DF822E5
:10D58A007E00206615E5700475F0B484E5F075F048
:10D59A000384FE6004C3743C9EFE745312D5B574B2
:10D5AA005712D5B5744E12D5B574457F2F12D49D36
:10D5BA00BE00077E3C12D49D7E00EE240875F03C26
:10D5CA0084AEF00F0F0F12DE280E12DE280F12DEC5
:10D5DA00281E12DE28EE240775F03C84AEF02230B5
:10D5EA00745C301259E54AB4040122B4060122E5FA
:10D5FA007112CB4D8F057C037E1E30662AE57004BE
:10D60A0075F00384241EFE24C6501C24FB500424F7
:10D61A00038013C00612D631D0E024C67C0160060E
:10D62A000C1460020C14FE12D63D0EEE24C1400208
:10D63A00DCF5228D0712DE280FEF24CE50F722E503
:10D64A0053206607C39570500224B40475F003840E
:10D65A00241FFE24C250032402FE12D6680E7F2322
:08D66A0012DE280FBF2DF9228A
:10DD5E00AF177E00E53C12D3677E0C742E12D4CF23
:10DD6E007E12E53B12D3677E1E742E12D4CF7E2414
:10DD7E00E53A02D3677E0E78ADE612D3D27E1874E2
:10DD8E002C12D4CF7E1B18E612D3D27E25742C1201
:09DD9E00D4CF7E2818E602D3D28E
:10CF2D007F797E00E54012D3D27E0A743B12D4CBBA
:10CF3D007E0CE54102D3D27F797E16743B12D4CBA1
:10CF4D007E18E53F12D3D27F797E0078AEE612D3FC
:10CF5D00D27E0A743B12D4CB7E0CE53E02D3D23086
:10CF6D005EE52043E27F6D7E0078AEE612D3D27E81
:10CF7D000A743B12D4CB7E0CE53E12D3D27F757E64
:10CF8D000075F00A84E5F012D4EA0F0F7E08743AAA
:10CF9D0012D4CB1F1F7E0DE53F75F00A84C0F01231
:10CFAD00D4EAEE2408FED0E002D4EA851C1E851BCF
:10CFBD001FAB1BAC1C305D0A7A1B125279783212F2
:10CFCD00541BC3EB33FBEC33FC923D12524A303D04
:10CFDD00087409F51DF51CF51B7F75E51D60157EA3
:10CFED002412D4EA7E2CE51C12D4EA7E34E51B1201
:10CFFD00D4EA803D7E22E51C601912D4EA7E2AE532
:10D00D001B12D4EA7F787E31742E12D4CB7F75E556
:10D01D001A8019E51B12D4EA7F787E29742E12D45A
:10D02D00CB7F757E2DE51A12D4EAE5197E3512D423
:10D03D00EA7F777E3C125BD4851E1C851F1B227FE9
:10D04D00397E1F12DE280FBF40F9781F79567A00FE
:10D05D007D1A12DCAD12DDABEA2406FABAAEF37816
:01D06D001BA7
:10D06E00C3E5119570500224B4FA604214603E1468
:10D07E00603A2450603A146036EA24A540278A1E8E
:10D08E00751D007D1912D09E0D30740312D09E0DA9
:10D09E00781F7956AA1DEA12DCAD12DDAB0AD3EA6F
:10D0AE00951E40F2228A1D751EB380D70808080807
:10D0BE007F367E1C90D807E571700390D81112D47C
:0BD0CE00FB7F3CAE0090842902D4FBE5
:10DA2E00787512DA7E7453201702744E207406E550
:10DA3E002E54074430AF1712DAA87E3BE57DC4544E
:10DA4E000F12D4BC2074077E07742012D4CF7878BE
:10DA5E0012DA7EE5172409FF745720170274452049
:10DA6E007402742012DAA87E3BE57D540F02D4BCFA
:10DA7E00E6FD3392171886041886033017031255E5
:10DA8E0006791778701254168B13AF06AED27C003F
:10DA9E007D641253848F148D15227E0012D4CF7E96
:10DAAE0007E51312D3847E19748112D4CF7E20E53C
:10DABE001412D3677E2B742E2073030E742C12D483
:08DACE00CF7E2FE51502D3679E
:10DC3D00E54A602E7A2420E00E7A26141460087AC4
:10DC4D0028141460027A297F667E01EA12D4CF204F
:10DC5D005505205406800B745B8002745C7E0012A7
:10DC6D00D4CF20110778A9B60007802130261EC217
:10DC7D0026909C957F681275F87F66A85AE54AB480
:10DC8D00060108E875F06484E5F012CFA620080FB0
:10DC9D00E537640260097F367E2E744112D49D22D1
:10D8D10020144F740512DECFEF33EE33F9EF03035B
:10D8E100541FF5F090D924E993A4C5F013C5F013A2
:10D8F100C5F013C5F013C5F0135403FCE5F013FB99
:10D90100E9242093C9244093C39BC4540FFBE99C91
:10D91100C4FC540FF9EC54F02B2446F57BE934F6A2
:10D92100F55F22FFFFFFFFFFE6C5AD9C8F857D7789
:10D93100726E6C6A696A6A6C6F747A828D9DB4D9F1
:10D94100FFFFFFFAE9DCD3CEC9C6C3C0BEBBB9B77E
:10D95100B5B4B2B0AFADABAAA8A6A4A2A09E9C9943
:10D9610096918C00381CE735D137246F00C5B3C1BF
:10D97100E61F66B60E68C21867AADBF4EDB94675F4
:03D9810010A200F1
:10DEAF00D2A27408D2A1D2A300C2A3C2A1D2A3004E
:10DEBF00C2A3D5E0EF7405D2A300C2A3D5E0F82228
:10DE8800C2A3D2A2D2A1D2A300C2A375F008339232
:10DE9800A1D2A300C2A3D5F0F5C2A175F003D2A305
:07DEA80000C2A3D5F0F8222F
:10C3EA0012DE88D2A300C2A3C2A175F008E4D2A3C8
:10C3FA0000C2A3A2A233D5F0F5FE75F008E4D2A3D9
:10C40A0000C2A3A2A233D5F0F5FFD2A300C2A32291
:10C41A00E478806608B88BFB70012274D512C3EAEF
:10C42A007881C3EE13FEEF13F692D118EE2460F66C
:10C43A0074D612C3EA7888EF33CE33CE33CE33CEF6
:10C44A0033A2D192E25407FCEEFB7A0812526BEC4B
:10C45A00244FF608EBF674D912C3EAEF543F7882F8
:10C46A00F67886EF33CE33CE33CE33CE335403F65B
:10C47A0008EEF618161608E6C4FF54F0F618E6C4D5
:10C48A00CF540F2FF674DA12C3EAEF232354FC7841
:10C49A0083F67884EEF608EF54C0F67880E46608EE
:10C4AA00B88AFBF62212C3F27889C3EF96FF18EE18
:08C4BA0096FEA2E79216501055
:10C4C2001254EE740FF8F91252B8EF2CFFEE3DFE43
:10C4D200788BEEF608EFF622E6182016072CF7E620
:10C4E2003D19F722C39CF7E69D80F66A405E8056AE
:10C4F200E050F04B0044803DC0384031D02BA025A5
:10C50200601F2018D014000F000AA0014401580136
:10C51200680178018801A001B401D001EC02100287
:10C5220038026802A002DA030C034D78BE8020852F
:10C532008E8A9D8F4D95BA9A97A0BEA631AC53B202
:10C542002AB801BD6AC1EDC4D1C78812C3F2788D81
:10C55200EEF608EFF67887798C1252B878837990E4
:10C5620012C4DA7885798C1252B87881799212C421
:10C57200DA788DE624E4FE08E63392D13392D5547C
:10C58200FCFFEEA2D133A2D533FE780F799212527C
:10C59200B878947990C3EC97F61819ED97F67994D8
:10C5A20090C4ED7F1F7D11EF93C3971F19EF9397EF
:10C5B2001F091DED600240EF0F90C50D798DEF93BD
:10C5C200F7090FEF93F7788E79941252B890C52D30
:10C5D200EF93C39BFB1FEF939C2420FC7897E62BE1
:10C5E200F618E63CF618E436F6740612DECFD237B9
:09C5F200EE24F740062402500279
:10C5FB00C237EEFCEFFD740712DECFC3ED9FFFECED
:10C60B009EFE78B7E6FD337C0050011CEF2DFFEE4C
:10C61B003CFE789CEF26F618EE36F62220141220FC
:10C62B00370F789DE6B4050912C6D812C70D12C78D
:10C63B0056222014577897799A12C787125476C3CB
:10C64B00EE9420FE924550031254EE7C007D0512B1
:10C65B0053843045031254EE8E618F60E531B40C78
:10C66B002B12DA14E56120E71124F8500DFAC3E51B
:10C67B00609AF560E5619400F561120D77E5BC25D4
:10C68B0060F57AE5BD3561F55E12DA217897799A16
:10C69B00C3E697FB1819E697FC7A0212526B3037F8
:10C6AB000B7A0212526BECFEEBFF800312C6D81210
:10C6BB00C70D20140312C75678957998E6F77600C4
:10C6CB000809E6F776000809E6F7760022799CE779
:10C6DB007700FB19E77700FC789DE6B40506EB3392
:0EC6EB00FBEC33FCECA2E792D550031254FE98
:10C6F9007A32125279ECFBEDFC30D5031254FEEC80
:10C70900FEEBFF22EE2408FE74042037167406306F
:10C719007511789DE6B40504740C8007F42406C3EA
:10C7290023540FFD7C00125257789FE6FC08E6FB64
:10C73900C374109DFA125279EFF8EEF9125476E8A3
:10C7490078A02FF6FF18EE39F62480FE2292754064
:10C75900031254EE78BBE6F5F02438400375F0E196
:10C76900EF33EE3378A8F6A485F07930E70205793E
:10C77900C276307508E57924F15002D27622E6278F
:10C78900FB1819E637FC1819E637FD2212BD977F09
:10C79900087871793A12C7B00249FE855E63857AD5
:10C7A90062787379647F06E6F70809DFFA2278640C
:10C7B900797380F1787379AF80EB78AF797380E51D
:1051F100E4FEFFFC7D0A791DE7540F2FFFE43EFE1C
:10520100B9190280061912525780ED301703125452
:10521100EE22305C2BEC33921750031254FEEC2437
:10522100D950047C277B007AD2125279EB33CC33EC
:10523100CD33CC33ED33FBEC33FC3017031254FE8A
:10524100EC33921750031254FE791912548DF70959
:10525100B91DF8A70322EFF88DF0A4FFEDC5F0CE3C
:10526100A42EFEEC88F0A42EFE22EB8AF0A4FBE52E
:10527100F0CC8AF0A42CFC22EB8AF0A4FBE5F0CC64
:105281008AF0A42CFCE435F0FD22EB8AF0A4FBE5C6
:10529100F0CC8AF0A42CFCE435F0CD8AF0A42DFDED
:1052A10022EB8AF0A430E70205F0E5F0CC8AF0A405
:1052B1002CFBE435F0FC2286F0E7FDA4FAABF019F3
:0652C100E786F0A42BFBC0
:1052C700E435F0FC18E68DF0A42BFBEC35F0FCE49C
:1052D70033FDE687F0A42CFCED35F0FD22EB89F0D9
:1052E700A4CBAEF08AF0A42EFEE5F03400FDEC89E5
:1052F700F0A42EFEE5F03DFDE433CC8AF0A42DFDAD
:10530700E5F03CCEFC22EB89F0A4CBAFF08AF0A409
:105317002FFFE5F03400FEEC89F0A42FFFE5F03E07
:10532700FEE433CC8AF0A42EFEE5F03CFCED89F0D8
:10533700A42EFEE5F03CFCE433CD8AF0A42CFCE57A
:10534700F03D8E058C068F04FF22C2D5EC30E705B1
:10535700B2D51254F6EE30E70DB2D51254EE125311
:10536700841254F6800312538430D5031254EE226C
:10537700C3EC13C0E0ED132FFFD0E03EFEBC000BE3
:10538700BE0029EF8DF084FFADF022E4CCF975F073
:0453970008EF2FFFED
:10539B00EE33FEEC33FCEE9DEC994005FCEE9DFEEE
:1053AB000FD5F0E9E4CEFD22EDF9F5F0EE8420D235
:1053BB001CFEADF075F008EF2FFFED33FD400799A4
:1053CB005006D5F0F222C399FD0FD5F0EA22EC334B
:1053DB00EE3400FEEF3400FF7D007A00790078098F
:1053EB00C3ED9AFDEE9BFEEF9CFFB392D54009ED0A
:1053FB002AFDEE3BFEEF3CFFA2D5E933F9ED33FD81
:10540B00EE33FEEF33FFD8D92279007A00C3801533
:10541B0079007A00C3EA13FFE913FEE8132BFBEEC6
:10542B003CFCEF3DFDE4F5D2F5D333FE7F19C3EE23
:10543B0098FEE5D299F5D2E5D39AF5D3B392D54040
:10544B000DEE28FEE5D239F5D2E5D33AF5D3A2D548
:02545B00EB3331
:10545D00FBEC33FCED33FDDF0122EE33FEE5D23301
:10546D00F5D2E5D333F5D380C3EDC454F0FEECC4CF
:10547D00FF540F2EFEEF54F0FFEBC4540F2FFF22FD
:10548D00EC75F00A84FCEB54F025F0C475F00A8439
:10549D00C4CBC454F025F0C475F00A842BFBE5F0A1
:1054AD0022AC10AB1112548DA904AD03FA7C197BFB
:1054BD009912526BAE04AF03EA75F006A4F8AC1264
:1054CD00AB1312548D2875F00A8485F014F8EF2B68
:1054DD00FFEE3CFEEF28FFE43EFEE43DFDE439FC2B
:1054ED0022C3E49FFFE49EFE22E4C39DFDE49CFCE9
:1054FD0022C3E49BFBE49CFC22C3E49BFBE49CFCE9
:10550D00E49DFD2275D4107B807A0079807800EAC5
:0A551D00F5F0A4FCADF0EBF5F0A4EE
:10552700FEAFF0EB8AF0A4C333C5F033C5F092D5D4
:105537002DFDC5F03EFEE430D501043FFFB5150D46
:10554700EEB51409EDB51305ECB51201224006EAD4
:1055570098FAEB99FBD5D40ABB0001220ABA0001DD
:105567000B22C3E913F9E813F8EA28FAEB39FB80B1
:10557700A478087B807D807C00EDF5F0A4FAE5F047
:105587008EF0B5F007EA8FF0B5F001224003ED9BEE
:10559700FDD827BDFF0122EDF5F0A4F9A8F0ED0431
:1055A700F5F0A4C399FAE5F09813CA1329F9E83A74
:1055B700F8C3E99FE89E50010D22C3EB13FBED2BC7
:1055C700FD80B6C374689511FB74019510FC8004C7
:1055D700AC10AB117A0B79B81252E480177473F8D8
:1055E700F9E627FB0809E637FC0809E637FD30E747
:0555F70003125506EB54
:1055FC0033FBEC33FCED3323FD242083F8ED241C2A
:10560C0083FFED241883FAED241483F9EF99F9E85C
:10561C009AFA1252E4EF9DFFE89EFE22FFFFFFB6BE
:10562C00FED7FD63FB5DF8C4F59BF1E3ED9EE8CF7F
:10563C00E379DD9ED743D06BC919C153B91CB0793E
:10564C00A7709E06943F8A237FB674FF6A045ECBD4
:10565C00535B47BB3BF1300423FB17DE0BB2FF80DF
:10566C00C21DC232532CF8C3E5679576FBE56895ED
:10567C0077FCE5699578FD30E705D2611255062473
:10568C00F05003125740AA06A90712530DEC2480C0
:10569C00E43DFBF9F51AE43EFCFAF519E43F60022F
:1056AC00D2321252E48B128C138D148E15C3E56416
:1056BC009573FBE5659574FCE5669575FD30E7051E
:1056CC00D262125506EBF9F51FECFAF51DED6002EE
:1056DC00D232303201221252E4EB2512F512EC35A3
:1056EC0013F513ED3514F514EE3515F51540E102EF
:1056FC00551112566C20323BEB242E40D3EA240178
:10570C00CB3400FC7A07793D1252E4C010C0118EE4
:10571C00108D118C128B13E4FCFD7E077FD012B41C
:0E572C00B4851203851302D011D010BB000506
:10573A00BA0002D21D22B261C374809BFB74F59C2D
:10574A00FC74209DFD22204D69204866303F637F0E
:10575A00697E0112C99A7E1F12CA0A75A7009004AF
:10576A00EDE0A2E792171392E7FC1582E013FB30F3
:10577A0017031254FEBC003AEB603720E73420E6E8
:10578A003110E513201707C3741F9BFE80027E1F8A
:10579A0012C9FF0EDBFA22FB2017097E00C3742010
:1057AA009BFB8008EB241FFE74209BFB12C9F90E99
:1057BA00DBFA2275A700758307E559C4440FF58201
:1057CA00E0A2E792522212C7BD1257BDC2E775F096
:1057DA000A84FEAFF075A7045382F1786412584622
:1057EA00AE07786712584675A700E57DC4540FFEC8
:1057FA00E57D540FFF787312583AAE07787612583F
:10580A003A74AF1255E61256FE8B148A1312080D1B
:10581A00ACCCAB017A0A12526BE5139B9004ECF004
:10582A00FBA3E5149CF0FCA2E7923DD23F02C7C35A
:10583A00860308860408860518188006E0FBE0FC43
:0A584A00E0FD7A0A12528B20E70CF1
:10585400EB2EF608E43CF608E43DF622C3EB9EF694
:1058640008EC9400F608ED9400F622204D09204837
:1058740006C23F302A0522C23380F6E54824F640AA
:10588400F5E5580460F075A700758307E559C4244D
:1058940008F582E0FEA3E0FF12080D7437125932B6
:1058A400500B30381BC23878C586468013743212C8
:1058B4005932400C203809D23878C5A646754600BE
:1058C400740D125932404A1257D0303D38201122FB
:1058D400204D1F20481C204019BCFF16EB243250D9
:1058E40011D240120D4FE5BF75F019A4F536D22E32
:1058F400D22F205238E55965586032204D2F204868
:105904002CD2338028201109204D062048037536F7
:1059140000303319204D1220480F1290510559C3FD
:10592400E55895595003855859C233C2402229FB82
:10593400E435CCFCC3EB9FEC9E22E558B4FF012276
:1059440085581175A704758307E54824F65002802D
:105954005C201259202905202A02805112C7BDE477
:10596400F516F5177510001259CAE510700312C721
:0B597400B71259E3302910E51B25177E
:10597F00F517F51BE51C3516F516F51C1259F01227
:10598F00C7B70510C3E511951050D175A70002C711
:10599F00C3E55AF51124F6500375110A75A704755E
:1059AF0083067510001259CA1259E31259F00510E7
:1059BF00C3E511951050EE75A70022E510C4F582CE
:1059CF00E0E0F564E0F565E0F566E0F567E0F568C1
:1059DF00E0F5692275A701125DDC123E1A75A70466
:1059EF0022E9F0E51CF0E51BF022E510C454F0F5B8
:1059FF0082E0F512E5822406F582E0F511E0F51C50
:105A0F00E0F51B22E512B426157F757E34740D1256
:105A1F00D4EA20442575110012D04C025B417F6DF2
:105A2F007E3BE012D4CFE5137E3512D4CFE5127E44
:105A3F002F12D4CF20440312D04C12CFB8025B41A7
:105A4F00202852E558B4FF012275A704758307E596
:105A5F0059F51030330965586005204802051012BA
:105A6F0059F9E0F513305E07204304E5376095E000
:105A7F007F797E3D12D49DE5137E3912D49DE512B8
:105A8F007E3512D49D30480B7F7F7E3512DE280E77
:105A9F00BE40F980392012012275A704758306854F
:105AAF005B101259F9305E0A204307E53770030285
:025ABF005C6326
:105AC100E512700B7E3A7F79745D12D4CF800D752B
:105AD100F06484E5F07E397F7A12D41FE537B40291
:105AE10005128EE98045B403028040E51C7006E58D
:105AF1001B24FB5036E511F964B4602F20062CE518
:105B010037600D200C0AC3E99570F9500324B4F9EC
:105B1100E912DCAD781D79547D1D90D7F9E53F2060
:105B2100E00390D80012DDAB12D4FB75177975161E
:105B31001930280375161DE51264266003125B8473
:105B410075A7009006E3E511F0A3120D68E5BC7599
:105B5100F01970040475F014A4951BFBE5F0951C75
:105B6100FC922450031254FEECF0A3EBF0C24FC29E
:105B710063EC700EEB24E64002D24FEB24C84002E6
:105B8100D26322E51C24ED402BAE1CAF1B125DA697
:105B91007C007D32125384C005EFAF17AE1612D3CD
:105BA100D8CE2405CE742C12D4CF0E0ED0E0231201
:105BB100D3D2801B125D9D125BDECE2405CE742CE8
:105BC10012D4CFCE2402CEE875F0058412D4B5CE1E
:105BD1002404CE7422305D02748302D4CBEE243DC2
:0D5BE10050047EC37F4B7C017DF412538481
:105BEE00C004C005EF6007AF17AE1612D3D8D007AA
:105BFE00D0067C007D32125384A805EFAF17AE1687
:105C0E00CE240ACE02D4B5125D9DEE2450305D0333
:105C1E00EE24A150047EC37F4B7C017DF41253848D
:105C2E00C004C005EF6007AF177E2F12D425D00732
:105C3E00D0067C007D32125384C005EFAF177E373D
:105C4E0012D48A7E3B742C12D49D7E3DD0E075F02A
:105C5E00058402D48A7F6D7E2F746312D4CFE51231
:105C6E0075F06484E5F07E3512D36712D04C02CF06
:105C7E00B830480320740122E4FCF5A79006E3E057
:105C8E00F9A3E0FE24FE40EFA3E0FF7D78E5376048
:105C9E0008304FE3200C2A800B120D54E5BD20E096
:105CAE0010304F0DD206E57124FE5015125D938013
:105CBE00107D3CE546600A7D141460057D0A147063
:105CCE00B689111252577D6F125377BE00A9EF2479
:105CDE00E240A4AD07E51112DCAD202404B2D5B22A
:105CEE00D1781F795612DDABA806A907E511242D30
:105CFE0075F0B484E5F012DCAD7407304F02740E0B
:105D0E00FDFA12DDABB2D5B2D112DDABB2D5B2D146
:075D1E00DDF0AD0212DDAB68
:105D2500850616850717B2D5B2D112DDAB85061EDD
:105D350085071F7A03304F027A06E511241675F0A0
:105D4500B484E5F012DCADA816A917AD0212DDABDF
:105D5500DDFBE51124EA400224B412DCADA81EA93E
:105D65001FAD0212DDABDDFBE5377021304F1E9014
:105D7500A545305D0390A5417F3C7E3312763D12EB
:105D85000D54E5BD20E00612CA1012D79A22C3E9C8
:105D95009570500224B4F922E51B2402FFE4351C5A
:105DA500FE305D1ABEC305BF4D028012AC06AB07BF
:105DB5007A1B125279783212541BAE04AF03227843
:105DC5007379641255E81256FE751CC3751B4B207A
:105DD50032048B1C8A1B22125DC430320122AC199D
:105DE500AE1AA91DAF1FB90005BC00028010C3E99A
:105DF50013F9EF13FFC3EC13FCEE13FE80E8BF2984
:105E0500005006BE2900500122C3EF13FFC3EE1355
:105E1500FE80EB3E7FE3E3E3E3E3E3E3E3E3E37FFA
:105E25003E0C1C3C7C7C1C1C1C1C1C1C1C7F7F3ED3
:105E35007FE3E3E3070E1C3870E0E3FFFF3E7FE3FB
:105E4500E3030F0E0F03E3E3E37F3E070F1F3F77E7
:105E5500E7E7FFFF0707070707FFFFE0E0E0FEFFB3
:105E6500030303E3E37F3E1E3F73E0E0E0FEFFE351
:105E7500E3E3E37F3EFFFFE3E30303070E1C38384C
:105E85003838383E7FE3E3E37F3E7FE3E3E3E37FB8
:105E95003E3E7FE3E3E3E37F3F030303E77E3C000E
:105EA5000000181818FFFF1818180000000000005F
:105EB500000000FFFF0000000000003FF000003878
:105EC5001C38F00180C1F020F0FC0038F03FE00004
:105ED5000000007CC6C6C6C6C6C6C6C67C183878CD
:105EE5001818181818187E7CC6C60C183060C0C65D
:105EF500FE7CC6C6061C0606C6C67C0C1C3C6CCCC5
:105F0500FE0C0C0C0CFEC0C0C0FC0606C6C67C3CD4
:105F150066C0C0C0FCC6C6C67CFEC6C6060C183028
:105F25003030307CC6C6C67CC6C6C6C67C7CC6C6F6
:105F3500C67E060606CC78000018187E7E18180066
:105F450000000000007E7E00000000000000000050
:105F55000000000000C6E2E2D2D2CACAC6C6C2002C
:105F65000000000000000000008080A0C0A00030FC
:105F75004020C08080C0A0A0000060A0600000A0FC
:105F850040A05098D090882050A850888850A8509C
:105F95002060806000000040E040000000000080BC
:105FA5000000E000000000000040002040800040AC
:105FB500A0A0A04040C04040E0C02020C0E0E020BC
:105FC5004020E02060A0E020E0C02020C06080E00C
:105FD500A0E0E020404040E0A0E0A0E0E0A0E0201C
:105FE500C0004000400000800080002060E060208C
:105FF50000E000E00080C0E0C080E0E0E0E0E0001C
:106005000000000040A0E0A0A0C0A0C0A0C040A02B
:1060150080A040C0A0A0A0C0E080C080E0E080C01B
:1060250080806080A0A060A0A0E0A0A0E0404040EB
:10603500E0202020A040A0A0C0A0A080808080E01B
:10604500A0E0A0A0A0A0E0E0E0A040A0A0A040C0EB
:10605500A0C0808040A0A0C060C0A0C0A0A06080FB
:106065004020C0E040404040A0A0A0A060A0A0A06B
:10607500A040A0A0A0E0A0A0A040A0A0A0A040405B
:1060850040E0204080E02020A870202070A820203B
:0D60950008F030D0100000F0A8A8000000B6
:1060A200E0000000902048708898984000E0E0E00E
:1060B20000A0E0E0E04060301030604040E040404E
:1060C20060909090909060206020202020706090DE
:1060D20010204080F060901020109060103050909E
:1060E200F01010F080E010109060609080E09090CE
:1060F20060F010202040404060909060909060607E
:10610200909070109060C0E0F0F8F0E0C0000000E5
:10611200000000000000000000000050605000700D
:106122007050000078807008F000F8888888F800C5
:10613200C0C8102040981800C0B098B0C0006020BD
:1061420040000000000090D8FCD8900000246CFCB5
:106152006C24000020A870A82000002020F8202035
:106162000000000000000080000000F000000000BD
:1061720000000000606000081020408000708888E5
:106182008888887020602020202070708808102065
:1061920040F8F810201008887010305090F8101055
:1061A200F880F008088870304080F0888870F8081D
:1061B2001020404040708888708888707088887885
:1061C20008106000606000606000000080000080D5
:1061D20000002040F84020000000F800F800000015
:1061E2002010F81020007088081020002000000005
:1061F2000000000070888888F88888F08888F08815
:1062020088F070888080808870E09088888890E02C
:10621200F88080F08080F8F88080F080808070883C
:1062220080B8888878888888F888888870202020B4
:10623200202070381010101090608890A0C0A0909C
:1062420088808080808080F888D8A8A888888888FC
:1062520088C8A898888870888888888870F0888814
:10626200F080808070888888A89068F08888F0A084
:10627200908870888070088870F820202020202064
:106282008888888888887088888888885020888844
:1062920088A8A8A850888850205088888888885064
:1062A200202020F80810204080F800CCAC9CACCC18
:1062B2000000CCD4E4D4CC0004781828C800FC40F8
:1062C200A04018202018000000000000F800000084
:1062D20000A040A050007888889868708840308874
:1062E20070200000F0A8A8A8A878484848487888F4
:1062F20070888080887020A88898A8C88888805074
:1063020048FC485080304C5C6060603C00E0F00823
:106312000808F88044485C484480F8808080808087
:106322008078484848484888B8A8A8E8A8A8B88803
:1063320088888888F808500070888888708080F083
:1063420088888888F8888888888888F090909090D3
:1063520090F0A8A8A8A8A8A8F8888888F80808082B
:1063620050008888888878A8A8A8A8A8F8080000FB
:1063720000000000000000000000000088888888FB
:10638200E8A8E8A8A8A870A8A8A800000000000033
:1063920000000000000000000000000000000000FB
:1063A200000000000000000000600060600060006B
:1063B20060006060205020000000005090B890D033
:1063C20090886050500070705000882020887000C3
:1063D2000080C0A090F8003048B4B4483000304883
:1063E200B4B44830FC0098D02058C800F8E8D880EF
:0A63F200D8E8F8404050F850404051
:0300000002005E9D
:03000B0002B544F7
:0C000E00206E06859950D26E32D26F32FF
:0E00230010990AC298206DE385994FD26D3274
:10003800E4F537F534F52F12DE1EC229C22AC2684C
:09004800C227C214C215022CDF0C
:03005B00022A6D09
:10B537008530F0C5F065308530F060F722C0D0C0A7
:10B54700E0C0F0C0A775A700C083C08275D008759A
:10B557008A00300503758A7A758CEA0532E5327000
:10B567000215320530E530640A6026201520E531E2
:10B57700B40C0BE530B4010612BA0912D8D1E53183
:10B58700B4180BE530B4060612BA0912D8D102B7BF
:10B597005EC2AFD2C075C07AD2AFF5300531E531A2
:10B5A70064197040F531201529C225C22C7D0A7413
:10B5B7000412DECFEF33EE339005CCF0EE24F540E6
:10B5C700112402400B24014005DDE4022A6DD22537
:10B5D700D22CE5A6600215A678B5E660011678B606
:10B5E700E6600116302E0BE5367007C22FC22E1209
:10B5F700B8EEE5367004C24B8002153678A9E660CE
:10B60700011678D8E66001160535E535700215355F
:10B61700E590307B0B30E008D278C27BC200801AFD
:10B62700307C0B30E108D279C27CC201800C307DBE
:10B637000930E206D27AC27DC202E59044F8F4707E
:10B6470003753500304A09E53324FA50037533058D
:10B65700E5336005153302B703E590F4540770032B
:0DB6670002B703A2E09200A2E19201A2E26C
:10B67400920230100320143D75330820001B201063
:10B684000C2011098013E59030E10E8006E5372483
:10B69400FC40F3E543541FF53320100375A6FF2047
:10B6A4002E5D301004E536705620100C201109E58B
:10B6B4003524F55003753304D21BD2A5D2A612B893
:10B6C400EE75B44075B24078D8E670020534202790
:10B6D4002E20682B202928202A25A2107211501F01
:10B6E400E52054076019E53424375004C24A800F1A
:10B6F4002401400B200026200119D27D7534C82076
:10B704001558E531702412DEAF74E812DE88802A01
:10B7140002B831E53724FC40E6D27C80DF3011DF0B
:10B72400E53724FC40D9D27B80D275F00384E5F060
:10B7340070DE12C4AF74E812DE88E531B406051277
:10B74400C6278016B40C0512C63D800EB41205122D
:10B75400C6278006B4180312C63DE59030E10530D3
:10B76400E202800620100820110520103C807D2074
:10B7740027F82068F52029F2202AEFE53424304008
:10B78400E9240750E5600B205E088590F020F20262
:10B79400740190B7A693D2A5201002C2A512B8D9FD
:10B7A400806FC8A08269554646202F12E536603C5A
:10B7B40024AA500AE53675F01984E5F06040D2A653
:10B7C400201002C2A6D2A5202F0C7418304B02748C
:0EB7D4006412B8D9803BE53675F00C3048039E
:10B7E20075F00684A2E0744640E9743780E5E52BE3
:10B7F2005403600C20100E301106E54A6402600505
:10B8020012B8F4800312B849101B08A25892A5A2DC
:10B812005992A675A700D082D083D0A7D0F0D0E0ED
:10B82200D0D0201009C5A67003022A6DC5A632C267
:10B8320018B40202D21812C54D30180874E412DE90
:10B842008802B73E02B73978A7E5B4600924E04020
:10B8520005760002B8F4E534702920412220751FD4
:10B86200300D1CE57924CE40167AFFE5B110E701D0
:10B872000A2325B3F5B3EA35B4F5B4C313F5B2E63A
:10B8820060021622C2412075028077C246E579FF26
:10B89200605820120424FD5051206502C21CD2655A
:10B8A200EF24B050027F4FEF90B9B99375C703757B
:10B8B200C6FC75B90185BFF0A4E5F0F624F4400298
:10B8C200760C301C2DE5BEC39FF5F0A4E5F024E014
:10B8D200400375F020E5F0C21C79AA770375B30026
:10B8E200F5B4C31375B100F5B222C26578A77680AC
:10B8F200D24179AA7703D21CE4F5B3F5B4F5B1F5D8
:10B90200B222C26579A1E57924CE500DE720E7E2A3
:05B912007628301CDD69
:10B91700743C80BE7680E720E7D3E57997404DC237
:10B927004679AAE7FAE5792323B4C500400274C42F
:10B937002437300E31F42437300D15F7BA0302FAE5
:10B947000AC39AF5B175B300EAF5B4C313F5B22289
:10B95700101C07D21C76C802B8DB763274FF200EA3
:10B9670002749B02B8DBC313247E80CC75C70375B2
:10B97700C6FB75B901E5BD6026C395795004C2467B
:10B98700801D78A720461B301C11E57975F008A4A7
:10B997002432F6E5792324AA02B8D97605D24602DD
:10B9A700B8F4301C077614747802B8D97696C24674
:10B9B70080EDFFF3E8DDD3C9C0B8B0A9A29A948F90
:10B9C7008A85817D7975716E6B6865625F5C595692
:10B9D70053504E4C4A48464442403E3C3A3836342F
:10B9E700333231302F2E2D2C2B2A29282726252597
:10B9F700242423232222212120201F1F1E1E1D1D38
:10BA07001C1CD2B5C28EAE8DAA8DAF8BAB8BE4F565
:10BA17008DF58BD28E3014012278B6BE0007EF2445
:10BA2700E24002800806E624EC50027614206705FF
:10BA3700E624F64005E4FEFAFFFB7C007D0A12527D
:10BA4700577C007D5E1253778F51EE60037551FF6F
:10BA5700EAFC7A3312526BEBF5F0A4E5F0CB8CF0ED
:10BA6700A425E0C5F035E0CB92D525F050060BBBF9
:0EBA77000002D2D530E7060BBB0002D2D5ECA0
:10BA8500F5F0A42BFBE5F03400FC30D5010C78A6CD
:10BA9500E6C39BFF18E608F6EB18F618E69CFE18B9
:10BAA500E608F6EC18F6301401227A0050040A1262
:10BAB50054EE7C007D6E1253778FF078A2E6A4FBDE
:10BAC500ACF012548DEBBA0002F404FAE4F8FFEA84
:10BAD50030E70118E57960062075031FF4042AF59F
:10BAE50079EF38D27520E70860037579FF02C779C9
:10BAF500C2750470F5E579F40460EFF57980EE120E
:10BB05000D4A78BBA6BC120D68E5BE78A2F624F6F0
:10BB15005007E4F5BEF6124E2C120C33E5BEF5487F
:10BB250024F65008E4F5BEF548124E2CE5BFF54362
:10BB350024F3503924F34035120D5E78A1A6BCE5F7
:10BB4500BF789DF61424FB50087403F6F5BF124E1A
:10BB55002C78B7A6BE120D54E5BDA2E39266A2E409
:10BB65009267035403C253B40102D25322740DF5F4
:08BB7500BFF543124E2C80C005
:10005E0078FFE4F6D8FDF4F5A6D2B4D2C075C07A16
:10006E0075D75075AE1375AF017581D87590F8754B
:10007E00EFBC75FDFFD2A412DDF5C2A47450122A96
:10008E0085758951D28C75A882D2BC12BB7D12DEC9
:10009E00AF12C42512BB0412D98412294B7F407EA5
:1000AE0001909B7E12760A124C8D12DDF512DAD675
:1000BE0012DD0D12DE1E7C1412DDFF300003022A4B
:1000CE006DDCF51247E2753A00124830E53A7016CB
:1000DE0012DEE37F437E0690A32712760A12DD0D11
:1000EE003000FD022A6D75A6FF1247E212BB041204
:1000FE00294B12DD0D12DDF112DE1E78B5761E12C1
:10010E00D98412C41AC215C21412294B909BC57FF2
:10011E00781275F8205E0A7F767E12909BD212D4EA
:10012E00FB7F4012DD837F497E0978AEE612D367EE
:10013E007E15743A12D4CF7E1AE53E12D3677E2610
:10014E00743A12D4CF7E2BE53F20E00805A6E5A633
:10015E00700215A6E53F12D3677F5312C98E7F57E3
:10016E007E0B12D29412D31C7F60207303020208FE
:10017E007E0BAC5DAB5C12D29812D31C7E31127624
:10018E00957F697E1212D81F3025087E1290DB3FB4
:10019E0012D4FBE5A60303543FFDFE0D7F7312DE62
:1001AE00280F12DE281EDDF478B5E57124F6400224
:0801BE00761E307419E660564C
:1001C6007F727E16744012D49D7E17E612D4257E69
:1001D6001F745312D49D12DD0D1000371001371015
:1001E6000237124782D2AC75369612DB85B4E0052B
:1001F600124878800AE53670F11247D012DDEE0219
:10020600010D2074097E2BE52E540712D4BC7E17EF
:1002160002018C022A6D022CA58072E53524C85095
:1002260049E59020E244D0E0D0E012027102725E0D
:10023600E53524D25034E59020E22FD0E0D0E0120C
:10024600DEE38038E53524D25020E59020E21BD04D
:10025600E0D0E012DEE3306B0B7F091275EF124E31
:1002660064127AC51202710205AB2212DEE390A374
:10027600E07F001275F812DD0D02DDEE12DEE3906E
:10028600A3E07F001275F812DD0D12DDF1C215C272
:1002960014C227C26812DE1E753701909CB2121C6A
:1002A600429002AB730200F7021705020A43021ED0
:1002B60055021E510205AB0205E802725E0202C635
:1002C60012DE1E75370790A051121C429002D6739B
:1002D6000202930208580208920208C60202FA02B3
:1002E600049A0202C60202C60203180202FF024A6A
:1002F600F6020326124833805A7F517E007472122A
:10030600D4CB121D9F40B9124D7812D98412BB046A
:1003160080AE7F49A25E120C1E925E120C3D80A03A
:100326007F64120D8B121D9F401DE5352480F475E8
:0C033600F0198460157F727E1F12D4BC89
:1003420012DD0D1001E810000280E30202C612BBAA
:10035200EA0202C6124E2C12DE1E75370290A22548
:10036200121C42900369730202C6020D95020DFA35
:10037200020E4E020EA3020EE7020EF60203CA029C
:1003820004000212B702038A7F5B120D8B120D6DFD
:10039200A8BE1203AE12DD0D1000081001071002F4
:1003A2000780EF18180880EA88BE80A85300037FF0
:1003B2005A7E0590A279E875F00BA42582F582E5B4
:1003C200F03583F58302760A7F40120D8B120D6D94
:1003D200E5BCF8E87F3F7E3212D3DE12DD0D10005D
:1003E2000810010D10021280EA18B84AE6787D80E2
:1003F200E208B87EDE784B80DA88BC02035612DE51
:10040200E37F0F90A5D41275F8121D5C12DD0DC2A8
:1004120014C21512DDEE7510651000DFE53170F9BA
:10042200E5106465700D855E14857A15E4F512F5A4
:1004320013800C78A8E51326F513E43512F5127F24
:100442001E7E19E51012D384C3E57A9515F517E5DA
:100452005E9514F5167F287E0BAC16AB1712D29858
:1004620012D31C12DD0D12DDFFD510ADAB17E51650
:10047200FC30E7031254FE7A0A79001252E4A91200
:10048200A81312541DEBF510243840037510C8123E
:100492000D4A8510BC02035612DEE3909C0A7F01CE
:0204A2007E09D1
:1004A40012760A909C137F0A7E0912760A7F131231
:1004B400C986751700120D59E5BC12057AE5BD12FF
:1004C400057AE5BE12057AE5BF12057A909C647F31
:1004D4005F7E0612760A121DE112DD0D75170012F9
:1004E400055A10000810011510024880F20517E59E
:1004F4001724F7500375170075100080E2E51764A0
:10050400087015120D5975BC0175BD2375BE45756E
:10051400BF67124E2C02049AE51012058C12DD0DF1
:1005240012053A0510531007E51724FE4003531033
:100534000380AC0202C6A9BCAABDABBEACBFE51722
:100544001304F8E640085407C42510C4800454700A
:100554002510F6027CA97800E875F009A42417FF99
:100564007E3B7D20E8651770027D89ED12D4CF08AB
:10057400B809E502DD0DF8C4120580E812058C7E89
:10058400030517E51702D4BC540775F009A4909C21
:100594001C2582F58250020583E51775F009A42411
:1005A40017FF7E0C02760AC26812DE1E75370590AC
:1005B4009DF4121C429005BD730202930278490215
:1005C400788E027A240205AB0205E102796602798B
:1005D400CC0216CE0205AB0216B4020B4F7F2E12CC
:1005E40015C980C312DE1E753706909ED1121C42B7
:1005F4009005F87302029302170B02176D0217E6B7
:100604000218B30218E502195C02063D020636021E
:1006140019A5021A4A02061C7F64120D54E5BDA2F4
:10062400E7120C1E120D54E5BD92E7F5BD124E2CD7
:1006340080B27F491215C980AB1207F9122AAC1295
:10064400DEE3121D36E558046077909FA11206E69A
:1006540012862912DD0D10000810011310021C80EF
:10066400F50559C3E558955950D575590080D015ED
:1006740059E55930E7C985585980C4E559B40F0282
:10068400802FB51F02802A75F007A42408F517757A
:10069400162774B82559F987001206D412DD0D10F7
:1006A400002810012810020280F574B82559F9A712
:1006B40000E53524FA508878C7A6481207F012DE00
:1006C400E312DD0D12DDF10205E81880CC0880C9C3
:1006D400E875F005A485F01CF51BC000125B84D0FE
:1006E40000221286BAB4FF0122751000751FFF1292
:1006F40086D1E510640F601712071D401274B825E7
:1007040010F8E675F005A485F01CF51B125C1505C0
:1007140010C3E558951050D72212109BF8602E6430
:1007240004602AE814B51025F51F120D68E5BC70A5
:10073400060475F014800375F019A485F01CF51BEC
:10074400125C157E2290A57512763DD322C322E554
:01075400584C
:10075500B4FF0122751000E510640F602EE51075D9
:10076500F007A42409FF74B82510F8E61207DA7516
:10077500F00A84C0F07E2012D4257E28742C12D471
:100785009DD0E07E2A12D48A12079A0510C3E55837
:10079500951050C32212109BF8603964046035E847
:1007A500146510702F120D68E5BC1207DAF8C31333
:1007B500923D7E1C12D43B7E28742C12D49DE430CD
:1007C5003D067405B80001147E2A12D48A7E187479
:1007D5002312D49D22305D1275F036A42432FBE439
:1007E50035F0FC12548D12548DEB2212080212754D
:1007F500DDDFFB22120802127DB9DFFB2275C7037C
:1008050075C6F078B87F042275C70375C6F375B948
:1008150001E5BFB54831E55924F1402BE55975F09F
:100825000484A9F024F0F5C675B901C5F0A9BC602A
:100835000CA9BD146007A9BE146002A9BFE975F033
:1008450005A4F985F0CC22120D68A9BD75CC00224E
:10085500124E2C12DE1E75370390A0BE121C42905C
:100865000868730202C6020B6802120C020B7D02B5
:100875000B880216290212D0020C49021304021336
:100885004A02167B02128602138F124E2C12DE1EAE
:0608950075370490A17A02
:10089B00121C429008A2730202C6020B97020BA213
:1008AB00020892020BB8020BC3020F10020892024D
:1008BB000BD2020BAD020BEC124E2C12DE1E753757
:1008CB000B90A1CB121C429008D6730202C6020FEA
:1008DB00BE020FBE02095C02099A0208FD02092042
:1008EB0002171102106302112B0210D40211BC0269
:1008FB000C06120D54E5BF1470C17F2E120D8B1F09
:10090B00120D54E5BDA2E6120C1E120D54E5BD925C
:10091B00E6F5BD80A37F37120D8B120D4FA8BFE8F4
:10092B0012095412DD0D10000810010D1002128077
:10093B00EE18B802EA780A80E608B80BE278038072
:10094B00DE120D4F88BF0208C37F367E2CE802D320
:10095B006D7F1C120D8B120D54A8BE12098E12DD69
:10096B000D10000810010D10021480EF18B800EBE9
:10097B00780B80E708E824F450E1780180DD88BE2D
:10098B000208C37F1B7E35E875F005A402D3677F91
:10099B0025120D8B120D54A8BF1209CC12DD0D10B0
:1009AB00000810010D10021480EF18B800EB780945
:1009BB0080E708E824F650E1780180DD88BF020863
:1009CB00C37F247E3BE802D4BC120D4AE5BF75F011
:1009DB003CA4ACF0FDE5BE75F005A42DFDE5F03CA7
:0D09EB00FC120D54E5BF14603675F005A434
:1009F80085BEF0A42DFFE5F03CFE7C007D3C125343
:100A080084C005EF75F01884E5F07F2D7E2412D39D
:100A1800677E30743A12D4CF7E35D0E012D36702A5
:100A2800DD0D7F2D7E0590A59712760A120D54E5EF
:100A3800BDA2E67F2D12155802DD0DD25712DEE356
:100A4800121D36120A510202937F177E02909D12E0
:100A580012760A7F4C7E02909D2812760AAC5DAB16
:100A68005C7F577E0412D314120D7785BC6285BD56
:100A780063E56124F84044909D337F371275F8AEE2
:100A880061AF607C017D5E125384C3741F9FFAAC12
:100A980063AB62EC33921750031254FE12526BABE5
:100AA800047C003017031254FE74F52BFB74033CCE
:100AB800FC1252417F377E1512D28C909D407F697F
:100AC8007E0F12760AE560240FFBE43561FCA25C18
:100AD800923BD25C7E1E12D298A23B925C7E30740E
:100AE8002012D4CF7E36742012D4CFE5602562FB65
:100AF800E5613563FC7F227E0412D314E562456309
:100B08007016742E7E3A12D4CF12DD0D10000D101F
:100B18000115100226020A79742080E81562E56240
:100B2800B4FF0C156380080562E56270020563E591
:050B38003524F5500317
:100B3D00753301020A79120D778562BC8563BD029A
:100B4D004E2C7F637E00747212D4CB121D9F400811
:100B5D007F631275EF124E330205AB120D5EE5BCCD
:100B6D00A2E77F0A120C21E5BC92E7F5BC020855FD
:100B7D007F1CA20D120C1E920D80097F25A20E1254
:100B8D000C1E920E120C3D0208587F0AA20F120C79
:100B9D001E920F802A7F13A208120C1E9208801F2E
:100BAD007F52A20C120C1E920C80147F25A20B12E8
:100BBD000C1E920B80097F2DA209120C1E92091298
:100BCD000C3D0208927F49120D54E5BDA2E3120CB3
:100BDD001E120D54E5BD92E39266F5BD02088F7F9E
:100BED005B120D54E5BDA2E5120C1E120D54E5BDB0
:100BFD0092E59243F5BD02088F7F6D120D54E5BD50
:100C0D00A2E0120C1E120D54E5BD92E0F5BD0208D6
:100C1D00C3120C338F1F9217120D8BAF1F1F7E390E
:100C2D00128313A21722120D6385BC2B85BD2122C1
:100C3D00120D63852BBC8521BD024E2C203714125D
:100C4D000D5E85BE12120C76120D5E8512BE124E11
:100C5D002C80057F3F120C680208587E0390A14539
:100C6D0012760A12DD0D02DDEE75A6FF12DEE3121D
:100C7D00B537740712DECF8FF0740612DECFEF2575
:100C8D0012C395F0A2E7923D4010FD24CD50027D98
:060C9D0032AC05C3743FF8
:100CA3009DFD800FF404FD24C850027D37AC05740C
:100CB300402DFD7F4012C9867E1212DE280EBE1E15
:100CC300F91F303D020F0FEF6D70EDE536700A75B9
:100CD3003606EC2513F5148C13120CF412DD0D10EB
:100CE3000007100108300207221512800205128046
:100CF300827F377E28742E12D4CF7F347E21740AEC
:100D0300303D010412D4EAE514FC249C50027C63B8
:100D13007F347E2DEC12CFA67F437E1E12D2947EAB
:100D230000E51212D42B7F057E0290A14E12760AA3
:100D33007F6D7E0190A15912763D7F747E0490A150
:100D43006A12763D021D3675C6F4803575C6F58088
:100D53003075C6F6802B75C6F7802675C6F88021D8
:100D630075C6F9801C75C6FA801775C6FB801275A7
:100D7300C6FC800D75C6FE800875C6FF800375C668
:100D8300FD75C70375B9012274721F12D4CB0F020C
:100D9300DD0D7F0A120D8B7E2A124833120D68A8CF
:100DA300BF120DC910001210010510021580F508BD
:100DB300E824E750EC781880E818E830E7E3780097
:100DC30080DF88BF805F7F097E0590A458B80C033D
:100DD30090A45212760A7E27E53D28240C75F0185C
:060DE30084E5F012D36765
:100DE9007E33743B12D4CF7E35E53E12D36702DDE4
:100DF9000D7F13120D8B120C33120E2B10000810DD
:100E0900010510021780F2105C07205D0BD25C808F
:100E1900E8105DE5D25D80E1D25C80DD852BBC0206
:100E29000356205C10205D1890A4AB7F127E23121C
:100E3900760A02DD0D90A4BF205DF090A4B280EB8C
:100E490090A4B880E67F1C120D8B120D63A8BF1207
:100E59000E8510000810011110021A80F2E824F220
:100E690050031880EA780D80E6E824E740030880FB
:100E7900DE781980DAE8F5BFF54380A37F1B7E266B
:100E8900E412D4BCE82323B464087E26740112D486
:100E9900BCE47E2E12D36702DD0D7F25120D8B1265
:100EA9000D72A8BCE8120EDE12DD0D10000810014B
:100EB9000D10021F80EEE824E050E9188006E824AE
:100EC900CF40E108120D7288BC124E2CD21512D9EE
:100ED9008480D180157F247E3724E202D3D87F2EE7
:100EE900A20A120C1E920A120C3D0203597F3712F4
:100EF9000D54E5BDA2E4120C1E120D54E5BD92E499
:100F09009267F5BD0203567F367E00747212D4CB08
:100F19000F7E16743F12D49D120D5EA8BD120F8963
:100F290012DD0D10000810010510021080EFE824F1
:070F3900875004240A800226
:100F400024E8F880E17F377E16742012D49D7E2C31
:100F5000743F12D49D120F8912DD0D10000810018C
:100F60001410022080EF18B80904787880E7B87868
:100F7000E478E780E008B87904780A80D8B8E8D542
:100F8000787980D188BD02088FE82487923DE850A7
:100F90000224917F367E30C313923B12D3D87E3C1D
:100FA000E4303B02740512D4B57E1A90A39E303D06
:100FB0000390A3A212760A7F3C7E3A02DE287F12BB
:100FC0007E00747212D4CB0F7E20743F12D49D1217
:100FD0000D4A85BE1085BF11121045100008100182
:100FE0001110021B80F21511E511B4FFEB751117FA
:100FF00080E60511E51124E850DE75110080D91254
:1010000010457F137E20742012D49D7E31743F12D0
:10101000D49D12DD0D10000810011110021B80DF9D
:101020001510E510B4FFD875100B80D30510E5102E
:1010300024F450CB75100080C6120D4A8511BF856F
:1010400010BE0208C37F127E24E51112D3677E30E2
:10105000743A12D4CF7E35E51075F005A412D3672B
:1010600002DD0D7F49120D8B12109BF81210A1109A
:10107000000810010D10021280F218B8FF02780467
:1010800080EA08B80502780080E2120D4A88BD1295
:101090004E2CB800030208C602112B120D4AE5BD02
:1010A000227F487E0590A3B812760AE8601CB4043B
:1010B0000A7E0590A3AD12760A800C90A3C4127626
:1010C0000A7E38E812D4BC02DD0D90A3BF7E29123F
:1010D000760A80F312109B601D640460197F5B1216
:1010E0000D8B120C33121106120D6310000B100140
:1010F0000810020C80EF0208C6105FE9D25F80E59D
:10110000852BBC0208C312109B601F6404601B7F08
:101110005A7E0590A3B812760A7E2390A3C8305F4A
:101120000390A3CF12760A12DD0D2212109B7003DA
:101130000208C67F527E11120D8B120D68A8BC12D8
:10114000116B120D6810000810010810020880EFE2
:101150001880EC0880E9120D6888BC124E2C120D24
:1011600072E875F005A4F5BD0208C312109B604B30
:10117000E875F03270040475F028A4ADF0FC305D21
:1011800011ACF0FB7A8A125279EB30E7050CBC0007
:10119000010DAE05AF047C007D64125384C005EFE1
:1011A0007F517E1A12D3847E2C742C12D4CFD0E0BF
:1011B0007E2F12D3671240FA12DD0D227F64120DCA
:1011C0008B120D68A8BD1211ED10000810010F1050
:1011D000021680F218E824CD50EC783280E808E856
:1011E00024CD50E2780080DE88BD0208C37F63E82A
:0611F00023C2E012CD391C
:1011F60075F06484C0F07E2612D4BC7E2C742C124A
:10120600D4CFD0E080A47F13120D8B120D5EE5BC07
:10121600A2E7923DC2E7F8E812125012DD0D100067
:101226000810010D10021280EE18B800EA7832801C
:10123600E608B833E2780180DEE8A23D92E7F5BC25
:1012460079A1F70213017F6380027F12547F305C1D
:1012560001237E2875F06484E5F075F00A84C0F0F9
:1012660012D4B57E2D742C12D4CFD0E07E2F12D49A
:10127600B50F7E3590A4C5305C0390A52102763D5E
:101286007F64120D8B120D6DA8BDE812124C12DD93
:101296000D10000810010D10021280EE18B8FFEABA
:1012A600780F80E608B810E2780080DE88BD020874
:1012B600557F52120D8B120D68E5BE7F517E2C12A2
:1012C6008368F5BE79A2F70203567F37120D8B129B
:1012D6000D63A8BC5300037F367E32E812D4BC12DD
:1012E600DD0D10000810010710020780E718180826
:1012F60080E2E5BC54FC48F5BCF52B0208557F4955
:10130600120D8B120D72A8BE12133B12DD0D1000CA
:101316000810011110021A80EFE8240AF82424505C
:10132600E778DB80E3E824F6F8247F40DB788180E9
:07133600D788BE80C6E8F471
:10133D0024DC75F00A847F487E3B02D4BC7F5212B8
:10134D000D8B120D72A8BF12138212DD0D10000845
:10135D0010011110021A80EFE82408F8245750E705
:10136D0078A880E3E824F8F824A040DB786080D7E3
:10137D0088BF021301E8F424A923C47F517E3B02E8
:10138D00D4BC122BB7754A00D210C211D214D2752B
:10139D0075791475340012DEE37F007E0290A1286A
:1013AD0012760A9041237F087E2612D4FBE52B543A
:1013BD00030F7E3912D4BC121D5112D165128DDC72
:1013CD0012DD0D10000810011A10022480C52075C1
:1013DD0004057980BE1579E579B4FF05C275757977
:1013ED000180B02075EB1579E57970A7D27580A3D2
:1013FD00C210C214020858120D63E5BE7F097E3A71
:10140D0002D4BC120D68A8BF120DC9120C33120EF6
:10141D002BA8BF120E85120D72E5BC120EDE7F2DAC
:10142D00A20A1215587F36A267121558120D6DE5D6
:10143D00BC7F3F7E3212D3DEA8BE1203AE120D4A20
:10144D00E5BC7F487E3212D3DE120D68E5BE7F51BA
:10145D007E2C02D4BC120C337F1BA20D1215587FAB
:10146D0024A20E121558120D5EE5BC1212507F0902
:10147D00E5BCA2E7121558A8BF121667120D6DE54F
:0F148D00BD12124CE52B54037F367E3212D4BCB5
:10149C00120D72A8BE12133BA8BF121382120D5468
:1014AC00A8BC0216AC120C337F09A20F1215587F80
:1014BC0012A208121558120D54E5BDA2E37F481272
:1014CC001558E5BDA2E57F5A1215587F51A20C1292
:1014DC0015587F24A20B1215587F2DA209121558EE
:1014EC00120D5EA8BD020F89120D4A85BE1085BF74
:1014FC0011121045120D54A8BE12098EA8BF120964
:10150C00CC1209D4120D63E5BE7F3F7E3A12D4BCD7
:10151C00120D4FA8BF120954120D4AA8BD1210A1EA
:10152C00120D68A8BC12116B120D63121106120D6C
:10153C0068A8BD1211ED120D54E5BDA2E07F6C80C0
:10154C000B7F098040120C337F48A25E744E400220
:10155C0074597E3A02D4CF127CB57F731279131270
:10156C007D047F6C1279227F2D801A120D54E5BDFB
:10157C00A2E77F63121558120D63E5BE7F097E3A10
:10158C0012D4BC7F481215B1B40104BF0901E4F5B3
:10159C001075F005A47E1E909EA22582F582500245
:1015AC00058302760A120D54E5BD035403C234C2FE
:1015BC005330E103D2342230E002D25322120D8B8D
:1015CC001F12159112DD0DE51010001210010610FE
:1015DC00020280ED22045403B4030AE4800714547D
:1015EC0003B403011423C5BD54F925BDF5BD124E3A
:0115FC002CC2
:1015FD0080CE1274D9EBF516F5147F6C1279221288
:10160D0074BD7F647E23E51612D43BC3E516951495
:10161D00F5167F731279137F2D0215917F2E120D02
:10162D008B120D5EA8BFE824FA4003303702780311
:10163D0012166712DD0D10000810010D1002128038
:10164D00E518B800E1780580DD08B806D978018085
:10165D00D5799DE8F7F5BF0208557F2D7E2C7420B6
:10166D00B80502742E12D4CF7E32E802D4BC7F5B53
:10167D00120D8B120D54A8BCE81216AC12DD0D1014
:10168D00000810010D10021280EE18B800EA780360
:10169D0080E608B804E2780180DE88BC0208557F38
:1016AD005A7E2CE802D4BCD26875480A124833D24F
:1016BD0014122ABA127DED123312C26B12024A8035
:1016CD00F3D214751501127C6F75B901E5BC20E7D5
:1016DD001C127D9F75A6FF127DF9121D5C12DD0D8A
:1016ED0012771310000F500512783B80E70515E5B2
:1016FD0015242050D10205AB1217170202931217B1
:10170D00170205E81217170208C6121723120D63E8
:10171D008548BE024E2C122AAC122AC612593E1210
:10172D00DEE3909F4AD24912865612860F121D0C87
:10173D0012DD0D10001410010510021B80F5054877
:10174D00E548640A7002F54880CF1548E54864FF06
:0A175D00700375480980C2854849F1
:10176700122AC6E55822124833122AAC854849C2C4
:1017770050E558B40F02D25012593E803AD227751D
:10178700480A122ABA12593E12DEE312857990A34B
:101797006F20290390A37A121DCEC26A123312104A
:1017A7006A0280E1C227127C47854948121B7912D9
:1017B7002AC6D22912593E12DEE3909E5D12865444
:1017C70020500E121DB812DD0D1000101001AE8052
:1017D700F8121D5C12DD0D10000280FB0205E812F5
:1017E7002AACE55830E7137F1B90A3597E05127684
:1017F7000A12DD0D12DDF10205E8122AC612593E62
:1018070085594912DEE3121D4690A37A12865412B7
:10181700861912DD0D10000810010A10020C80F560
:1018270012187E80DB12188B80D612DEE3121D465B
:10183700909F5912865412861912861D12DD0D10BB
:10184700000810010A10020C80F512189780DB12AD
:1018570018A580D6121B3F122AC612593E12DEE384
:1018670090A2C0128654121D8412DD0D10000510BF
:10187700028880F80205E80559C3E55895595003D1
:10188700755900221559E55964FF70038558592287
:101897000549D3E549149558400375490022154970
:1018A700E54964FF7005855849054922122AACE5C8
:1018B7005830E7057F240217F0122AC612593E1244
:1018C700DEE3909F64128654121DC312DD0D1000D3
:1018D7000A10010280F8121BE880DE0205E8122ACE
:0618E700ACE55830E705F6
:1018ED007F2D0217F0C26B7559FF12593E12DEE3C0
:1018FD00121D36E55930E703121D51909F76128661
:10190D005412862912DD0DE55820E7061000081047
:10191D00011110021B80F00559C3955950CF75590F
:10192D00FF80CA1559E55964FE70C285585980BDAE
:10193D00E55920E711D26B75A700758307C4F582B1
:10194D00E0B2E7F080A7306B03121B960205E81298
:10195D002AACE55830E7057F360217F0122AC61279
:10196D00593E12DEE3909F81128654121D9F40094D
:10197D00121BDD121C121219890205E8120D68E501
:10198D00BD75F00584F5BCF5BDF5BEF5BF120802B9
:10199D00124E2C05C6DFF922122AACE55820E708B5
:1019AD007F51909F8B0217F312DEE390A385128671
:1019BD0054121D5C12DD0D124792D2AC10001FE5C2
:1019CD005830E7F8306DF5121ADF7E207F00501386
:1019DD0090A3D612763D12DD0D12DDF180CAC2AC98
:1019ED000205E81B8B13909E7A12763D12DD0DC217
:1019FD006B7B007514B8121BD2127D6E127D2050B8
:101A0D0025A814E824384004A60105140BC3E513DA
:101A1D009B50E678B8121C14306B03127AC5122A4B
:101A2D00C612593E8082127CB5E51660E6D26B1265
:101A3D007DCBC003127C86D003A91580C4122AACBD
:101A4D00E55830E7057F5A0217F0122AC612593EA3
:101A5D0012DEE3909F96128654121D7912DD0D1041
:101A6D00003510010280F8754605121AA750157F32
:101A7D00007E357407954612D43B12DD0D12DDF153
:101A8D00D546E7D390A390500390A3D61286541257
:101A9D00DD0D12DDF180B30205E812479212DC274D
:101AAD00745212DC38745412DBF5E5580475590084
:101ABD0012DC161276C24016127C47127D9F1277E9
:101ACD0013400B0559C3E558955950ECC322C2ACD0
:101ADD00D322124792D2AC12DB80204CF1B440F7E6
:101AED0012DB85B4400312DB85B452E2F53812DB0C
:101AFD0085B454DA12DB85FA60D424EF40D012DBC2
:101B0D0085E53870C912DB8512DB851276A77B005F
:101B1D007E0312779E50102050B412DB85204C03AB
:101B2D00B440F7DEED80A7127D7E0B1276A7DAE0CA
:101B3D00C322121C23E55924C8F88602E54924C89E
:101B4D00F9986013146010500F18E608F618E8693C
:101B5D0070F7A702121C1222E559640F60F91908DB
:101B6D00E618F608E86970F7A70280E8121C2378DA
:101B7D00C8C250E6B4FF02800708B8D8F6D250228A
:101B8D00B8D702D250A615807C78B8121C25E4F97E
:021B9D00F5A7AA
:101B9F00758307E9C4F582E030E70AE924B8F82431
:101BAF0038400276FF09C3E5589950E7121BDD78DC
:101BBF00B879C8E6B4FF028002F70908E824385064
:101BCF00F2804079B877FF09E9243850F82279C8B4
:101BDF0077FF09E9242850F822121C23C23D78D739
:101BEF00B6FF04A900D23D18B8C7F5203D0279D839
:101BFF001978C8B6FF0122C3E8995007C6C7C608AF
:101C0F001980F478C8121C34127DDB127DDB127D33
:101C1F00DB027DDB78C8121C34127DB9127DB9123C
:101C2F007DB9027DB975C703E54875F004A424801A
:101C3F00F5C62212DEE3C23C1275FCE53760531481
:101C4F00604D14604514603D14603514602D1460B0
:101C5F002514600E14600B14600D14601414600CC6
:101C6F008030121551802B1215FF80261214F4802C
:101C7F002112154D801C12157780171215638012D3
:101C8F001214B1800D121462800812141080031206
:101C9F00140412DD0D12DDF5121D3612B8FAA81F4D
:101CAF0008E814C23BB51D02D23B75F007203C0378
:051CBF0075F009A4FF0F
:101CC4007E00303C0C7420303B02743E12D49D8064
:101CD4000A740B303B02740A12D4B5D8CF12DD0D4E
:101CE400E51D10000810011010021880B9651F705E
:101CF40003751DFF051D80AE7005851F1D80A7158A
:101D04001D80A375F003A4227F7B7E0090A2D812CD
:101D1400763DE54824F640087E0A90A33C12763DC1
:101D24002212793F7E05745B12D4997E1D745C0285
:101D3400D499121D257E3490A2E902763D12793F92
:101D44008003121D257E3190A2ED02763D121D25E1
:101D54007E3190A3E102763D12793F7E0080051228
:101D6400793F7E2D90A3E102763D121D797E31905C
:101D74009EB602763D121D5C7E1A909EBB02763D95
:101D8400121D5C80C0121D5C7E18909E6702763D19
:101D9400121D5C7E1A90A3E602763D121D5C7E1A2B
:101DA40090A3EB12763D12DD0DD3100006C3100193
:101DB4000280F622121D5C7E1A909F5402763D1218
:101DC4001D5C7E18909F6F02763D7F007E20127608
:101DD4003D02DD0D12793F90A3F102763B12793F6B
:101DE40090A40202763B12BE04120D81E5BDF55E9D
:101DF400F56CE5BCF55FF56B756A007561FF75A759
:101E04000490070012BDAEB4FC23E582C313F56150
:101E1400E56CF0E56BF0E582600F12BD25E56C65BD
:0D1E24005E70E1E56B655F70DB75A7002265
:101E31003024EA0460E7240F40D380E1E560758334
:101E410007C333F582E0A3F56CE0F56B756A0022F8
:101E5100D2248002C224D214C21F121DEA7560006E
:101E6100E561B4FF1612DEE3909D437F0A7E051201
:101E7100763D12DD0D12DDEE020293C210C2111287
:101E8100DEE3121D36301F0A7F07909D5112763B0B
:101E910080647F007E01C3E56012D43B7E0E74280E
:101EA10012D4998560487407F51FFF7E00743E12B5
:101EB100D49DE548121E3F12C79512241B0548C345
:101EC100E5619548FD401CE51F2407F51F24C85016
:101ED100E17F387E01ED0412D43B7E0E742912D4C9
:101EE10099800DE51F2407FF7E0190A3E012763D46
:101EF100201F0312245E12DD0D10001910012C1099
:101F0100020280F5120236301F3D020282101F02CA
:101F1100D21F021E7CE56160F4E5606561700520F9
:101F21001FF080E9201FE6056080E7E56160DEE5DE
:101F31006065617005201FD58009201FD5E560709F
:101F41000280CA156080CB121DEA121E3D12C79590
:101F5100122552756A1012BD97122609909D5BD207
:101F61003C1275FC121CA7901F6C73021E7C02327E
:101F710052021F8C021F78121D9F40CB121E3D1270
:0B1F8100BDAEC2E2FF12BBD4021E5531
:101F8C0012DEE37F6490A5BA1275F87F7990A5C72D
:101F9C001275F812DD0D75160010000A10010910EB
:101FAC00020280F505160516C253121E3D12C79586
:101FBC0075370A909D77121C42901FC973021F48F7
:101FCC00021FF00221BF0221C4021FB4021FF7023C
:101FDC001FFC021FB402203A02203E0220420220C3
:101FEC004902204D7F0A1215C980BD1247AB8003F0
:101FFC001247A0780A12211C740112DBF312215B28
:10200C0012DC0F12219612BD9712BDBF12BCE61244
:10201C00BED61222A5D5150C75150A1221A91223AC
:10202C00CC12DC0F100204E57F70DB021F48780A2B
:10203C0080067804800278011247AB8009780A8008
:10204C000278011247A012211C740112DBE8122144
:10205C005BE54812DBD4E5165403443012DBF5740F
:10206C002A12DBF512DBF512DC0F12219612BD974A
:10207C0012BDBF12BCE612BED61222A5D5154885DC
:10208C0048151221A9E51C12DBD4E51B12DBD4E5A3
:10209C001B2548F51BE4351CF51CE4A27792E7A23E
:1020AC007492E0A27392E112DBD4AD75AC74AB7395
:1020BC00E57DC41220DDAD78AC77AB76E57D1220E2
:1020CC00DD1223EA12DC0F100204E57F709F021F61
:1020DC0048540F2375F00584F8C3EB33FBEC33FC49
:0620EC00ED33FDC3EB33F0
:1020F200FBEC33FCED33FD20E713EB28FBE43CFC67
:10210200E43D12DBD4EC12DBD4EB02DBD4C3EB985C
:10211200FBEC9400FCED940080E88848121D63E417
:10212200F54AF549756A2075150112BD9712BCE68C
:10213200D5150E854815E5492401F549E4354AF5DA
:102142004AE57F70E5744012DC38747812DBF5746E
:102152006312DBF5742302DBE81223A7E56012DBCE
:10216200D4121E3D12C795E53A12DBE8E53B12DBBD
:10217200E8E53C12DBE8E53D12DBE8E53E12DBE890
:10218200E53F12DBE8740112DBD4E54A12DBD4E549
:102192004902DBD4121E3D756A20E4F51CF51BF5DD
:1021A20014F51375150122753800E51412DBD4E518
:1021B2001312DBD40513E51370020514221247AB88
:1021C2008003124795121D631222FF12DDF9756A10
:1021D2002075150175A6FF754A0112BD3F12BCE6B6
:1021E20012BED61222A5D5150975151E1222C912C4
:1021F200DE031223CCE57912DBD4E412DBD4E571E1
:1022020012228A12DBD4E57012DBD4E57B24ACFF08
:10221200E55F340912DBDAEF12DBD4E51520E03397
:10222200857D56E412DBD4E52EC412DBDA12DC1E05
:0E22320012DE0310021A30559B744012DBF5C9
:10224000744512DBF5744F12DBF5744612DBF512A0
:10225000DC1E021F48E556122264C4FAE57D1222F4
:10226000642A80C2FBC41222712323CB1222712B59
:1022700022540FFC24F650027C00902280EC932222
:1022800000000101010202030303FA2440400A2472
:10229000804003EA3322D2E72274FF2220E703C3FF
:1022A000132224C022E53F701F7F7B7E0078AEE6BC
:1022B00012D425EE2404FE743A12D49DEE2404FEBA
:1022C000E53E12D41F12DD0D22C015C016D2121227
:1022D000A612C212D016D01578AEE612DBE8E53EA3
:1022E00012DBE8E53F12DBE8E54512DBD4E55212EC
:1022F000DBD4740A12DBD474C012DBD402DC1E748B
:102300004012DBF5745412DC38744E12DBF5743075
:1023100012DBF5E5165403443012DBF51223A774E3
:102320002312DBE8E53D12DBE8E56012DBD4121E88
:102330003D12C79578ABE60812DBE8E60812DBE849
:10234000E60812DBE8E612DBE8E53E12DBE81229DC
:1023500032E51212DBE8E51112DBE8740112DBD47E
:1023600090A41312240C756A1012BD97057F057F87
:10237000787F12DBCD787B12DBCD787D12DBCD78D8
:042380007712DBCD28
:10238400E4FEFF780712DBCD12DBCDE57412DBD45B
:10239400E57512DBD4E412DBD4E412DBD412DBCD1A
:1023A40002DC1E75C70375C6FF75B901C217751D1A
:1023B4000085BC1C85BD1B85BE1A85BF191251F151
:1023C400EE12DBD4EF02DBD4E57512DBD4E5741234
:1023D400DBD4E57312DBD4E57812DBD4E57712DBCA
:1023E400D4E57612DBD4E51664016011E55E12DBF8
:1023F400D4E57A12DBD4E516640260012278BCE6E7
:1024040012DBD408E602DBD475A700E49370012242
:10241400A312DBF51A80F4AF1F7E0478ADE612D464
:102424001F7E0C742C12D49D7E0E18E612D41F7ECF
:102434001A78AEE612D41F7E22743B12D49D7E24F9
:10244400E53E12D41F7E2FE54012D4257E37743B1F
:1024540012D49D0E0EE54102D41F753200121E3DAA
:1024640012C795857946787A796412C7AE74641276
:1024740055E68E47122552756A20D23D12BD971239
:10248400BDBF122589303D09307406C23D8E1E8FB2
:102494001FE57F602BE54C24FFF54CE54D34FFF53B
:1024A4004D454C600512BCFB80D2751D3C12BD9796
:1024B40012BDBF12BCE6122589E57F6003D51DED70
:1024C4001225EA90260212D4FB203D0DAE1EAF1F4A
:0924D4001225EA9025FB12D4FB4D
:1024DD00E546FD700B90A549305D1190A545800C2A
:1024ED0004701090A545305D0390A5417F381240D2
:1024FD00F5804BE4FFFC7E05305D047E027FB31258
:10250D005377AC06AB071252417F38C23DE51C60D4
:10251D0007D23D7E2C12D48AE51B203D026007D2E6
:10252D003D7E3012D48AE51A203D026007D23D7EF1
:10253D003412D48AE5197E3812D48A1240FAE53263
:10254D0024C850FA22E54075F03CA42541FFF54C16
:10255D00E435F0FEF54D7C007D101253840F8F4B4A
:10256D00AF4CAE4D7C007D3C1252577C00AD4B12F2
:10257D005384EE4F70010F8F4C8E4D22786479731A
:10258D00C2D11225A0FF78677976D2D11225A0FE8F
:10259D0002DE28C3E796FB0809E796FC0809E796D3
:1025AD00FDA2E79217500312550675135A30D10E3E
:1025BD00751320B217AA4712528BAB04AC05E54632
:1025CD00600B04600BAA461252A2EB03FBEB03FB5C
:1025DD00EB543FFBE5132B2017029B9B22EE1414AB
:0825ED0030E701E4FEEF1414D5
:1025F50030E701E4FF2205057088A88870050520ED
:1026050020F8202075320012DEE37E1E7F1C12DECC
:1026150028DFFB12DE287E1E7F1C12DE28DEFB7EF5
:102625001D7F1D12DE28DEFB7F007E2178ADE612C0
:10263500D41F7E29742E12D49D7E2D18E612D41F28
:102645007E35742E12D49D7E3918E612D41F7F076D
:102655007E21745412D49D7E25744F12D49D7E2DF7
:1026650078AEE612D41F7E35743A12D49D7E39E5D4
:102675003E12D41F78AE1229327F0E7E21744C1281
:10268500D49D7E25744112D49D7E2DE51212D41F52
:102695007E35743A12D49D7E39E51112D41F7F150B
:1026A5007E25744412D49D7E2DE54012D4257E35B9
:1026B500743A12D49D7E39E54112D41F7F217E01E3
:1026C50090A51412763D7E0EAC77AB7612D2D17EF4
:1026D5002B85795F85787B12D8787F287E0190A538
:1026E5001812763D751D2B751E10E5741228E67EB1
:1026F50025742F12D49D751D2D751E2BE575122879
:10270500E67F367E0290A50412763DE57212279388
:1027150012282B121E3D756A209004E6E56CF09098
:1027250004E7E56BF0AE4DAF4C7C007D4012538461
:10273500BF00010F0FAC07AD07E4FED23D12BD97F8
:1027450012BDBF1227D4E57F602CE54C24FFF54C64
:02275500E54D50
:1027570034FFF54D454C600512BCFB80DE751D3C12
:102767000E12BD9712BDBF1227D9E57F600612BCB6
:10277700E6D51DED1227A97F7812C9987F767E00CE
:10278700743012D49DE53224C850FA227E2112CD2E
:102797003912D43B7E2F90A51C305D0390A52102F2
:1027A700763D9004E6E0FD9004E7E0FCC3E56A941B
:1027B70020FBE56B9CFCE56C9DFD50032410FD128E
:1027C70054769004E8EEF09004E9EFF022DD03ADD3
:1027D700040E7F78E55E20E72AE57A8549F0A4A90B
:1027E700F0E57A854AF0A429F9E435F0FAE55E8543
:1027F70049F0A429E435F02AFAE55E854AF0A42ACF
:10280700CF9FFF12DE28103D18C3EF9B50131BEF1D
:102817006B600E8F018B0712DE281FEF6970F8AF10
:1028270001AB072290A4C9305C0390A4E2754A402B
:10283700754900AF76E577FE20E76B7005EF24104A
:102847005064EF24A8EE34FD401190A4CE305C0311
:1028570090A4E6754A1975499A8075EF2450EE34AD
:10286700FB401190A4D3305C0390A4EB754A0C7520
:0528770049CD805CEF7B
:10287C0024A0EE34F6401190A4D6305C0390A4F062
:10288C00754A067549668043EF24F0EE34F1401327
:10289C0090A4D9305C0390A4F5754A047549448022
:1028AC002A8028EF2490EE34E8401190A4DC305CB0
:1028BC000390A4FA754A0275498F800F90A4DF30FB
:1028CC005C0390A4FF754A0175499A7F4012763BD0
:1028DC007F4612C9987F5F02C998AE1E75F06430AE
:1028EC005C0375F03284C0F0F87004EE2404FEE54D
:1028FC001D12D49DEE2404FEE8600712D48AEE2447
:10290C0004FED0E075F00A305C0375F00584A8F085
:10291C0012D48AEE2404FE742C12D49D0E0EE830D0
:10292C005C012302D48AE53E2541F51124C45003F1
:10293C00F511D3E63540F51224E85002F5122212B7
:10294C00B8F4C21012DEE37F057E09909B751276F7
:10295C000A7F137E0890297F12D4FB7F2B7E019077
:10296C0029E712D4FB20370A7F277E27902A591299
:10297C00D4FB22113007FE1FE001E101F80F000625
:10298C001B00F80C00180E007C10007006003C2098
:10299C0000E006003E4001E004001E8003C004007D
:1029AC001F0003C004000F00078000000F80078089
:1029BC00000017800F00000027C00F00000043C06C
:1029CC000F00100083E00F00200301F00700C00F80
:1029DC0001F80383007F87FE01FC000E3E18000007
:1029EC000300000000180000030000000038000085
:1029FC0000000000003000000000000000FC761F0A
:102A0C000E1C6030ECFCBC3F172DF0F97861386679
:102A1C00264F619A706070C60E1EE330E06060C68F
:102A2C000C1CC360C0E0618C0C18C7C0C0C0E18C2A
:102A3C001C39C611C0C4C19C9931963180C8C1FFE4
:102A4C001E31E7E180F0C0EE1C31C38180061630E8
:102A5C0091882892884924904927909248A0E3C8ED
:102A6C00BCC2AFD2C075C0107581D874FE122A8555
:102A7C00E4F5F9F5FBC2B480F7D2A6C2A512B8D919
:102A8C0012DDF502B8FA75C703E54875F004A42405
:102A9C0080F5C6C23C75B901E5BC047002D23C227B
:052AAC00120D63E5BE00
:102AB100F54824F65003754800753400753704C293
:102AC10028D229D22A75C703E54824E7500375485F
:102AD10000E54875F004A42480F5C675160775173E
:102AE10000C23C122B07122B07122B07122B078552
:102AF10017581558755900E548B40A09E558600595
:102B0100F46002055922203C1D75B90105C6AABC15
:102B1100ABBDACBEADBFEA122B28EB122B28EC12D9
:102B21002B28ED122B2822203C07F515B4FF03D2E8
:102B31003C22C0C7C0C6127C6F75A704851683E509
:102B410017C4F8F58275B90105C6E5BCF0C582F870
:102B51002406F92403C582E5BDF0E5BEF0E5BFF02A
:102B610075B90105C6E5BCF0E5BDF0E5BFF0851618
:102B7100838982E4F075B90105C685BC1385BD144E
:102B8100E4F0F08882E5BEF0E5BFF075B901E5BC7F
:102B9100F0E5BDF0E5BEF0E5BFF0758306E517236E
:102BA100541E24B0F582E513F0E514F075A700D0AA
:102BB100C6D0C705172212BB0478BEA64808E4F6A2
:102BC100F55908761808F6D23608760A08F6060886
:022BD10076BECE
:102BD300C254C25512BE19122ABAC229C22AC20746
:102BE300C227C268120D54E5BDA2E59243C24AE46E
:102BF300F52EF534F536F52F78B6F678B5F678A9CF
:102C0300F6789EF678B8A65E08A67A12D23AC26B18
:102C1300C233C238C240C223C222122C37754602C5
:102C230078C5A646C23AD221C219C226E4F542F5B6
:102C330041F54022E45407205E09B40400400274C5
:102C430003801B120D59C313A9BC600C14A9BD60EA
:102C53000714A9BE6002A9BFE94001C45407F537B0
:102C630022122AAC12593E1207F912DEE3121D8416
:102C7300E55804700A7F327E0590A35912760A90B4
:102C8300A5B11286561207537F7290A5A61275F846
:102C930012DD0D10000510020480F8D322C32202B6
:102CA30000F7120D54E5BD20E705122C6440F075C2
:102CB3004E50122BB712843475440312483012AEAF
:102CC30037D54403022A6D201EF1789F7680754A1A
:102CD3000012BC35D210C211C213C2121247827540
:102CE300A60C12D98412C41AE5A624FA4006124788
:102CF300D075A60C20250CE59054057009E5352404
:102D0300E25003022D97E5322418400D75F00C8430
:072D1300E5F070D412331546
:102D1A0080CFD21ED2AC306DC87532F012DB8AB4C5
:102D2A00E0BF124878E53124F392052012031231EC
:102D3A00A7122D5DC014128D22D014200A03122E60
:102D4A008012331512A5E112331512843712331586
:102D5A00022CDF30122EE54024F0401C7A0AC3E52B
:102D6A003F954B6013401E24E2400D305405C25477
:102D7A00757F0112BC5BDAE679BCE7D2E7F57F0919
:102D8A00877EC27722F40424E250ED80DE12DEE36D
:102D9A007F2A7E0E90A41712760A75A6FFC210101B
:102DAA0012137F367E08909E9812760A12DD0D1253
:102DBA00DDEE0200F7D22112485412BC657F1E7E56
:102DCA000B90A33212760A12DD0D122DEA7F3E7E97
:102DDA000790A02E12760A12DD0D12DDE8022A6D86
:102DEA00D215D21412BDF0120C3375B90575B90299
:102DFA0012BDFAD25512BD1F7F0012BBD412BDFA02
:102E0A00E56A600512BCE680F7857A62120D818553
:102E1A00BEBC85BFBD856BBE856CBF75B90575B96E
:102E2A000285BD6C85BC6B756A2012BDF01230211B
:102E3A0012BDFA756A0012BD97E57064FE703475AA
:102E4A0070FC854077854178851F797818797A12E0
:102E5A00C7AE12BC9412DE0312BDFA756A1012BD17
:102E6A00977F087810797212C7B085627C855E7D7B
:102E7A0012BC94C215221247AB122FCD745212DB28
:0B2E8A00F5744D12DBF5744312DBF50C
:102E9500122FDC12DC307441207402745612DBF5FB
:102EA500122F29122F7312DC30E53C12DBE8E53BCB
:102EB50012DBE8E53A12DBE8122FA912DC30744583
:102EC50012DBF5123012122FCD744712DBF5744761
:102ED50012DBF5744112DBF5122FDC122F2912DCFF
:102EE50030E43074010412DBF312DC309004C3E0EB
:102EF50012DBE812DC309004E4E075F00A84AFF0F0
:102F050012DBE812DC34EF12DBF3AC5EAB7A122F86
:102F1500EEAC5DAB5C122FEE12DC3012DC30123001
:102F2500120247827875C23D122F347878D23D124D
:102F3500DC30128119303D05E51E12DBF3E51D126B
:102F4500DBF3122FB6E51812DBF3E57D203D01C456
:102F5500540F12DBF312DC30303D09744530170293
:102F650074578007744E301702745302DBF52074D2
:102F750008122FA9122FA9802775A7049004BFE076
:102F8500FCE0FB7A1B125279783212541B12524123
:102F9500122FB39004C1E0FCE0FB125241122FB393
:102FA50075A7002212DC30E4F51AF519800D12DC44
:102FB50030E51C12DBF3E51B12DBF3E51A12DBF33C
:102FC50012DC34E51902DBF3742412DBF5744712C5
:102FD500DC38745002DBF512DC30E53D12DBE8E548
:102FE5003E12DBE8E53F02DBE812817512DC30E5D5
:0E2FF5001D12DBF5781CE612DBF318B817F896
:1030030012DC34E412DBF312DC30744D02DBF5C066
:1030130038742A12DBF5D03812DC0F02DE03781085
:103023007F0EE4F608DFFCF564F565F567F5687572
:1030330015FC751AC0751DC0756640756940754AE3
:103043000112BD3F3055030230D712BCE6E571B51E
:1030530010004002F510E4F511E512207502E513A6
:10306300C395795006207545857913D3E57A951470
:10307300E5156480FFE55E64809F400C857A1485C6
:103083005E15857B16855F173074B3C2D17864797A
:10309300731230B5786779761230B5D2D178187952
:1030A300731230B5781B79761230B5809185791219
:1030B30080B9D3E7960809E7960809E66480FFE735
:1030C30064809F20D101B3400AE7F61819E7F61888
:1030D30019E7F622E51AB4C00E7873791812C7AE51
:1030E3007873796412C7AE78187964C2D112314803
:1030F30074181255E68E47AE1EAF1F781B7967D240
:10310300D1123148C3E51F9FE51E9E50048E1E8FCA
:103113001F7EFF7FFFAC1EAD1F1253847A04EF8A1C
:09312300F0A4E5F0CE8AF0A42E20
:10312C00FEE435F0BEFF011E60051460057EFF8EC7
:10313C001F22EE7E0020E7F77EFE80F3C3E697FBAE
:10314C000809E697FC0809E697FD1818191930E7E5
:10315C0003125506C3EB33FBEC33FCED33FDEB33C1
:10316C00EC33FBED33FC30D105AA471252A20BBB5A
:10317C0000010C751E03751FFFEC24FC40048C1E13
:10318C008B1FE627FB0809E637FC0809E637A2E7A0
:10319C0013F618EC13F618EB13F62210131978B576
:1031AC00E624FA401AE57124F64008E57924F64045
:1031BC000280360606803212DDFFE59030E2DF75C4
:1031CC003612D22EE4F534F55A12BE4B1231F8C237
:1031DC0019C257122C3712905112907ED212853F81
:1031EC004B754C00205E02D228022C2FD2141232C6
:1031FC0047E6F008DFFB857A6212323D7570FE7887
:10320C003A797112C7AE12BC9412323D85627A853E
:10321C005E7B120D7785BC7E85BD7F7570C012BC40
:05322C0094123247E09E
:10323100F608DFFB75A700D254C2142274FF787020
:10324100F608B880FB2275A7049004F078707F100F
:1032510022121E3D122BB712DEE312DD0DC258C23F
:1032610059754A01753901756A2012BD3F1255E43D
:103271008E47C210D211D214D21212BE4B129051EB
:1032810012907E12D98475A6FF753609753200E554
:103291009020E206E5352405400CE5905405701FA9
:1032A100E53524E25019C211C21212DEE312DD0D1E
:1032B100E4F535F52F7E0612DDFBC202021F48C27E
:1032C10021E54AB40202D22112BD3F12A5E1302606
:1032D1000F1259A0128437753606E53670FCC226E6
:1032E100128434123315E54A20E021B402097539FC
:1032F10000E53670F9808CE53960FAFD24E2400280
:10330100053912BD3F2026C9DDF880E975390080F5
:10331100E475370410003A100116100216E52F5417
:1033210007600312B8EE20783D20790A207A1F2227
:1033310002350B02345FE537600914600914600936
:103341000235B702352A023588C2790235D40234F2
:1033510092E53724FC500FE5376407600302364FCE
:103361000236130234292011FAE59020E202805638
:10337100753400201203D2132278A9E67017C226F1
:0D338100767DE5377005106B02D26BD277B8
:10338E00753614D22E02BE40E5376043146040B449
:10339E000227200B24E6249B401F2414501C12905D
:1033AE005190A3047F207E0812760A12DD0D753629
:1033BE0008D22E78A9E624ECF622241940FB241418
:1033CE0050F712905112907E90A30D7F2980D72036
:1033DE0028E7E54824F640E1E5580460DC7F5D7E91
:1033EE0010E6249B40D324145015C2330559C3E56F
:1033FE005895595005855859D22690A2F280A92485
:10340E001940B6241450B2E559600215591026061B
:10341E00E5596002155990A2FB808D107801227536
:10342E003900E53424384007754A0175340022709E
:10343E000AE54A30E0F2754A0280F0146008754AD7
:10344E000612907E8006754A0412905175390180DD
:10345E00DA302909C229D22A7559008005302A1B73
:10346E00D2291286051285D3E53524AF4004753472
:10347E000022753700C229C22A80F3206841302706
:10348E0003D26A22D2221237EB12DD0D107A0122FC
:10349E00E53424384007122C3775340022700FAAF9
:1034AE0037122C376A70F27401122C3880EB04122A
:1034BE002C3824FC50E3E537B40706D22880DA8096
:0834CE0036C228E53724FC2377
:1034D60024BEF879C4E7F9A74809A75979C4E8F7DB
:1034E6008648088607E537B40505754818D23612AA
:1034F6002AC68F59E53764067002D2070234A7122E
:1035060037C7023771E537601B14607614600F14F5
:103516006009E53724F940090236C90235B7023693
:1035260002023696D223123FD910790122E53424BD
:103536003840077546017534002278D87020304A25
:103546000BC24AE624F85004B243800AD24A7614E3
:10355600E54624FE40DDE54660D9154680D8B6002E
:10356600D5B40500500C04F54624FA50C975460535
:1035760080C424F95005127A6380BB100FB8D20FAD
:1035860080B4D223E53464C86003123FD9107901B0
:1035960022E534243750097011105B32D25B802E3D
:1035A600100802D208123FD98024100C21D20C80B8
:1035B6001DD223123FD910790122D24BE53424378C
:1035C6004010C258C259201105D22E7536077534DF
:1035D600002224FD401524037006D258C25980EEFD
:1035E600C258D2591460E7D25880E3120D5EE5BC8A
:1035F600B2E7F5BC79A1F7124E2C80D278B8A65E58
:0B36060008A67A2011C8753605D22EE8
:1036110080C130122B12863F055BE55B75F00B8490
:10362100E5F0F55BE55A24F64009E55A955B500350
:10363100755B0012864312DD0DE5346003D534D28B
:1036410075340022D229D22A75480A023737C2407E
:103651001007F1302903023737128601128615103F
:103661002A1BC2330559C3E558955920E702500872
:10367100755900E548B41816E558B4FF03755900AB
:1036810012862912DD0DE5346003D534C122D22A18
:1036910012860580EE30122312863F155BE55B3002
:1036A100E70C755B0AE55A24F64003855A5B1286DE
:1036B1004312DD0DE5346003D534DA75340022D2CE
:1036C10029D22A754817804CC2401007F22029449C
:1036D100128601128615102A22C2331559E5593076
:1036E100E71C855859E558B4FF03755900E548B4FE
:1036F1001802800AD22A128605800E855859E5588B
:10370100B4FF0375590012862912DD0DE5346003FB
:10371100D534B52220106220115F7F180548E54895
:1037210064187008F54830270375480A122A923048
:103731003C2DDFE8802620105A2011577F181548AC
:10374100E54830E705754817800A64097006302797
:1037510003754817122A92303C05DFE275480A12B8
:103761002AC612593EE532244C50051285D38003F6
:1037710012857975340002DD0D1237AE7F15E548EB
:103781006B70048A4880020548122A92303CD0DFCF
:10379100ED80CC1237AE7F15E5486A70048B488006
:1037A100021548122A92303CB6DFED80B27A007BD6
:1037B10009E537B40401227A0A7B17B406012274A1
:1037C10018FAFBF5482275A704758307E559C4F576
:1037D10082E0E0F573E0F574E0F575E0F576E0F58B
:1037E10077E0F57875A70002593EE59020E23EE5C5
:1037F100342437503812382F12380C205E4F7F2C6A
:10380100909C2E123876909C37806AE53424377567
:10381100F009A42435FF205E0624BE50027F3EEF4E
:10382100249B50027F627E32748912D4CF2275A705
:10383100049000317E087F3AE4F0DFFDE582244602
:10384100F582E43583F583DEED75A700227F2C1226
:103851000D59E5BD12385FE5BE12385FE5BFF8C40A
:10386100123865E8540775F009A4909C1C2582F56F
:0C3871008250020583EF2409FF0275F865
:108431000284EE12DEE3E53724FC40F4B4FE14209E
:10844100110EE590F45407600122E532247450EFD7
:10845100028D2E12DEE312D67212D70412CD47120C
:10846100D29012D0D97E197F3612CE8112DC3D1204
:10847100CE97C206E53760051460338053C23A12C5
:10848100859212409C1242311245171263FC12640C
:1084910024123D47E54864186009E54824F6500375
:1084A100124602128CC412CF6C1241378014D23A98
:1084B1001285B812388512410612C8FE128CC412F8
:1084C100CF2D125C7F12D74B125750125A4F801288
:1084D10012859E12C83B12D81B12C8CD128CC41231
:1084E100CF4430101412CE0A12CDD9800C12DEE323
:1084F100E53724F9401E12857B3022091237EBE55E
:10850100347002C222302309123FD9E5347002C20D
:108511002302DD0D121D3675170012DA2E7F12129D
:10852100C98630124A75100075A704758306125961
:10853100F9E51075F009A42415FFF5177E00E51281
:10854100602F75F06484E5F00F12D41F1F7E0EE5D5
:108551001112CD8F751623125BB50510C3E55A951F
:10856100104006E51024F550BF30120312864380F7
:1085710088745D12D4CF80D5C249302905121D0CF3
:108581008003121D36909E5D128656202A76028641
:1085910029301223305E2030501D02893A301217E3
:0385A100305E0643
:1085A400200B11028F9B12C97F7F1712DD83751771
:1085B4002002DA2E12D5E912D58A30121120510583
:1085C40012D649800612CCD312CAB31250B322E495
:1085D400FEFFE54824F6400D90A33C12763D7E163E
:1085E400E54802D48AB40E0690A34202763D90A3D5
:1085F4004912763D7E12E54824F702D4257D208079
:108604000C7D3F302A077D633029027D3C7F00804A
:10861400247D2080127D3E800E7D3CE54975F00767
:10862400A42406800A7D3FE55975F007A42409FFB8
:1086340064027001FF7E1CED02D49D7D2080027DCA
:108644003FE55B75F009A42416FF7E09ED02D49D75
:10865400C2491286BAB4FF01227510001286D1797C
:1086640020E030E702792F30491712109BFAB40446
:1086740008E510700C79658008EA146510700279B9
:1086840023E97E1812D49D7E20E51230E708909EDF
:108694009812763D8016E511128747125C1520105A
:1086A4000520110280063012031286F90510C3E575
:1086B40058951050A7227E207F0012763D1285D354
:1086C4007E007F0690877912D4FBE5582275A704B3
:1086D4007583071259F9E51075F007A42409FFF50D
:0D86E400177E00E51212D49D7805EE2404E7
:1086F100FEE012D49DD8F622128801128817FD7C63
:1087010000AE1CAF1B125377BE003A8F00C3E57A4F
:108711009513FFE55E9514FE402B7C007D281253D6
:1087210084C3EF98401F75F0058404FB24F95002BF
:108731007B067E2CAF170F12DE280F12DE280F12D8
:10874100DE280EDBEF2264B4602464B475F0328459
:10875100C0F012D48ACE2404CED0E075F00584C0D6
:10876100F012D48ACE2404CED0E02302D48A90879A
:108771007502763D2D2D2D000140FFFFFFE0FFFF2B
:10878100FFFFC25030123F20283CE558F4603720EB
:108791004803200931D250E559F5103033066558A8
:1087A100600205101287CB12882775A7049006DC9A
:1087B100E512F0E511F0E517F0E510F075A704906A
:1087C10006E0ECF0EBF075A7002275A704758307AE
:1087D1001259F97813E0F608B819FA9006D0781111
:1087E100E6F008B819FAE51CF516F0E51BF515F0E9
:1087F1001288019006DAE514F0E513F075A700225E
:1088010075A704758306E51023541E24B0F582E094
:10881100F513E0F51422120D5EE5BD2487E5BD9246
:018821003B1B
:10882200500224912212881775F005A485F012F5E2
:1088320011E4F519FEF51CF51D12BDF0C23DC2563C
:108842007F3C12CA29303D05751900807DDFF3E5B2
:10885200596558700A301007EE24D35002D2568C54
:108862001B8D1AE519FD24E250DEAE1CAF1D7C0003
:10887200125377EFF51924F650CEAC1BAD1A12C97C
:108882006E20D1108E048F05E51975F0A7A4AEF005
:10889200FF125377AC12AB117AA01252A2EB33FB48
:1088A200EC33FC20D11AEF9BEE9C5014C3E512135B
:1088B200FCE51113FBC3EF9BEE9C4004AC06AB0737
:1088C200204807203B048C128B119006E2E519F038
:1088D20012890FAC16AB157AC8125279A912A811D7
:1088E20012541DED7005EC249E50057C807B0822FD
:1088F200C3E57A305602E55C9513FFE55E30560219
:10890200E55D9514FEC3EF9BFBEE9CFC22AE16AF19
:10891200157C00E519FD24F6501A1253777C007D70
:10892200061252577C007D051253778F10EEF51711
:0889320024E950037517FF2230
:10893A0012C97F12895712899A12D23F1289C0200E
:10894A004809128AAE128ADE028B4180747F177E32
:10895A002020480E748A204D101257BD500E742FD5
:10896A008007746A305F02746712D4CF75A70490C7
:10897A0006D07811E0F608B819FA7F177E00781247
:10898A00751905E60812D4CFEE2406FED519F4228D
:10899A0075A7049006D8E0F516E0F515E0F514E0A1
:1089AA00F513E0F512E0F511E0F517E0F510E0FC3B
:1089BA00E0FB75A700227F187E26AC14AB1302D207
:1089CA00D19006E4E0F51CA3E0F51B7F2A304E1394
:1089DA00120D54E5BF90A3A6B4010390A5A0127589
:1089EA00F880420F7E00745312D49D9005CBE0F8B4
:1089FA0030E705E53F30E0091F7E00E8540F12D446
:108A0A00B59004EEE0FEF51EA3E0FFF51F128A56AC
:108A1A00E51E24E9500C7E06742B12D4CF7E0C126C
:108A2A00D4CF128A86C20375172A751627125B8459
:108A3A00202415205F15D2037F2A7E1E908A743067
:108A4A004E03908A7D02D4FB205FEB227C007D3CA2
:108A5A00125384A805EF7F2A7E0812D3D87E127497
:108A6A003B12D4CB7E14E802D3D20707384C9EBA05
:108A7A00F264380707387CE6C2E67C38AC1CAB1BCC
:108A8A007A48305D027A27125279A91EA81F125419
:108A9A001DED4C60027BFF7F207E28EB12D3DE7E29
:108AAA003902902E7F2B90A34F12763BE517F46084
:108ABA0022AE17AF107C007D3C125384A805EF7FCD
:108ACA002A7E0C12D3D87E16743B12D4CB7E18E8B9
:108ADA0012D3D222AE12AF117C007D0A125384A89F
:108AEA0005EF7F207E3012D3D87E3A742C12D4CF71
:108AFA007E3CE812D4B50F7E29744502D49D748554
:108B0A008007748720560274867E2912D4CF3017C4
:108B1A0007742D7E3A12D4CF227C007D0A12538428
:108B2A00A805EF7F2A7E3012D3D87E3A742C12D44D
:108B3A00CF7E3CE802D4B5128C72E54824F6500583
:108B4A00128B2380B9E559046558600D128B2312E4
:108B5A008B08E559655860AA22A217923D8E1E8F8E
:108B6A00188515179006D0E0F511855810151012C2
:108B7A0044F7C3E51195105002F404F924A65005F0
:108B8A00C374B399F9E975F00584F924EE500279B2
:108B9A0011908CB2E993F5F012080DE5CC7004E956
:108BAA0030E702747F23A4A9F0E51B2517FDE51C15
:108BBA003516FEC3ED99F515EE9400F51675A70066
:108BCA00758306E55823541E24B0F582E0A3F513F5
:108BDA00E0F514128C72203D2C201729120D5EE547
:108BEA00BD2487E5BD5002249175F007A4FB9518B2
:108BFA00E5F0951E400FEB9FE5F09E4008EF9518B3
:108C0A00EE951E500EA23D9217AE1EAF18128B2380
:108C1A00028B08306B10128C0FE53F20E007748638
:108C2A007E2212D4CF2275A7009006E0E516F0A3A3
:108C3A00E515F0128B23128B0C74857E2312D4CF88
:108C4A008558101287CB12895712899A8C168B1560
:108C5A001289C01288D51287BD12D23F9006E2E06F
:108C6A00F51912890F028AAEC3E57A305602E55C1D
:108C7A009513FFE55E305602E55D9514FE92175096
:108C8A00031254EEAC16AB157AC8125279A906A88B
:108C9A000712541D7E037FE7ED700CEB2418EC34A9
:108CAA00FC4004AE04AF032200172E43576C809297
:108CBA00A4B6C5D3DFE6EDF3F8FD305E4F30504C75
:108CCA0075A7009006E0E0A3FCE0FBECA2E7921790
:108CDA00402024FE50047F3B8022AE04AF037C0078
:108CEA007D1412538474542F2017029F9FFF7462BD
:108CFA00800C1254FEEC24FE50E07F6D743D7E0021
:108D0A0012D49D7E017D197C03128D17227F3D129C
:108D1A00DE28EF2DFFDCF822E537B40206E534241D
:108D2A003750292212DEE312D67212CD47128EAEC6
:108D3A0012C7C912CF54128F06125A4F7F207E2BA8
:108D4A0012CE8112D70412DC3D1237EB12D1651212
:108D5A008DDC12504D02DD0D20041EE579FD24A0A4
:108D6A0050027D5FED24CD401E744520750C2DFF09
:108D7A00F512128DB11FBF44F922C39DFFF51212DD
:108D8A008DB10FBF46F92220750EED2413FFF5129F
:108D9A00128DB10FBF78F922C374779DFFF51212B5
:108DAA008DB11FBF12F922EF24BA40082433FCC345
:108DBA0074329C1404FC24D750047C238009EC23CD
:108DCA0075F005842413FC7E0512DE280EECB50628
:108DDA00F822E59020E206E53424374003128D623A
:108DEA007F457E047D1212DE280EDDFA7F437E0067
:108DFA00746412D49D7F4F7D12128E977F3B7D1231
:108E0A00128E977F597D16128E977F317D16128E9C
:0F8E1A00977F637D1A128E977F277D1A128E978E
:108E29007F6D7D1E128E977F1D7D1E128E977E058A
:108E39007F1912DE280FBF72F97804E57924CD5025
:108E4900027809E8305C0123F87F1B128E867F6B5C
:108E5900128E8618305C01187F25128E867F61126A
:108E69008E8618305C01187F2F128E867F57128EDE
:108E79008618305C01187F39128E867F4D7E00E896
:108E890075F00A847004E802D48AE802D425EF65F3
:108E990012600C7E04EE20E00712DE280EDDF622B9
:108EA90012DE5880F790A4667F287E2C12763D7ECC
:108EB9003B12D2E8AC5EAB7A7F307E19C23D12D349
:108EC9002790A3537F5D7E2D12763D78B9C3E57A4D
:108ED9009618FBE55E96FC7F507E19D23D02D3279A
:108EE900E51164B4700122E51112DCAD7831790F16
:108EF9007D0B12DDAB1F1E908F9602D4FBE57160CE
:108F090012E57012DCAD7831790F7D0412DDA70D01
:108F1900BD0AF97F01128F6E7F1D128F6E7E23129B
:108F29008F787E3F128F787E247F17128F827E3949
:108F39007F02128F827E247F07128F8C7E397F1CDD
:108F4900128F8C7E317F0212DE287F1C12DE287F71
:0F8F59000F7E2412DE287E3E12DE287F0C7E2E35
:108F680090D7F002D4FB7E2A12DE280EBE39F922F1
:108F78007F0812DE280FBF17F9227D0612DE280EA1
:108F88000FDDF9227D0612DE280E1FDDF92203030C
:108F9800E0A0E012C97F7F18909C6D12763B7F217C
:108FA8007E01744112D49D7F2A7E01745312D49D90
:108FB8009005BEE0F51AA3E0F519A3E0F51EA3E0BD
:108FC800F51D851A1C85191B75172012904BE5197C
:108FD800251DF51BF51DE51A351EF51CF51E751723
:108FE8002912904B9005BA12903BAC1AAB19751721
:108FF800201290099005BC12903BAC1EAB1D751752
:1090080029EC7006EB24CD4001227A48305D027AC3
:109018002712527912541DED4C600122AF177E07BA
:10902800EB12D3847E1A0F90A529305D0390A52CEE
:1090380002763DE0FEA3E0FD12BF46C3EB9DF8ECCF
:109048009EF922751627025BB512BF4675A70490D4
:1090580005B478737F06E6F008DFFBECF0EBF0E090
:10906800E0E0FCE0FDE0FEE0FFEF2DFFEE3C9005C8
:0D907800C0F0EFF0801275A7049005BAE07B
:10908500FBE0CBF0EBF0E0E0E4F0F075A700227533
:10909500A7049005B478647F06E0F608DFFB75A7A2
:0F90A50000125DC49005BEE51CF0A3E51BF02290
:10387D00D23C799E77008002C23C12BDF0E4F51077
:10388D00F511F512F513F514F515F516F517C23DED
:10389D00123BCD203D1F123BCD203D19E51F30E5DC
:1038AD001130E40E1238F4303C08799EE724F550BF
:1038BD000122D510DBAE14AF157C00AD12125351A1
:1038CD008F55AE16AF177C00AD1312537712557886
:1038DD007E00E55530E7011E2DFFE43E30E7027F07
:1038ED0000740A2FF55622C235E51CAF1DBFFF052A
:1038FD000FD235F404FABF003F532CF8E518AF1979
:10390D00BFFF050FD262F404BF002D20E72A205B14
:10391D000123FF24AA4021E51AAE1BBEFF050ED2DE
:10392D0061F404BE00128547F0A4E5F020E70920FC
:10393D005B0123FE24AA5001227C807B80305166DE
:10394D00302163C006C0078AF0E545A4AEF0FFE55F
:10395D0056205B011375F009A4ACF0FD125377747A
:10396D00FFBE0001EFFA24C050027A3FD007D00607
:10397D00E55212DCAD303504B2D5B2D1EA8CF0A4EB
:10398D0030E70205F0748025F020D10495F095F014
:0A399D00FCEA8BF0A430E70205F00D
:1039A700748025F030D50495F095F0FBC3EC2F20FB
:1039B7006203C39F9FFFEB2E306103C39E9EFE20D1
:1039C7003C64200C05123A614064123A43405F128E
:1039D700DE28E51EFD24FB50550E12DE28ED24F6E9
:1039E700504C1E1F12DE28ED24F150421E0F12DE2E
:1039F70028ED24EC50380F12DE28ED24E7502F1F56
:103A07001F0E0E12DE28ED24E250231E0F0F12DECA
:103A170028ED24DD50180E12DE28ED24D8500F1E95
:103A27001E1F1F02DE28123A434003799E0722E930
:103A3700242AFFE82461FE123A61401DEF2460400A
:103A470018243F5013EE2460400F243F500AEF2400
:103A5700D6FFEE249FFEC322D322532CF8432C0417
:103A6700EE10E706D2E7F404D261FE24D340EAEF72
:103A770010E706D2E7F404C262FF24D340DBEFB5B8
:103A870006005003CED26070057480FE8062FF246A
:0D3A9700FD5060903B4D938EF0A4AAF033DB
:103AA400CA33CA33CA33CA33CA33FA903B77938FC3
:103AB400F0A433C5F033CA903B9893FB123B1595A1
:103AC40070500224B412DCADEA8BF0A430E7020596
:103AD400F0C3748095F020D50425F025F0FEEA8C1F
:103AE400F0A430E70205F0C3748095F030D10425CA
:103AF400F025F0FFC3227A01EE6F70097B16BF0236
:103B0400BB7A0380B7BF01047B0080B07B0D0A80C1
:103B1400ABE52C540723C3903B1F73800E800E80AB
:103B240024801E8010800A80108012EB22742D9B4A
:103B340022742D2B22745A9B22745A2B2274879B35
:103B44002274872B2274B39B22FFFFCCAA9280712C
:103B5400665D554E4944403C383533302E2C2A2876
:103B6400272524232221201F1E1D1C1B1A1A191865
:103B74001817178181818282838384858687898A45
:103B84008B8D8F90929496989B9D9FA2A4A7A9AC8D
:103B9400AFB1B4B400010203040405060708090A1E
:103BA4000A0B0C0D0D0E0F0F101111121313141418
:103BB400151516161612BD2812BBB6E4F5F7C2B2D7
:103BC400C2B2E5F7D2B264C022203D07123BB970FD
:103BD40003D23D22056D056D12BBB67D008DF7C283
:103BE400B2C2B285F71F8DF7C2B2C3E5F79573F57C
:103BF400188DF7C2B2C2B2E5F79574F5198DF7C204
:103C0400B2C2B2E5F78DF7C2B2C3E5F79576F51AFD
:023C14008DF72A
:103C1600C2B2C2B2E5F79577F51B8DF7C2B2C2B252
:103C2600E5F78DF7C2B2C2B2E5F7F51E8DF7C2B25F
:103C3600C3E5F7957AF51C8DF7C2B2C2B2E5F78DEA
:103C4600F7C2B2C2B2E5F7D2B2543F30E50244C081
:103C5600955EF51D156D156DE51024784001227EE3
:103C660000AF55EF30E7011E0512E51FA2E592D51C
:103C7600400EE515951EF515E5149400F514800B18
:103C8600E515251EF515E43514F5147800E51E60D6
:103C96000620D50318F404C39FF5F0E89E30E7012B
:103CA600220513E5F0A42517F517E5F03516F516E8
:103CB60022303D03D23D22123BB960F8123BB96077
:103CC600F3E546600A123BB960EA123BB960E505C6
:103CD6006D056D056D12BBB67D008DF7C2B2C3E5ED
:103CE600F79573F5188DF7C2B2C2B2E5F79574F57C
:103CF600198DF7C2B2C2B2E5F78DF7C2B2C3E5F7C6
:103D06009576F51A8DF7C2B2C2B2E5F79577F51B2F
:103D1600D2B2156D156D156D2230742412BDF0C228
:103D26003D75101E123CB7203D167902123D8B40A0
:0A3D36000CA806A907123A36400354
:103D400012DE28D510E422200F4030123D2006CF8D
:103D5000304806200C03204FC6E5467902601479EE
:103D60000614600F791614600A79361460057976A6
:103D700014701712BDF0C23D7896123CB7203D0A70
:103D8000123D8B400312DE28D8F022532CF8AB18DA
:103D9000E519FC339262123DDDBC002BEB89F05338
:103DA000F00784FF24DF401FAB1AE51BFC33926150
:103DB000123DDDAA471252A2BC000CEB89F053F071
:103DC0000784FE24DF5002D32274562F2062029F04
:103DD0009FFF741F2E3061029E9EFEC3225003126D
:103DE00054FEE920E40122C3EC13FCEB13FBE920B1
:103DF000E50122C3EC13FCEB13FBE920E60122C32F
:103E0000EC13FCEB13FB2274542F2062029F9FFFE4
:103E1000741D2E3061029E9EFE2279B4203249200C
:103E20001D46EFB506009260AC06AB074004AC0738
:103E3000AB06903E69EC2304938BF0A4A9F0EC232D
:033E4000938BF071
:103E4300A429F9903EC993C9903FC9E52C5407931F
:103E530013E95001F4903FD1F9E52C5407932975E8
:103E6300F0B484A9F022FFFFFFFF7FFF55553FFF0A
:103E730033332AAA24921FFF1C711999174515552C
:103E830013B1124911110FFF0F0F0E380D790CCC1E
:103E93000C300BA20B210AAA0A3D09D8097B09247D
:103EA30008D30888084207FF07C107870750071C84
:103EB30006EB06BC06900666063E061805F405D119
:103EC30005B0059005720000000000010101010129
:103ED30001010101020202020202020202030303C0
:103EE3000303030303030404040404040404040594
:103EF3000505050505050505060606060606060667
:103F0300060607070707070707070708080808083B
:103F13000808080808090909090909090909090A12
:103F23000A0A0A0A0A0A0A0A0A0B0B0B0B0B0B0BE7
:103F33000B0B0B0C0C0C0C0C0C0C0C0C0C0C0D0DBF
:103F43000D0D0D0D0D0D0D0D0D0E0E0E0E0E0E0E97
:103F53000E0E0E0E0F0F0F0F0F0F0F0F0F0F0F0F72
:103F6300101010101010101010101010101111114B
:103F73001111111111111111111112121212121228
:103F83001212121212121213131313131313131305
:103F930013131313131314141414141414141414E4
:103FA30014141414141515151515151515151515C3
:103FB30015151515151616161616161616161616A3
:103FC30016161616161600FFFF00FF0000FF002E40
:103FD300B5875B2D5A88E537607414603EB4025888
:103FE3007F347E12E5342437400810644B90A323BA
:103FF300801AF890412312D4FBE824FD501179A1D3
:10400300E77E0590A13320E70390A13C0F803A247B
:10401300040F7E2312D4BCD26480627F357E02E516
:10402300342437401410641090A02530081B1276F6
:104033000A7E1A90A322801122700590A03980096C
:10404300909C9A200C03909CA612760A80C97F3517
:10405300E5342433402A2404501B7D0F600C7D1E5D
:104063001460077D3C1460027D78ED305D02C3135C
:104073007E2B12D3847E0090A03A12760A02DD0DC5
:104083007E0524FE5005909E858009909C7D200F1F
:1040930003909C8912760A80E4E546604A14603CEA
:1040A30014602E14602014601290A55D205D419071
:1040B300411C7F367E3412D4FB803C90A55D305D7D
:1040C3000390A559802A90A559305D0390A555808A
:1040D3001F90A555305D0390A551801490A55130D4
:1040E3005D0390A54D800990A549305D0390A545DA
:0240F3007F3616
:1040F5007E3312763D7E3C7422305D02748302D499
:10410500CF305D0890A535305BE4800690A53D2055
:104115005BDC90A53980D70508B28D8DB5BA09103D
:1041250006000A10F248922492249224F2480A10BA
:104135000600305E5220434F20284CE55864FF604E
:1041450046E54824F640407F3FE55804F9C23D1254
:10415500418D12109B601AB404047401D23D75F0B0
:1041650003A4243CB5070A7E3A303D027E3612414F
:104175008F0F0F0FD9D7E55975F003A4243EFF1211
:10418500418D0F0F12418D227E3D12DE280EBE405D
:10419500F922C248C249305E56202853E55864FFCB
:1041A500604DE54824F6404712109B6042D249B461
:1041B5000402803B1465597036D248304E31E559BA
:1041C5006558602B3074281241FA120D54E5BFB4BE
:1041D500011DE5BD20E618202416205F129006E497
:1041E500E0700CA3E024CE40062425500205592298
:1041F500305FFC80E820113375A7009006E4E0707D
:1042050028A3E0302402F404305F02F4042404F906
:1042150024F74015E924FC4003D26C2270012230BA
:104225006C097536A7D22ED22FC26C22305E0830AB
:104235007405E558B4FF0122C244C24D780075A744
:0B4245000475830712457988188A1E53
:104250008E168F17C23EC23BE54824F65003024338
:104260000AD23EE55860F7E8655970F22048EF122F
:1042700043BF30D13BAE16AF17A818E546705512B4
:10428000080DE5CC49604DD244E5CC7033E924CD2E
:10429000402EE975F038A4ACF0FB12548D12548D09
:1042A000EBFDF511124320304D2CC206C23B80437A
:1042B000E546705C12080DE5CC7005E924CD505040
:1042C000124E8475A704758307A8181245798A1EB3
:1042D0008E168F178037120D54E5BDA2E0B3923BC6
:1042E0005011307428123A364026A907A806D20683
:1042F00012CA1012433C12433312437C89078806CA
:104300001E1F90457412D4FB800630D10312435413
:10431000A81808C3E55898400302424375A7002235
:1043200074562F2062029F9FF9741F2E3061029EE7
:104330009EF822E51865586001227D057A00EA1290
:10434000DCAD12DDAB0A0AED24F240020A0AEA24CF
:104350004C50EB22AE16AF17123E071E303E021E27
:104360001EE51E12D49DEE2404FEE51212D49D30EB
:084370003E09EE2404FEE513F2
:1043780012D49D22E5186558603CC001C000C012E7
:10438800C0138518101244F7D013D012D000D001F2
:10439800E510303B07C39570500224B412DCAD2001
:1043A8003B07AE16AF17124320E5112402FD7A062B
:1043B80012DDAB1DDAFA2212109BB40457E87054D0
:1043C800120D72E5BD604D78C6A61308A61208A6A0
:1043D8002C12C7BD75A7047583077510011259CA39
:1043E80012C7B715101259CA1255E48E628F63129C
:1043F800566C8B1C8A1B12C7C320320E1244A7208E
:104408003B08D24D12660712441D78C686130886EB
:104418001208862C22120D72AABD7C027BB312529E
:10442800A28C128B13AA1DA91F1252E4A91CA81B47
:1044380012541D8C1D8B1FAC12AB13AA19A91A128A
:1044480052E4A91CA81B12541D8C198B1AE56E2561
:104458001AF9E56D3519F8C3E56E951AFBE56D9502
:1044680019FAC3E554951FFDE56F951DFCE5542524
:104478001FFFE56F351DFEE52C23652C30E206ECA9
:10448800CEFCEDCFFD75A7049005C2E8F0E9F0EC8D
:07449800F0EDF0EAF0EBF09B
:10449F00EEF0EFF075A70022D23BC3E5649573C52C
:1044AF00659574F564E5669575600404600822E50A
:1044BF006424E0500822E5642420400122C3E5670C
:1044CF009576F567E5689577F566E56995786009FE
:1044DF0004600122E566F48002E5668562F0A4744B
:1044EF00E025F04002C23B2212C7BD75A7047583B9
:1044FF00071259CA12C7B705101259CAC02C125940
:10450F00E3D02C891002C7C330125120064E780019
:10451F0075A70475830612457930D139123E07E528
:10452F004624FE500A0E0F90456F12D4FB8026EAE8
:10453F007007745D12D499801C75F06484ADF070AF
:10454F000FED75F00A847008E5F00E12D48A80051D
:10455F001EED12D41F08C3E55A9850B475A7002258
:10456F00030340A040030340E040D2D1E8C4F582EA
:10457F00E0FA79731245D230D146AF06532CF8EDDD
:10458F00BFFF07F40460390FD262BF003312470632
:10459F00402E79761245D230D126E5822403F5825A
:1045AF00E0F512E0F513EEA2E713FEED13BEFF07E1
:0A45BF00F404600C0ED261BE000689
:1045C900124723400122C2D122C3E09709FDE09797
:1045D90009FEE097600904700AEE30E7068007EEED
:1045E90030E703C2D122E546600E14600BF9EDCE27
:1045F900A2E713CE13D9F8FD227C007B44E546607F
:10460900207C007BCC1460197C017B981460127C9F
:10461900037B3014600B7C067B601460047C0C7B8C
:10462900C08C148B157AE9125279A84712541B8C45
:10463900168B1775C70075C6047510DF75B901E5C6
:10464900BC20E76FF51385BD1205C605C675B9010E
:10465900532CF8C3E5BE9573FBE5BF9574FC05C6FD
:1046690075B901E5BC9575FD5005D262125506C3B1
:10467900E5159BE5149CE49D40338C198B18C3E523
:10468900BD9576FBE5BE9577FCE5BF9578FD5005B0
:10469900D261125506C3E5179BE5169CE49D400DB2
:1046A9008C1B8B1A1246CDE5322428401305C6E52A
:1046B900C68006E5C62404F5C6700205C7D51001F3
:0F46C90022024645AE19AD181245EFED12470615
:1046D800AE1BAD1A1245EFEE13ED13124723123E2F
:1046E80007E54624FB50080E0F90457402D4FB1EC4
:1046F800E51312D49DEE2404FEE51202D49D75F054
:10470800067FFDA946B9000575F0027FFF84C5F054
:104718002F500205F0C5F0FF24DE228547F0A430B3
:10472800E70205F0E5F0A946B9000280050475F036
:104738000384FE24E022E537B4020122E537700243
:10474800D23964027002C239E53724FC799EE760E9
:1047580005640B600C22D27E20081E401C107F10BE
:1047680022D27F2008134011107E012275370122C2
:104778007537002039037537022275F9FF75FB007C
:10478800800E75F9FF75FBFF801C2053F51247C09A
:10479800759E85759D2D80141247C0759E84759DE4
:1047A8002D80091247C0759E83759D09C2AC759806
:1047B80052C26DC26EC26F221215B1C253E4F5F92E
:1047C800F5FB30340215FB22D2A47F3212DE05C27B
:1047D800A412D98412DD0D12DDEEC214C2151247DF
:1047E8008274C012DC3874A312DBF5748F12DBF507
:1047F80012481674C012DC3875A7049048207F1040
:10480800E49312DBF5DFF912481675A70022E538A4
:0548180012DBF574CA7B
:10481D0002DBF5A29494859C8080808080818380CA
:10482D00819E8075A60A1247E2D269D2ACE5A62414
:10483D00FA500C306DF712DB8AB4E0F1124878C2F1
:10484D00ACC26975A6FF22D21EC274C273E4FDF517
:10485D0071F570C22D124782D2AC12DB8AC5F07091
:10486D0005DDF7C2AC22C5F0B4E0EFF538E4F53262
:10487D0012DB85A2E19273A2E2927475A7049004F3
:10488D00B4F012DB85C2D1124A5F20690330740B7C
:10489D008D758E748F73E514C4F57D124ADF124A3F
:1048AD005F20690330740C8D788E778F76E5142533
:1048BD007DF57D124ADFD2D1124A5FEEF0F55DEF44
:1048CD00F0F55C207303E4FEFF79BCA70609A7078A
:1048DD0012DB857D0A124ACC8F71EE60037571FF74
:1048ED007D14124ACCC22DED24F150010F240A5033
:1048FD0002D22DBFB4027F008F7012DB85F05407FA
:10490D00C52E54F8252EF52EE571700EE4F571F5D2
:10491D0070C22D9004BFF0F0F0F012DB85E5386029
:10492D0009D21EC27412AE3B8005C21E12AE3712E2
:10493D00DB85B4E1FA75A7049004C412DB85F0128F
:10494D00DB85F0F53A12DB85F0F53B12DB85F0F5F2
:0B495D003C12DB85F0F53D12DB85F01D
:10496800F53E12DB85F0F53F12DB8512DB85B4E2FC
:10497800FA12DB85F07E0C12DB85FF12DB8512DB79
:104988008512DB8512DB8520E1027F00EFF012DB68
:1049980085DEE412DB85B4E3FA12DB85FF12DB85E2
:1049A800CF60027F7F9004E4EFF0E4F012DBB59073
:1049B80004D8124ACC12DB85B4EAFAC2AC75A70453
:1049C8009004DAE561F0E560F0E55EF0E57AF0E59F
:1049D80079F0E52EF0E55FF0E57BF0E551F0207425
:1049E80012E4F571F5709004B4F09004BDF0F0F0A5
:1049F800F0F0F075A70078ABA63A08A63B08A63CED
:104A0800120D68E5BF253D240C75F0188478AEA614
:104A1800F0186005640260182216E670121816E68F
:104A28007004760C181678ACE6904A529308F62271
:104A38000618E608904A52930466700D7601180627
:104A4800E6640D70047601180622001F1D1F1E1F44
:104A58001E1F1F1E1F1E1F12DB85FC12DB85FD1289
:104A6800DB85FE12DB85FFECA2E692E7921713FCCA
:084A7800ED92E713FDEE92E759
:104A800013FEEF92E7301701F4F513ECA2E713FCE5
:104A9000ED92E713FDEE92E7301701F4F512ECA268
:104AA000E713301701F4F510ED92E7301701F4F534
:104AB000111254AE20D10E8C1C8D1D8E1E8F1F1214
:104AC000B2431254AE30170312B21D2212DB85C35B
:104AD00013FEF012DB8592E7FFF07C00025384ACFA
:104AE0001CAD1DAE1EAF1F30170312B21DECF0ED52
:104AF000F0EEF0EFF022124AFF0202C612BBF5C23E
:104B0000101248337F5A7E0590A33212760A12DDC6
:104B10000DD214D215C255122C2F789F76800876AC
:104B20000012BC3512323D7570FE853A71853B72BC
:104B3000853C73853D74853E75853F7612BC941225
:104B4000323D7570C0757B03757A54E4F57FF57E50
:104B500012BC94751421751348755F01757B00753F
:104B6000750475745275780175776CE4F57DF551AF
:104B7000757F0190DF5C85836E85826DC23D124B2F
:104B8000DD851C1D75A6FF305505C221022DEA12D8
:104B90004BDDE572A2E59275A2E79277D274D273EB
:104BA000E51275F008A4AEF0FF2075031254EE1262
:104BB000C70D12C756124C60E51C251D13F57185F3
:054BC0001C1D12BC0DDC
:104BC50012BC65757F02E56A70B57F5A7E2FE54197
:104BD50012D38412DD0D80A7856E83856D82C25543
:104BE5007873124C417876124C41E493F570B4B465
:104BF50002D255A3E493F51CA3E493F512A3203D3B
:104C05000FA97BE493F57BC399502A20E702055F42
:104C1500A385836E85826D103D16D23DE582240500
:104C2500F582E43583F583E493F52654F0F5722295
:104C3500E526C480F630E7D8155F80D48601E49375
:104C4500F6A308C399500A20E70606B6000208062F
:104C55002230E70616B6FF0218162230750DE51349
:104C65002579F513E43514F514800DC3E51395790D
:104C7500F513E5149400F514AE14AF137C007D0A0A
:104C85001253848E5E8F7A22124D22851617203D8F
:104C950001227F5A909B8E1275F87F64E516640495
:104CA500700C909BA612763B12DD0D02DDE8909B01
:104CB5009A1275F87F6E7E0890A52512760A121D48
:104CC5004612DD0D7515B87514047F6E7E20C2245D
:104CD500A815E82404F9C23DE7124D6A203D06E611
:0A4CE50012D4CF8008E6128368E8BD
:104CEF00A815F60515EE2406FED514DA851716124B
:104CFF001D9412DD0D10000510018D80F878B8128B
:104D0F000D7C86BC0886BD0886BE0886BF124E2C59
:104D1F0012DEE3120D7CC23D75160078B87F4B7E14
:104D2F000890A52512760A7E20E5BC12D4CF124D2D
:104D3F00617E26E5BD12D4CF124D617E2CE5BE12E9
:104D4F00D4CF124D617E32E5BF12D4CF124D610226
:104D5F00DD0DF608080808F618181824D050052499
:104D6F00F64001220516D23D2275C70375C6FE1205
:104D7F007576124E2C75C6FC75BC2675BD6475BE56
:104D8F00A975BF70124E2C75C6FB12757675BC6473
:104D9F00124E2C75C6FA75BC1475BD1475BE007510
:104DAF00BF0C124E2C75C6F975BC4E75BDBF75BEC6
:104DBF000075BF19124E2C75C6F875BC0A75BD7EED
:104DCF0075BE0075BF01124E2C75C6F775BC017507
:104DDF00BD2375BE4575BF67124E2C75C6F675BCE3
:104DEF000275BDAB75BE0175BF01124E2C75C6F5B0
:104DFF0012757675BE0275BF0A124E2C75C6F41267
:104E0F00757675BCE1124E2C75C6F3127572124E83
:104E1F002C15C6124E2C15C6124E2C15C675B9057B
:104E2F0075B90222751500127C6F75B901E5BC6466
:104E3F008160031275590515E515242050E975C7D2
:104E4F000375C68075B90505C6E5C6241C50F51255
:054E5F004E64027AC55B
:104E6400E4F5C7F5C6742612757775BD4E124E7EED
:104E7400124E7BE4124E7B127577124E2C05C6221D
:104E840020740122D24475A700758307E559C454E0
:104E9400F02407F582E0F51A244C40E7A3E0F5126C
:104EA400A3E0F51312080D8938120D54E5BDA2E0F4
:104EB400923BE51A40069570500224B4F51A203B43
:104EC40005D20612CA10E51A124FE7E5152437F584
:104ED4001DE43514F51CE5172437F51FE43516F5E4
:104EE4001E85CC12853813AC12AB137A0412526BA4
:104EF40075380124FA401A05382402401405382470
:104F040001400E05380538240140060538053805EA
:104F140038C3E51A945A500224B4F51AC23BC23C71
:104F2400C23D751B00A23B823C406D203B2CE51A20
:104F340075F008A4951BFBE5F0303D049401800254
:104F44009400FC5008EB24A0FBEC3405FC124FEE5B
:104F5400124F9D923B4003124FC0203C2CE51A7522
:104F6400F008A4251BF9E4303D010435F0FAE99476
:104F7400A0FBEA9405FC5004AB01AC02124FEE1204
:0F4F84004F9D923C4003124FC0E51B2538F51B93
:104F93005094203D04D23D808D22E51F2517FEE568
:104FA3001E35167016EE24914011E51D2515FFE5FB
:104FB3001C35147006EF2491400122D3228E027C0B
:104FC3008A7B3B125279ED2402FE8F027C8A7B3B63
:104FD300125279ED2439FF02DE281255D78031129F
:104FE30055CA804675F008A4ACF0FB751900C3EBF5
:104FF3009468F9EC9401FA40080519AC02AB0180FE
:10500300ED8C108B11531903E51920E0CD1255CA0D
:10501300125042AF05E51924FE50031254EE8E16CA
:105023008F17E51920E0B81255D7125042AF05E5A6
:10503300191460061460031254EE8E148F1522ACFB
:1050430006AB07AA12A9130252E412512F203D49BD
:1050530074857F227E0812D4CF7E0830173CAC1EA5
:10506300AB1FEB2418EC34FC402F12524AE51B60B3
:10507300077F207E0812D4EA7F207E10E51A12D41F
:10508300EA7F237E17742E12D4CB7F207E1BE51B71
:105093007011E519C2E012D4EA227F207E0E740A51
:1050A30002D4EAE51975F0058475F005A402D4EA83
:1050B30012512F203D5E74857F227E3A12D4CF3069
:0450C3001753AC1EB5
:1050C700AB1FEB2418EC34FC4046EC7033EB249C0C
:1050D700402E7E2D12512112548DC0E07F2A7E2E44
:1050E700EB12D4EA7E39D0E0C2E012D4EA7F347EF4
:1050F7003712DE281E12DE281F12DE280E02DE28D7
:105107007E3012512112548DEB7F2A7E3112CFA6A9
:10511700227F2A7E39740A02D4EA7F2912DE580FC9
:10512700BF34F90EBE40F322D23D301266120D5E37
:10513700E5BDF51C75F00AA4F824E15002781EE4D9
:10514700FCFBFEFFC23D12BDF012519B203D44D82F
:10515700F8751DCEE51C146009751D9C1460037558
:105167001D6AC217EC30E705D2171254FE8C018B6B
:1051770000E9487003D23D22EE7008EF251D400379
:10518700D23D22AC06AB077A1C12527912541D8C01
:105197001E8B1F22203D07123BB97003D23D22050B
:1051A7006D12BBB6E4F5F7C2B2C2B2ADF7F5F7C2FE
:1051B700B2C2B2E5F7FAD2B230E4E3ED2FFFE43E34
:1051C700FEE56D2408F56D12BBB6E4F5F7C2B2C271
:1051D700B2ADF7D2B2EA30E508EB2DFBEC3400FCB8
:0A51E70022C3EB9DFBEC9400FC22B8
:0100030055A7
:10DF5C0069FC362E06FD69FC372F071169FD383038
:10DF6C0007FD69FD3931061169FE383107FD68FE80
:10DF7C003732091168FF373008FD68FF372D07115C
:10DF8C006800362909FE680036290C116801372B08
:10DF9C000CFF6801372F0A116802383009FF68023C
:10DFAC00372E08116803372C0AFE6803372E081128
:10DFBC006704373208FE67043633091167053535B7
:10DFCC0005FF6705353303116706362F02FF670619
:10DFDC00362B05116707362B07FF6707352F051101
:10DFEC006708353104FF6708332E0511670931289E
:10DFFC000700670931250A11670A35240B01670AE6
:10E00C003A240A11660A3C210801660B3D1E0B11CD
:10E01C00660B3D1E0C00660B3D200A11660C3B2165
:10E02C000CFF660C39220E11660C37231100660D9D
:10E03C0036240D11660D34260F01660E3226111191
:10E04C00660E32251401660F35251311660F37271E
:10E05C0016016610392918116610392B1502651135
:10E06C00392D11116511372E0C026512332F081141
:10E07C006512312F07026513302C0A1165132D29F7
:10E08C000E0265132A271011651429270E02651438
:10E09C002C290C1165153129080365153726071134
:10E0AC006515321F09036516411B09116516411CC4
:10E0BC0008036416461F081164164D2105046416E6
:10E0CC005922031164166425040563156A2407118B
:10E0DC0063156D23090663156C230D1163156C25EF
:10E0EC00130762146E2B151162146E2F1406621333
:10E0FC006E30161162136E30150761136F311211E9
:10E10C0061126F350F0761126F380D116011723A81
:10E11C000A086011763F0611601079420209600FFF
:10E12C007A3A0533600F7832040A5F0F742C01338E
:10E13C005F0E722B030A5F0E732E08115F0E743084
:10E14C00050C5F0D722C02135E0D6C2B010C5E0D19
:10E15C00622C05315E0D5F2B030D5D0D5E290833BE
:10E16C005D0D5F23030B5D0D5F1B01335D0D5A16B7
:10E17C00020A5D0D521B00115C0D4D26000C5C0E4D
:10E18C00462802335C0E3926040C5C0F2C2B08330A
:10E19C005C0F23320C0F5D0F172E0A335D0F0C2E04
:10E1AC0009105D0F043507335E0FB23C080F5F0F8B
:10E1BC00AB4209335F0EA43E070F5F0EA2430B3335
:10E1CC00600EA746120B600D9F490C73610C9C49A5
:10E1DC000F0C610B97460973610B8B440A0C610A97
:10E1EC008B420B336109843A080C6108823A043380
:10E1FC0061087934030C60086F2F063360086228BD
:10E20C00050C6008572505336008511F040D5F0885
:10E21C004E1B05335F08491B090D5F094120103760
:10E22C005F0938270D0D5F0A302F06335F0B2B3239
:10E23C00070F5F0B282F0A335F0B262E0E0E600C78
:10E24C0023361137600D1F3F160F600D18411277E2
:10E25C00610D0F320A13610D042B0633610D022E72
:10E26C00040E620D043A0231620E0343050D630D78
:10E27C00B1470113630DA94A000B640CA14D0511A4
:10E28C00640C9B44070E650B99490911650A944768
:10E29C00090D65098E49021365088848060D650845
:10E2AC0081400E336407793B130F6407722F187784
:10E2BC0064076D231A106407692911776407651CBC
:0DE2CC00080F63075D180B33630751190D30
:10E2D9000D630746220E336308402B110F6308387C
:10E2E900291837630932271B0D6309312B1477620B
:10E2F9000A372C0F0A620A3C280973620A441E0B6A
:10E309000C620A48150E33620B46190C0A620B4758
:10E31900260D33610B4C280C0B610B54251037610A
:10E329000B5E24170C600B63291A77600A66361492
:10E339000A600A68390B735F0A6C2C100A5F09724C
:10E349002015775F097422120A5F0873300F775F0F
:10E35900087639140A5F077D3816775F0785370F06
:10E36900095F068D3B0D735F058B4410075F048BB6
:10E37900490C735F048E3F0C075F03863604335FD5
:10E389000394280708600299300E1160029E400527
:10E39900076102A34A0C336101AA4810086201B15E
:10E3A90042127762020131150A6202062B13776362
:10E3B900020830110C63020B361277630310331114
:10E3C9000C6403182B147764032223110A640426AE
:10E3D90023107764042226110A64051C2715776423
:10E3E900051D251508640521271277640628270FBE
:10E3F9000764062F1D11776406350F140764063E5E
:10E409000A19776406401216086407431B117763DB
:10E41900074A22120663075228127763075A2713FD
:10E429000662075E2314776206612011076206649B
:10E439001E0E7362066A1E0E076206742110376289
:10E44900057828130661057A2F157761047A332038
:10E459000661047A301B7761037A281B0761037F01
:10E4690023187761028429160661028832177761B9
:10E47900018D371305610193340C7362009A2E09DB
:10E489000562009D2E043362009D370C0663FFA0D0
:10E4990040103763FFA844140564FFAF4612776440
:10E4A900FF014511056500043F12776500053E101F
:10E4B900076600073F117766000B430D07670110D8
:10E4C9003D117367011539120767021A321277670E
:10E4D900021A2C12076702192C107768031B2E0FDA
:10E4E9000668031F2C117768042729100468042E75
:10E4F9002A0F776705322F130467053330127767C0
:10E5090006362D140567063B291677670643231B34
:10E51900046706471E16776607491E150366074CEA
:10E529001B157766074C2217046607522214776574
:10E53900075B26150265066229157765066D291799
:10E549000165067529137765057D281A0265058217
:10E5590028187765047F1F160265048F2A117765CD
:10E5690003953211006602993D157766029C401C9D
:10E57900FF6602A13E1F776701A43F1CFF6701A741
:10E589004314776801AB4710FF6901B1490F7769F7
:10E5990001024911026A0207490D736A020B480C0C
:10E5A900056B030F480B336B03144A0D026B0419F7
:10E5B9004914376B051F491CFE6C06224824776CE9
:10E5C90006233F21FC6C07203023776C0721272184
:10E5D900FC6C07262420776C08292812FC6C082873
:10E5E9002C0F776C0927230CFF6C09251802316C55
:10E5F90009350F05FC6C094C1401116C09561D01F4
:10E60900FC6B095F2003136B086B2108FB6B087413
:10E619002509336B08772507FC6B0778210D336BC8
:10E62900077A1E0AFB6B077F220C336B06832E0ABF
:10E63900FA6B05853C09336B0489410EF96B048C2F
:0DE649003E10376B038D3C0FFA6B038D40C4
:10E6560013776B02904112FA6C01934110776C01AB
:10E66600984410F86C009B471A776D009F461EF879
:10E676006DFFA24519776EFFA14019F86EFFA640FF
:10E6860014776FFEAA4417FA6FFEAF4A127770FE30
:10E69600B34D18FA70FF024B1B7771FF054718FD43
:10E6A60071FF0942177772000E4012FD7200163D87
:10E6B6000C7372011B3510FA7201232E1577720244
:10E6C60029321AF872032C371D7772032F3014F88B
:10E6D600720336210F77710346190DF87103502026
:10E6E6000B33710353290EF87003572B143770033D
:10E6F600612712F870036F2911777002793017F7C6
:10E706007001803722777001843D1FF67000883FC4
:10E71600197770FF8D3F11F670FF933D0C7371FEF4
:10E72600973D0EF571FE9B3E0C3372FD9F4310F62E
:10E7360072FDA448127773FDAB4C13F573FDB14F10
:10E74600167774FD034F14F775FE074C127775FEA6
:10E756000A4510F975FE0E400F7776FF124111F843
:10E7660076001745167776001C4614F67601214288
:10E7760017777602263D17F3760229382177760336
:10E786002A3315F276032B3009737604302A07F004
:10E79600760439220A337604472110F07504512590
:10E7A60012777504552416F1750459210F777504EF
:10E7B6005F2111F0740463231477740468240EF245
:10E7C600740370230933740379270AEF74028030C7
:10E7D6000B33740185360DEF74018B3913377400D2
:10E7E600903D1BF075FF94441E7775FF984823EF04
:10E7F60075FE9B46207776FE9F4221F076FEA13F6E
:10E80600177777FDA44313EF77FDA747157778FDB4
:10E81600AA4915EF78FDAD4C157779FDB04D19EE87
:10E826007AFDB34D1C777AFD024E19F07BFD054F3C
:10E836001B777BFE094F24F37CFE0D531D777CFF6F
:10E84600114619F37CFF173F12777C001F3810EF33
:10E856007C00263613777C012B3115ED7C012F2B9E
:10E8660015777C02332513ED7C02392214777C025E
:10E87600402110EE7C0249210B737B02531F0FEBE4
:10E886007B02601E15777B026A2214EA7B017428DC
:10E8960019777B017B2D1AEA7B00833122777B0077
:10E8A6008A3320EB7BFF91371A777BFE953C1FEA74
:10E8B6007CFE983C26777CFEA74621EC7CFD9939A8
:10E8C60023777CFC9A3B1FEA7DFC9A3F1C777DFBF5
:10E8D6009A401EE87DFB9B3F20777EFA9B3F1FE612
:10E8E6007EFA9C431A777EF99E4717E57FF8A04A81
:10E8F6000E737FF8A34A0AEA80F8A548073380F822
:10E90600A94402EA81F8AE46041182F8B24C00E747
:10E9160082F80351021183F8085304EA83F90E4D75
:10E92600061183F914430CEC84FA1A400E1184FB89
:10E93600203F0AE884FC2540061384FC2B4008E6A9
:10E9460084FD3039073383FD36300EE483FE3C2BDD
:10E95600193783FE402A1EE783FE3D25187783FE7E
:10E96600371B16E783FF3114137783FF35170FE440
:10E9760083FF3E220D738200412C15E58200432C55
:10E986001A77820046251BE782004C201577810006
:10E99600552116E581005E2510778100682718E469
:10E9A60081FF72291E7780FF7A2E22E580FE7E3057
:10E9B600277780FE812B22E680FD85251C7780FD4A
:0DE9C600882618E281FC8A2F187781FC8DCD
:10E9D3003821E181FB903F287781FA924025E0813D
:10E9E300FA943D237782F9973C18E082F99A3F1510
:10E9F3007782F89E4412E083F8A347107783F8A741
:10EA03004A0CDF84F8AA4D133785F7AC5214E2851C
:10EA1300F7AF56107786F7B2580DE087F802560223
:10EA23003387F8055002E388F8094C051188F90C7F
:10EA33004E02E489F91052011189FA155004DF8955
:10EA4300FB1D45041389FB233304DE89FB292306BD
:10EA53003389FC2B1F05DE89FC2F23093389FD3302
:10EA6300280ADC89FD3B23103788FD471E0EDD880D
:10EA7300FD511E0E3388FD53200CDD88FD54210B00
:10EA83003387FD57200DDD87FD5C20093387FD5D4E
:10EA93002403DE87FD5B29013386FD592C04DE86C2
:10EAA300FD5D2C093385FD622F0CDC85FD652D0B87
:10EAB3003385FC672908DF85FC6722093385FC6BF6
:10EAC300210CDD84FC72280A3384FB783005DD8455
:10EAD300FA7C37073384FA7E390ADC84F9813B06F2
:10EAE3003384F8843F05DB84F8873F023384F78A55
:10EAF3003C04DB84F78D390A3384F6903908D985D1
:10EB0300F5923F113785F595430FD985F498440A5B
:10EB13007386F49B440AD986F39C440C3386F39C96
:10EB23004507DA87F29C47063387F19E4C0AD9885A
:10EB3300F1A251103788F1A65516D989F0A7571FAE
:10EB4300778AF0A9541BDA8AF0AA4D12778BF0ACBE
:10EB5300460DDB8BF0AC4906338CEFAB4D05DB8CFC
:10EB6300EFA95002318DEEA85209E28DEEA7530EA4
:10EB7300118EEEA75316E58EEDA44A20118FEDA05A
:10EB83004423E28FEC9C4821118FEB9A4A22E090B8
:10EB9300EB95411D1190EA8E391DDF90EA893621EC
:10EBA3001190E9873223E590E9852C2C118FE87DBC
:10EBB3002A26E08FE8762124118FE8662122E08F50
:10EBC300E856221F118EE947201DE08EE9392116F0
:10EBD300118EE9302518E28EEA2D2917118EEB30BC
:10EBE3003213E18EEB333711118EEC373C10E18E8B
:10EBF300ED393E07138DED3B4203DD8DEE3B3E09C0
:10EC0300338DEE3B310DDE8DEE392812378DEF3823
:10EC13002319DC8DEF382A18778DF0372A12DC8D13
:10EC2300F0382214778DF0361B0EDC8DF1361B0C79
:10EC3300338CF1371F0DDB8CF136250E378CF23414
:10EC4300270CDC8CF22A270D338DF31F2A0CDC8D65
:10EC5300F3173409338DF4143A08E48EF4123A0CA2
:10EC6300338EF4103D11EA8FF50E411A778FF50CB0
:10EC73004917EA90F50A50157790F5054F13E79178
:10EC8300F5B24F107792F5AD5408E492F4AB5A0104
:10EC93003393F4AB5C05E893F4A9500A3394F3A4DB
:10ECA300450CE094F3A041093394F29A3A05E295B6
:10ECB300F29734043395F1913208DC95F19E310DCE
:10ECC3003395F08A320CDA95F0872D0B3395EF806C
:10ECD300250EDE94EF73220C3394EF6C2412DD9433
:10ECE300EF6928157794EE6B2812DF93EE69280EEF
:10ECF3007393EE64270DDF93EE5C260B3392EE578E
:10ED0300270EDB92EE5828123792EE5E2610DB9226
:10ED1300EE64240D7391EE6C2108D991ED722304F6
:10ED23003391ED782904D991EC7C320A3391EB7F4E
:10ED33003A08D891EB833D093391EA883C0CD7918B
:0DED4300E98D3B103791E9903E12D792E820
:10ED50009143137792E794420ED792E7993E073397
:10ED600093E7A03901D993E7A63B0A1194E6A83F9F
:10ED70000CD794E6AB490E1195E6AE4F07D695E653
:10ED8000004D011396E6034601D996E6033E0811AD
:10ED900097E7043D0ED997E70740151198E70C4314
:10EDA00012DA98E812460F1198E918490CDA98E936
:10EDB0001D44081198EA243D05D898EB293A03111F
:10EDC00098EB2C3707D898EC2D38093398ED2E3D69
:10EDD0000ADC98ED2E3E0A3398EE2D3F0BDB98EFC0
:10EDE0002C420C3398F02B430ED998F02B3D113761
:10EDF00098F12D3710D898F130340D7398F23433E0
:10EE00000FD698F237330F7798F339331CD597F331
:10EE10003C32167797F43E2F11D797F440280973A8
:10EE200097F4422109D797F4461F0AB396F44B2171
:10EE300008D796F45325083396F45C2505D796F445
:10EE40006723023395F4722503D695F3782B0231AC
:10EE500095F37B3102D695F27E31063395F1832FFF
:10EE600004D695F18A2F023395F0913201D596F0B0
:10EE70009638061196EF9A3F02D497EF9D450213FC
:10EE800097EE9F4704D497EEA247073398EEA64427
:10EE900008D398EEAA430B3399EEAD440CD499EE07
:10EEA000B1400D339AEE013F11D39AEE054512772A
:10EEB0009BEE064A15D59BEE064712779CEF05425E
:10EEC00012D79CEF063E0F779DEF084111D39DEFBF
:10EED000094619779EF00B4718D39EF00D431C7717
:10EEE0009FF10F4015D69FF1114113779FF2134602
:10EEF0000ED9A0F2174A0B33A0F31C4A08D4A0F491
:10EF000023420333A0F42A3305D3A0F53127071198
:10EF1000A0F5382300D29FF53D2702339FF6442900
:10EF200003D39FF64F2808119EF55E2807D19EF562
:10EF30006C2D04119EF4752F01D09EF47C2D0433AA
:10EF40009EF3822B04D09EF3872E05119EF28B3503
:10EF500007D09EF2903D01119FF1954203D09FF0A2
:10EF600094400333A0F09F3F0BD0A0F0A13D0F379A
:10EF7000A0EFA33C0DD1A1EFA43C0C33A1EFA43C26
:10EF80000AD0A1EEA53D0533A2EEA63C00D1A2EE2B
:10EF9000A8390211A3EEAA3C04D0A3EEAD3F05119F
:10EFA000A4EEB24008D0A4EE03410C11A5EE064138
:10EFB0000AD2A5EE08450711A6EF094A05D2A6EF29
:10EFC000094C0111A7EF0A4807D3A7F00B420B1118
:10EFD000A8F00B420DD4A8F00D461311A9F111466B
:10EFE00014D9A9F1173F1B11A9F21E381ADAA9F397
:10EFF00021381811A9F31F3A17DFA9F41839151190
:10F00000AAF4163A1DDCAAF5183C1A11AAF51C3A06
:10F010001AD9AAF61F391A11ABF6203615D9ABF753
:10F0200021341711ABF8203B19D9ABF81E3F17114B
:10F03000ACF91D4011D9ACF91E3F0E11ACFA1F40BE
:10F040000CD6ACFB22410D11ACFC23450FD6ADFC18
:10F0500023490B11ADFD214A0DD6ADFE2047091104
:10F06000ADFE21450CD6ADFF22430E11AE00224568
:10F070000CD8AE01214B0A11AE0220500DD7AF03C0
:10F080001D4F0B11AF031A5109D9AF04174A0D11C7
:10F09000B00418470BDBB0051A500A11B0061C5516
:10F0A0000ED7B1071C560B11B10719470ED9B1087D
:10F0B000173C0C11B208183D0CDCB2091C490E11AA
:0DF0C000B20A1E4E0AD9B30B1D500B11B33E
:10F0CD000C1A5109D9B30C174F0711B40D17490B71
:10F0DD00DBB40D17480D11B50E19490ADCB50F1922
:10F0ED004F0B11B50F185605DBB61017550711B696
:10F0FD0011174C0ADBB61116430B11B711173F0D43
:10F10D00DDB71219430C11B7131A480BDCB8131ADB
:10F11D00450F11B81419410DDCB81418400B11B975
:10F12D001518430DDBB91618470F11B91618490DEF
:10F13D00DBBA1718470A11BA1717450CDBBB1814A1
:10F14D00460F11BB18134C0EDBBC1912510A11BC22
:10F15D001A125007DBBC1A12470B11BD1A10400DC5
:10F16D00DCBD1B10400A11BE1B124509DCBE1C156F
:10F17D00490B11BE1D184A0ADBBF1D1B4A0811BFE2
:10F18D001E1B480CDBBF1F1A470E11BF1F1A490B60
:10F19D00DBC0201B4B0D11C0211C4910DBC0211DF4
:10F1AD00470F11C1221D4711DBC1231C4B0F11C18C
:10F1BD00231B4B0EDBC22419441111C224193D0F20
:10F1CD00DBC2251B3B1011C2261D3F0DDAC2261EC8
:10F1DD00411011C3271D3F12DAC3271C3D0F11C368
:10F1ED00281B3D10DBC4291C401111C4291C450FDF
:10F1FD00DCC42A1C460E11C42A1B4510DCC52B1974
:10F20D00431111C52C184511DDC62C164A1011C617
:10F21D002D174A11DEC62D18491211C72E19471088
:10F22D00DEC72F1A460E11C72F1C4410DFC7301F23
:10F23D00471111C731214B0CDBC832224D0E11C8BD
:10F24D0032224A10DAC83321471111C83420460F33
:10F25D00D9C83520461111C93521430CDBC93623D8
:10F26D003F0F11C937253D11DBC93725400E11C997
:10F27D0038254211DCC93925431311C939254312EB
:10F28D00DCC93A25431111CA3B24400DDCCA3C248C
:10F29D00411011CA3C23400EDCCA3D22401111CA57
:10F2AD003E20420FDECB3E20451011CB3F204714B0
:10F2BD00DECB4021441211CB40213F10DFCB412248
:10F2CD003C0D11CB42234011DFCC42233E1111CC1A
:10F2DD0043202F0EE0CC4319221211CC43122011E2
:10F2ED00E3CC4311250E11CD43132B10E3CD441266
:10F2FD002D1111CD440F2B0FE3CD44092B1211CE3F
:10F30D004404320FE2CE4401360E11CF44B3370D13
:10F31D00E0CF44B3330E11D04401370EE0D0440595
:10F32D003D0D11D0450A3B0CE3D14512330D11D1E2
:10F33D00451A2D0EE3D1461E2B0F11D1461D2E0F52
:10F34D00E4D1471D300F11D1471E320EE3D24821B3
:10F35D00330F11D248233510E2D24923350F11D284
:10F36D004A20360EE3D24A1D360E11D24B1B3410F5
:10F37D00E3D34B1B320F11D34B1B300EE4D34C1B7D
:10F38D00340D11D34C1B3A0DE5D44D1A3B0E11D44F
:10F39D004D1B360AE6D44E1D340E11D44E1E360DBD
:10F3AD00E5D44F1F360C11D5501F350EE5D5501F26
:10F3BD00340D11D5511E340EE5D5511E370C11D516
:10F3CD00521E390EE5D652203B0F11D653223C0F5B
:10F3DD00E4D65423391111D654243710E3D65524CD
:10F3ED00360F11D655253310E3D65626330D11D6CB
:10F3FD005627350BE2D657273A0C11D658273C0F16
:10F40D00E2D75827391011D75927370FE2D75A2786
:10F41D00381011D75A283B0FE2D75B293C1111D771
:10F42D005C2B3C12E2D75C2D391111D75D2C3910B4
:0DF43D00E3D75E2B3C0F11D75E293B0EE399
:10F44A00D75F27371011D75F26360EE3D760273CE0
:10F45A000E11D761284310E3D76229451111D762EB
:10F46A00293F0FE4D763283A1011D763293A11E4E8
:10F47A00D7642A3E1011D7652C4211E4D7662E4272
:10F48A001011D7662D3F11E4D7672F3A1011D768AC
:10F49A002D3B0CE4D7682E3D0711D7692E4204E4B0
:10F4AA00D76A2E470111D76B2E4702E4D76B2D403E
:10F4BA000513D76C2B3503E4D76C2A2B0711D76DAC
:10F4CA002B2909E5D76D2B300611D76E2A3A04E4A9
:10F4DA00D76F28400611D76F283E08E4D77027381F
:10F4EA000C11D87026320DE6D871252F0911D87162
:10F4FA0024310AE9D87221340811D8721B3A08EA71
:10F50A00D9730D420A11D973104909EADA730C4505
:10F51A000811DA730A3B06E8DB74093D0211DB7451
:10F52A000A4003E9DB740B3C0213DC75103406EA6B
:10F53A00DC7517350333DC761A3F06EADD771C469D
:10F54A000433DD771F4001E8DD7824360731DD78A2
:10F55A002C3206E7DC7933320413DC79373409E7D5
:10F56A00DC7A3A340C33DC7A3C3508E7DC7B3D370D
:10F57A000233DB7C3C3A05E7DB7C3C3D0333DB7D35
:10F58A003B3A04E7DB7D3B320331DA7D3E2D09EA63
:10F59A00DA7E43270D11DA7E4D230AE9DA7E5726F1
:10F5AA000B11D97D5E2C0BE9D97D61300C11D97D07
:10F5BA00632F08EAD87D662F0511D87C683005EAE2
:10F5CA00D87C6D330611D77B733608E9D77B7C3834
:10F5DA000511D77A853A04E8D8798B3B0711D8798F
:10F5EA008E3809E9D8788F371011D878903B0BE814
:10F5FA00D87791420D11D976954A08E7D976984974
:10F60A000411D9759D4008E8DA75A23A0B33DA7508
:10F61A00A53C0AE8DB75A8430031DB74AA4603E976
:10F62A00DC74AF460213DC74004A02EADD75054C4D
:10F63A000333DD75084D00EDDE75084B0533DF76C3
:10F64A00064902EDDF76044A0131E076044902EA0E
:10F65A00E076044C0513E176045006EAE176014DA2
:10F66A000D33E276B1450FEAE276AD3F1077E375E6
:10F67A00AB3F0DEAE375AC430A33E475AE4604EAE0
:10F68A00E475B0400131E575B23908EAE575013C27
:10F69A000611E675054607ECE6760A4B0311E7768E
:10F6AA000F4604EEE777163B0611E778203405EC9F
:10F6BA00E77827350611E7792D3409ECE7793234F2
:10F6CA000B11E77A3B260AECE67A45250B11E67A16
:10F6DA004D230BEAE67A56250711E67A5F270AEAEE
:10F6EA00E579672A0C11E579731F0AEBE578792E1B
:10F6FA000811E578843302EAE5778D3B0313E67651
:10F70A00954104EAE676993F0733E6759A3801EAA5
:10F71A00E67595310531E6748F3202EAE6748E3564
:10F72A000111E773923301EAE77398310413E77220
:0AF73A009D3304EBE872B4370911A7
:00000001FF
